:020000040000FA
:10000000506F0020D900000009AC0000E3000000A0
:1000100000000000000000000000000000000000E0
:10002000000000000000000000000000E5000000EB
:100030000000000000000000E7000000E9000000F0
:10004000EB000000EB000000F5C70000EB00000033
:100050000D190000EB000000EB000000EB000000B9
:10006000EB000000EB0000003DDA0000EB000000B8
:10007000EB000000EB000000EB000000EB000000D4
:10008000EB000000EB00000000000000EB000000AF
:100090001952000071220000EB000000EB0000008C
:1000A000F9150000EB000000EB000000F114000067
:1000B000EB000000EB00000045350000EB00000005
:1000C0000448854600F0E4FD004800472907010088
:1000D000C046C046506F002004488047044800478F
:1000E000FEE7FEE7FEE7FEE7FEE7FEE789D8000051
:1000F000C100000030B50B4601460020202201243B
:1001000009E00D46D5409D4205D31D469540491B4B
:100110002546954040191546521E002DF1DC30BD94
:1001200070B500242546002801DA01244042002948
:1001300001DA01254942FFF7DDFFAC4200D0404221
:10014000002C00D0494270BD0549064A086850435A
:10015000054A8018086040087047014908607047E8
:10016000740700206D4EC6413930000038B5044692
:10017000C0681821401E4843A16840183C214843EC
:10018000616840183C2148432168451860690C218A
:100190004843216940186921C900401A3021FFF7FE
:1001A000BFFF114A50434219084600921A2902DB48
:1001B0000E49511800910C21FFF7B2FF0C4A504331
:1001C000009A801800900B4806E0491E425C074BDD
:1001D0005A43009BD21800920029F6DC214668465B
:1001E00000F07CFC009838BD801F8607805101001C
:1001F0008033E1015125010003460B439B0703D0E7
:1002000009E008C9121F08C0042AFAD203E00B78DB
:100210000370401C491C521EF9D27047D2B201E053
:100220000270401C491EFBD270470022F6E710B551
:1002300013460A4604461946FFF7F0FF204610BD54
:1002400030B505462A460B4610781C78521C5B1CBC
:10025000002801D0A042F7D0002C03D0002802D003
:100260006D1CEFE7284630BD0321001D401E0378BA
:1002700012021A43491EF9D510467047034610B5BD
:1002800008330722040E090221435B1E1C7800027A
:100290002043521EF6D510BD034603220870000A03
:1002A000491C521EFAD51846704770B504460D46D3
:1002B000072310700E06000A3043090A521C5B1E09
:1002C000F7D52046294670BDF8B502464A40D40FFE
:1002D00042004B0052085B089A4202D2024608468E
:1002E00011464A0023D0C30D4A00DDB2120EAD1AEA
:1002F000202D35DA49020126490AF6058A19002C13
:1003000000D0524220214F1B1146B9402A411018FB
:10031000C20D9A4221D0002C17D0012D08DCDA053D
:10032000801AD20F8019D207DBB200F019FCF8BD99
:10033000DA05801A012340001B06C01880185A42B3
:100340008018CA0F1043490007E04908C20711434B
:10035000DA05801A80194008801800F0F9FBF8BD12
:1003600061000122511A001BF7E70122D207514018
:10037000AAE70122D2075040A6E7024670B54A40DC
:10038000D30FDB0740002DD04A002AD0010E140EF7
:10039000000212020919400A520A8418E5010446B3
:1003A0005443000A120A2E045043A4194219200C87
:1003B000C543AA18120C0125AD03521C5219120490
:1003C0007F39240400D0521C104301D44000491E40
:1003D000C2B20C06C0092018401C4008802A02D076
:1003E00003E0002070BD40084000002900DA002032
:1003F000184370BD70B502464A40D50F40004A0010
:10040000ED0740085208002814D0002A12D0C40D6D
:10041000D30D41020120C0055202490A520AE41AD2
:10042000091812187D34914201D3641C00E0490080
:10043000002C01DA002070BD0023914201D3891AFB
:100440000343400849000028F7D100290AD091420F
:1004500002D10121C90705E0914201D2012101E049
:100460000121C943E005C018401900F071FB70BDBF
:10047000F0B507460846584087B0C00F04904800C2
:100480000E46590040084908BC1A884105D2384632
:1004900031461E4617460B46024658004008104398
:1004A0004DD0300D039040055900400D490D059089
:1004B000401A0290402873DA18030121000B090545
:1004C0000843019004980092002806D01146019A32
:1004D00049420020904100910190029840210A1A5F
:1004E0000199009800F0C6FA05460C466B4607CB0A
:1004F00000F0E1FAC0197141039A0E0D0023D717DD
:1005000056401A467A40164344D0049A002A2DD009
:10051000029A012A039A15DC1205C01A914101269C
:100520003605001C7141D20F059ED207009301923F
:1005300002962A46234600F059FB07B0F0BD384624
:100540003146FAE71605234A0F46B218C01AB741DA
:1005500001210905001C4F4100187F411146181860
:100560007941E20F10436D19644113E0E2076D0811
:1005700015436408C2071443039A01261205C01AE2
:1005800091413605001C7141CE07400830434908AF
:10059000C01851412A46234600F01BFBCDE7FFE778
:1005A000049801224000C117121A00238B410498BD
:1005B0003146C417381AA141EEE730B40124E407EC
:1005C000634030BC54E730B40124E407614030BCE0
:1005D0004EE700000000E0FFF0B51FB488B00B99B3
:1005E0000998002448400999C00F49004908099119
:1005F000C0070B990090490049080B910999089888
:10060000A64608431CD00B990A98084318D00998AD
:1006100001244000420D4800410D099824050003C3
:10062000000B204309900B980003000B20430B9014
:1006300050181C494018002201901446104605E04D
:10064000002001460DB0F0BD032801DA034600E0AA
:1006500003239C46C11A0AAE0AE05F0008ADED5BB9
:100660004F00F75B7D430027AA187C41491C5B1EA5
:100670006145F2DD410004AB5A522104120C0A43D9
:10068000240C401C0828DFDB01980290009970467A
:1006900001910090059B049A0799069800F0A6FA2C
:1006A000D0E700000DFCFFFFF0B50C465C4085B0C4
:1006B000E40FE40703944C000026640859009446B4
:1006C000490802460296224321D062460A431ED0C0
:1006D0006200570D4A000E032303550D0124024604
:1006E0002C492405781B1B0B360B4018234326434B
:1006F000614600901C46501AB44103D30098401C38
:10070000009002E0921800985B41002803DA002074
:10071000014605B0F0BD00200121090507468646C7
:1007200011E064461D46141BB54106D36546521BB5
:10073000B341744607430C43A646CD074008490819
:10074000284392185B4105460D43EAD110461843F1
:1007500013D06046194650407140084306D06046A9
:10076000101AB34106D20122002306E00022012321
:10077000DB0702E00122D2435310009874460105C2
:10078000381C6141029C039D0019694100F021FA67
:10079000BFE70000FD030000C217C10F504010B5B5
:1007A0004018CA079623002100F0DAF910BD10B5F1
:1007B00000229623114600F0D3F910BD0EB5C217E2
:1007C000C10F5040CA0740180021054B0293019207
:1007D00000910A460B4600F009FA03B000BD000084
:1007E000330400000EB505490291002100910A462C
:1007F0000B46019100F0FAF903B000BD330400008C
:100800003EB5CA17CB0F002450405140C01861417B
:10081000DA07054B0293019200942246234600F02A
:10082000E5F903B030BD000033040000C20F410001
:1008300040020123400ADB05D207090EC0187F29B8
:1008400001DA00207047962903DC9623591AC84024
:1008500001E096398840002AF4D0404270474100B8
:1008600040020122400AD205090E80187F2901DAD0
:1008700000207047962903DC9622511AC840704721
:10088000963988407047000070B5CD0F4A000903C3
:100890000123090B1B0519430B4BED070024520DD7
:1008A0009A4201DA002070BD074B34339A4203DCD0
:1008B0009A1A00F0EFF802E00449511888402C43DE
:1008C000F1D0404270BD0000FF030000CDFBFFFFF0
:1008D0004A0009030123090B1B051943094B10B5F5
:1008E000520D9A4201DA002010BD064B34339A4271
:1008F00003DC9A1A00F0CEF810BD03495118884065
:1009000010BD0000FF030000CDFBFFFF70B5CD0F51
:100910004A0009030123090B1B0519430D4BED0781
:100920000024520D9A4202DA0020014670BD094BA4
:1009300034339A4203DC9A1A00F0ACF803E0064B19
:10094000D21800F097F82C43F0D0002240428A41A0
:10095000114670BDFF030000CDFBFFFF4A000903F5
:100960000123090B1B0519430A4B10B5520D9A427E
:1009700002DA0020014610BD064B34339A4203DCF4
:100980009A1A00F087F810BD034BD21800F072F8E5
:1009900010BD0000FF030000CDFBFFFFC20FD20718
:1009A000400040080BD0C10D0723DB01C9184002ED
:1009B0000905400A1143C20840071143704700204F
:1009C0000146704710B5002904DB0124E4074042CA
:1009D0008C412146002B04DB1C460123DB075242DD
:1009E000A3418B4200D1824210BD000010B5002906
:1009F00004DB0124E40740428C412146002B04DB48
:100A00001C460123DB075242A341994200D1904288
:100A100010BD0000CB0FDB07490010B549080246A6
:100A20000A4307D00A0D07240903E401090B121B2E
:100A3000002A01DC002010BDC900440F0C43C10096
:100A4000E018D205801800F083F810BD0122D2070B
:100A5000002800DB101A002900DB511A8142704780
:100A60000122D207002800DB101A002900DB511AEE
:100A70008842704710B5202A04DB0146203A914095
:100A8000002010BD914020239C1A0346E3401943E7
:100A9000904010BD10B5202A04DB0846203AD04013
:100AA000002110BD0B46D340D0402024A21A914013
:100AB0000843194610BD10B5202A06DBCB1708469F
:100AC000203A1041C1170B4306E00B461341D040BA
:100AD0002024A21A91400843194610BD70B50C4657
:100AE00000683C21FFF706FB21603C21FFF702FB79
:100AF00061601821FFF7FEFA0546A1600721001D7D
:100B0000FFF7F8FAA1610F48A90008180E49FFF78E
:100B1000F1FA0246443288086261E0613B2802D360
:100B2000910700D0401C0021084B0A462161995CC6
:100B3000814203D8401A521C2261F8E7401CE06051
:100B4000204670BD6C0B0000B50500005D2501005E
:100B5000002904DA401C490001D1400840007047D8
:100B600070B40024050C05D11024000402D1002922
:100B700021D01124050E01D100020834050F01D146
:100B80000001241D850F01D18000A41C002801DB79
:100B90004000641C002908D020252E1B0D46F5407E
:100BA000A14000D001212943084301061B1B000A74
:100BB000DB1D02D5002070BC7047DB0518188018BB
:100BC0000029F8DA401C4900F5D170BC400840000B
:100BD000704710B5002B08DA0024401C61419218C0
:100BE0005B411A4301D14008400010BDF0B51FB46D
:100BF00082B005460C0003D008460EF0DBF902E097
:100C00000EF0D8F920300246009021462846FFF722
:100C100031FF049B059A04460F46184311430843CD
:100C200014D0184610431BD0009840210A1A1846C9
:100C30000599FFF72FFF05460E46009A059904987F
:100C4000FFF718FF084305D0012004E0204639468D
:100C500007B0F0BD0020C11705430E432C433743B6
:100C600000990E986305401A7905E40A00220C43A6
:100C7000FD0A0A3002D500200146E9E701051019F6
:100C800069410C9C0D9D00196941FFF7A2FFDFE748
:100C9000064C0125064E05E0E36807CC2B430C3CCF
:100CA00098471034B442F7D3FFF70EFA6C250100D1
:100CB0008C25010070B58C180578401C6B075B0F04
:100CC00001D10378401C2A1106D10278401C03E0B0
:100CD00006780E70401C491C5B1EF9D12B0705D409
:100CE0000023521E0DD40B70491CFAE70378401CF8
:100CF000CB1A921C03E01D780D70491C5B1C521E20
:100D0000F9D5A142D8D3002070BD00000146064AA3
:100D1000106907231B0402469A4310461A460A40EC
:100D20001043014A1061704700FA0140012806D1C2
:100D30000649096920221143044A116105E003496B
:100D4000096920229143014A1161704700FA01406C
:100D50000146054A1069000900010A07120F1043F5
:100D6000014A10617047000000FA0140012806D1D5
:100D70000649096840221143044A116005E003490D
:100D8000096840229143014A1160704700FA01400E
:100D9000012806D10649096801221143044A11605D
:100DA00005E00349096849084900014A1160704794
:100DB00000FA01400146064A1068082302469A4399
:100DC000104608220A401043014A10607047000094
:100DD00000FA01400146064A1068042302469A437D
:100DE000104604220A401043014A10607047000078
:100DF00000FA0140012806D1064909680222114380
:100E0000044A116005E00349096802229143014A3E
:100E10001160704700FA01400148806880B2704755
:100E200000FA014010B5012000F0C2FC0DF032FACA
:100E300001200DF041FA02200DF01CFA01200DF006
:100E400007FA0A20FFF784FF0120FFF76FFF042055
:100E5000FFF7C0FF0120FFF7CDFF0020FFF7AAFF3B
:100E6000064800F051F801208004FFF74FFF0020F2
:100E7000FFF77CFF0020FFF78BFF10BDFF0700008E
:100E800010B5012000F094FC0DF004FA01200DF0E3
:100E900013FA02200DF0EEF901200DF0D9F905202A
:100EA000FFF756FF0120FFF741FF0420FFF792FFF5
:100EB0000120FFF79FFF01208004FFF727FF00209C
:100EC000FFF778FF044800F01FF80020FFF74EFFFF
:100ED0000020FFF75DFF10BDFF0700000548C06858
:100EE000FF2101310840002801D001207047002077
:100EF000FCE7000000FA0140FF2001300149C86012
:100F00007047000000FA01404105490D014A516057
:100F10007047000000FA014010B5012000F048FCC5
:100F20000DF0B8F901200DF0C7F902200DF0A2F97B
:100F300001200DF08DF90F20FFF70AFF0120FFF7C8
:100F4000F5FE0420FFF746FF0120FFF753FF074897
:100F5000FFF7DAFF01208004FFF7D8FE0020FFF73B
:100F600005FF0020FFF714FF10BD0000FF07000081
:100F700070B505460E4614462946204600F002FC90
:100F8000044804600448066004F072F803F08EFD23
:100F900070BD0000000000200400002070B5054670
:100FA0000E4614462946204600F0ECFB0448046037
:100FB0000448066004F05CF800F0E6FE70BD000036
:100FC000000000200400002030B50246002018E098
:100FD000002112E0130184001B195B180A4CE35C2A
:100FE00084000A4D2D686419645C63408400074DD9
:100FF0002D68641963544B1CD9B20429EADB431CE5
:10100000D8B20428E4DB30BD100800200000002026
:1010100000200BE00022C1004118064BC918CA711C
:101020000A72C82800DD03E0411C88B24228F1D3CF
:1010300000BF70474600002030B50246002A01D1AB
:10104000012030BD002131E0C80008181A4BC31838
:1010500058781B7800021843904222D1C800081823
:10106000154BC018037AC0791B020343C800081847
:10107000114C0019047AC57920022843401C84B21F
:10108000C80008180C4D4019C471240A0472C80025
:1010900008182C4600198079834201DA0120D0E734
:1010A00006E0C82900DD03E0481C81B24229CBD309
:1010B00000BF0020C5E700004600002070477047D1
:1010C000F3B58DB00C46A2494879FFF78BFB054676
:1010D000A04AA14BFFF780FA0B910A900D98FFF7F9
:1010E0005DFC099108900B9B0A9AFFF76BFC02D2FA
:1010F0000120A0735FE096494879FFF773FB05462E
:10110000944A954BFFF768FA924A944B07910690E0
:10111000FFF7AEF90B910A900D98FFF73FFC09918C
:1011200008900B9B0A9AFFF74DFC07D2A07B012881
:1011300001D1A0733FE00220A0733CE0844908790C
:10114000FFF750FB0546834A834BFFF745FA0B91A7
:101150000A900D98FFF722FC099108900B9B0A9AC0
:10116000FFF730FC02D20220A07324E0784908790E
:10117000FFF738FB0546774A774BFFF72DFA754A9C
:10118000764B07910690FFF773F90B910A900D9833
:10119000FFF704FC099108900B9B0A9AFFF712FCD9
:1011A00007D2A07B022801D1A07304E00020A07325
:1011B00001E00020A073A07B012802D10020A075CF
:1011C000C3E0A07B022852D1614800796049497987
:1011D000884249DD5E4909795D4A5279881AFFF7EC
:1011E000EDFA05465B4A5C4BFFF7F6F9099108906A
:1011F00057490879FFF7F6FA0546564A564BFFF766
:10120000EBF9039102900D98FFF7C8FB0191009054
:10121000039B029AFFF7D1F90022514B05910490EC
:10122000FFF7DAF907910690099B089AFFF73CFA55
:101230000B910A90FFF7EEFB07463846FFF7AEFB2F
:1012400005460022464BFFF7D1FB01D2454F05E092
:1012500000213846FFF7FAFB00D200273846FFF797
:10126000E5FA40B2A07570E00020A0756DE0384945
:101270000879FFF7B7FA374A374B0B910A90FFF717
:10128000ABF9054605225207374BFFF79BFB5AD2B5
:101290002F490879FFF7A6FA05462E4A2E4BFFF78D
:1012A0009BF905225207304B05910490FFF78BF90B
:1012B0000991089026490879FFF794FA0546254ACE
:1012C000254BFFF789F9039102900D98FFF766FB14
:1012D00001910090039B029AFFF76FF90022234BC4
:1012E00005910490FFF778F907910690099B089AF9
:1012F000FFF7DAF90B910A90FFF78CFB07463846A7
:10130000FFF74CFB05460022184BFFF76FFB01D29D
:10131000174F09E03846FFF741FB05460022134608
:10132000FFF750FB00D200273846FFF737FB054692
:1013300000220B4BFFF79CF80B910A90FFF7A4FAE1
:1013400040B2A07501E01420A0750FB0F0BD000000
:10135000A80300209A9999999999B93F9999C93FF9
:10136000000034400000A041999919400000544009
:101370000000A04210B50121054800F069FB0220E1
:1013800000F086F800221021024809F0F9FD10BD96
:1013900007000001400D00407FB506460D4614468B
:1013A0006A462946304602F083F80098A84227D1C1
:1013B0006846C079002823D1E007C00F002803D178
:1013C0006846407900281BD1E007C00F002803D0F1
:1013D00068464079012813D102202040002803D11B
:1013E0006846807900280BD102202040002803D0D5
:1013F00068468079012803D16846007902281DD00B
:10140000029500206946C873E007C00F002801D18B
:10141000487302E0012069464873022020400028FA
:1014200002D16946887302E0012069468873022070
:101430006946087302A9304602F0F2F97FBD7FB514
:1014400005460C466A462146284602F031F80098C7
:10145000A0420FD16846C07900280BD16846407978
:10146000002807D168468079002803D168460079B2
:1014700003280BD0029400216846C1734173817325
:101480000321017302A9284602F0CAF97FBD0000BA
:1014900070B505460024002600F07EF9002802D130
:1014A000012000F085F9002416E00120A040064646
:1014B0002846304000280ED00C4800680121A14089
:1014C00088430A490860084681686200032090400A
:1014D000014306488160641C042CE6D300F05CF9EB
:1014E000012802D1002000F063F970BD00FC01402A
:1014F00010B500F005F8002801D000F00DF810BD7F
:1015000004480069C007C00F002801D001207047BF
:101510000020FCE70060014001200149086170479C
:10152000006001400A4681688908890093079B0F83
:10153000194381607047012904D1026880231A434E
:10154000026003E0026880239A430260704710B58E
:101550000A46016810240B46A34319461023134082
:101560001943016010BD10B50A46016820240B46DE
:10157000A3431946202313401943016010BD10B541
:101580000A46416830240B46A343194630231340D2
:101590001943416010BD10B50A46416880240B46CE
:1015A000A3431946802313401943416010BD01290C
:1015B00004D1426804231A43426003E042680423D2
:1015C0009A4342607047012904D1C26B10231A4329
:1015D000C26303E0C26B10239A43C26370470129C0
:1015E00004D1C26B04231A43C26303E0C26B042319
:1015F0009A43C2637047000010B5144800F02CF8FD
:10160000012813D1114800F034F8104800F02EF8EA
:1016100000210E48FFF78FFF00200D4908700D488C
:101620000088401C00B20B4908800DE00748443098
:1016300000F012F8012807D10448443000F019F8EE
:101640000248443000F012F810BD000000300140A4
:1016500096060020940600200146086C10221040D7
:10166000002801D0012070470020FCE71021016410
:101670007047082101647047012904D14269102391
:101680001A43426103E0426910239A434261704762
:10169000012904D1426901231A43426103E04269EE
:1016A0005208520042617047CAB282627047CAB2A1
:1016B00042627047CAB202617047000070B50446CA
:1016C0000E4615462D48844204D02C4844308442AE
:1016D00000D070BD2948844204D10121284800F07F
:1016E000B7F904E001212648401C00F0B1F90021BF
:1016F0002046FFF738FF10212046FFF728FF002182
:101700002046FFF748FF00212046FFF70BFF711E20
:101710002046FFF7CFFFE9B22046FFF7C8FFFF20C2
:101720000002284001122046FFF7BEFF002120469C
:10173000FFF725FF00212046FFF739FF2046FFF77E
:1017400095FF01212046FFF7A3FF01212046FFF767
:1017500093FF182009F066FA0121182009F0FEFA1B
:10176000182009F077FA01212046FFF72CFF01210C
:101770002046FFF734FF00BFABE700000030014018
:10178000010000040246002003E00B5C1354431CDC
:10179000D8B21028F9DB7047044800680007000F32
:1017A0000A2801D1012070470020FCE700E0014039
:1017B000012803D10A21034A116002E00521014AF0
:1017C0001160704700E0014000B502460023002090
:1017D000D060106110605060906000F0A3F90128A3
:1017E00007D100F087F903461B0C581C3B494843BE
:1017F000D06000F061F901280ED100F071F90346C4
:101800001B0C581C36494843106100F061F9082848
:1018100002D110694000106100F0FCF9034600BFDE
:10182000002B06D0012B07D0022B08D0032B0DD1A3
:1018300008E0D06810600CE02A48106009E01069E8
:10184000106006E00120C003106002E0D068106064
:1018500000BF00BF00F09AF903461B0A042B06D014
:10186000052B08D0062B0AD0072B10D10BE01068EF
:10187000400850600EE01068800850600AE0106870
:10188000C008506006E010680009506002E010686F
:10189000506000BF00BF00F091F903461B0C042B01
:1018A00006D0052B08D0062B0AD0072B10D10BE051
:1018B0005068400890600EE05068800890600AE030
:1018C0005068C008906006E050680009906002E02F
:1018D0005068906000BF00BF00BD000000127A0099
:1018E00040420F00001BB700012806D10649896954
:1018F00001221143044A916105E0034989694908BD
:101900004900014A9161704700240040002070475F
:101910000548C069FF2101310840002801D001209D
:1019200070470020FCE700000024004010B504468A
:10193000012C02D11148036813E0022C03D10F4897
:101940004038C36B0DE0032C03D10C484038836B47
:1019500007E0042C03D109484038436B01E00748F5
:101960000368180CD94389B2884203D1D8B200F079
:10197000F7F802E06B2000F0F3F810BD40FBFF1F0A
:10198000012806D10649096BC2071143044A1163B5
:1019900005E00349096B49004908014A1163704792
:1019A000002400400146064A106B130502469A4384
:1019B00010461A460A401043014A1063704700005F
:1019C00000240040012806D10749096B0202114397
:1019D000054A116306E00449096BFF220132914375
:1019E000014A116370470000002400400146054A87
:1019F000106B800880008A07920F1043014A106321
:101A00007047000000240040012806D10749096BF7
:101A100042021143054A116306E00449096B0122A1
:101A200052029143014A11637047000000240040B4
:101A30000146064A106B0C2302469A4310460C22BC
:101A40000A401043014A1063704700000024004020
:101A500030B502460B4600200F2424061440FF2513
:101A60002D066419002C09D06419002C08D06419C3
:101A7000002C08D06419002C0BD107E00D4809E0B8
:101A80000C48001D06E00B48083003E009480C3004
:101A900000E000BF00BF00280BD092B201219140AE
:101AA000002B03D004680C43046002E004688C43FC
:101AB000046030BD2024004004480069C007C00F06
:101AC000002801D0012070470020FCE700240040DE
:101AD00002480069082108407047000000240040C7
:101AE0000248006902490840704700000024004095
:101AF0000000FF03024840680F21090408407047B6
:101B0000002400400146064A50680F231B04024689
:101B10009A4310461A460A401043014A50607047E3
:101B20000024004004484068C007C00F002801D0CE
:101B3000012070470020FCE700240040012806D166
:101B40000649496801221143044A516005E00349EE
:101B5000496849084900014A516070470024004023
:101B60000146044A9068000A0002CAB21043014AC2
:101B7000906070470024004010B504462068FFF7CD
:101B8000C1FF2079FFF7DAFF10BD000002480068AE
:101B90000721090208407047002400400146064A18
:101BA000106807231B0202469A4310461A460A4051
:101BB0001043014A1060704700240040024800684A
:101BC0000721090408407047002400400146064AE6
:101BD000106807231B0402469A4310461A460A401F
:101BE0001043014A1060704700240040012806D1CC
:101BF0000749096842061143054A116006E0044995
:101C00000968012252069143014A116070470000A1
:101C100000240040024800684007400F7047000061
:101C2000002400400146054A1068C008C0004A0769
:101C3000520F1043014A106070470000002400401A
:101C400010B504462068FFF7EDFF6068FFF7A6FFB8
:101C5000A068FFF7BBFF207BFFF7C8FF10BD0000A7
:101C6000012806D10649496901221143044A5161FC
:101C700005E00349496949084900014A5161704733
:101C8000002400400146064A506907231B02024611
:101C90009A4310461A460A401043014A5061704761
:101CA00000240040F8B504460F461D462E46422C3F
:101CB00005D10320A8720020E872B07308E0522C0E
:101CC00006D10023142231460E3102480DF01DFBCF
:101CD000F8BD00002E030020F0B587B0064614467C
:101CE0001D462F46422E28D10023062204A9204655
:101CF0000DF00BFB60792179E2780092019102905E
:101D0000A27861782078012303900BF05BF81248E9
:101D1000407900020690104881790698081880B230
:101D200006900320059B049A06990FF00AFC0320F5
:101D3000A8720020E872B8730CE0522E0AD1082075
:101D4000A8720020E8720023062239460E310348AB
:101D50000DF0DBFA07B0F0BD04130020CC02002028
:101D600010B501210648FFF773FE0022082105483F
:101D700009F006F90821034801F095FD10BD0000A7
:101D800007000001000C004010B500240020FFF700
:101D90001BF901240AE00BF04BFC0BF0C5F808F02E
:101DA00077FE2046FFF710F9601CC4B20A2CF2DB64
:101DB0000BF03EFC0BF0B8F80A20FFF705F910BD58
:101DC00070B50A460021002300BF12E001248C40B8
:101DD000234614461C40002C0AD0046801258D407F
:101DE000AC430460C4684E000325B540AC43C460F6
:101DF000491C1029EAD370BD10B501210448FFF732
:101E000027FE002201214903024802F04CFD10BDCB
:101E100007000001000C004010B501210448FFF745
:101E200017FE012149030348FFF7CAFF10BD000058
:101E300007000001000C004010B592B001240023FF
:101E40000A220FA902311C480DF05FFA00230E226E
:101E500007A9023119480DF058FA00230E220BA9E8
:101E600017480DF052FA0023162201A90231154835
:101E70000DF04BFA0C23144A14490FA80EF086FDFE
:101E8000002800D100241E230F4A14320F491431B8
:101E900007A80EF07BFD002800D1002418230A4A71
:101EA0004C328321490101A80EF070FD002800D1B9
:101EB0000024204612B010BD0A00002014000020AB
:101EC0002200002030000020144C000014100000FC
:101ED00010B592B001240C231E4A1F490FA80EF022
:101EE000ABF9002801D1002406E000230A221B4997
:101EF0000FA802300DF009FA1E23164A14321649B3
:101F0000143107A80EF098F9002801D100240CE044
:101F100000230E22124907A802300DF0F6F9002323
:101F20000E2210490BA80DF0F0F91823094A4C3283
:101F30008321490101A80EF07FF9002801D1044650
:101F400006E000231622084901A802300DF0DDF951
:101F500012B010BD144C0000141000000A00002044
:101F60001400002022000020300000200320012166
:101F700089074860704700000146064AD06913157A
:101F800002469A4310461A460A401043014AD0615D
:101F90007047000040040040012806D10649C96985
:101FA00001221143044AD16105E00349C969490886
:101FB0004900014AD1617047400400400146064A89
:101FC000D069931502469A4310461A460A401043B8
:101FD000014AD0617047000040040040012806D14A
:101FE0000649C96904221143044AD16105E0034945
:101FF000C96904229143014AD161704740040040FD
:10200000012806D10649C96902221143044AD16157
:1020100005E00349C96902229143014AD161704731
:10202000400400400146064AD06903231B030246D0
:102030009A4310461A460A401043014AD06170473D
:10204000400400400146064AD069531502469A43AF
:1020500010461A460A401043014AD06170470000FA
:10206000400400400004054AD169054A1140D243AA
:1020700002401143014AD161704700004004004012
:10208000FFFF00E0C103490C014A116270470000E4
:102090004004004030B50246D400064D631918686C
:1020A00030250446AC43204630240C4020431860C1
:1020B00030BD0000040400400146C800054BC218B2
:1020C000042310681840002801D001207047002028
:1020D000FCE700000404004010B50246D300074CA2
:1020E0001819012904D1042403682343036003E081
:1020F00004240368A343036010BD000004040040EF
:1021000010B50246D300074C1819012904D1022446
:1021100003682343036003E002240368A3430360CE
:1021200010BD00000404004030B50246D400064D46
:1021300063191868ED140446AC4320462C460C4045
:102140002043186030BD00000404004030B5024652
:10215000D400064D6319186803252D030446AC43CB
:1021600020462C460C402043186030BD040400403B
:1021700030B50246D400064D6319186807252D02B4
:102180000446AC4320462C460C402043186030BD2A
:102190000404004030B50246D400054D631909041B
:1021A0001868044C2040E4430C402043186030BDC4
:1021B00004040040FFFF00E010B50246D300074CC6
:1021C0001819012904D1082403682343036003E09C
:1021D00008240368A343036010BD0000040400400A
:1021E00010B50246D300074C1819012904D1012467
:1021F00003682343036003E003685B085B0003603C
:1022000010BD00000404004030B50246D400064D65
:102210006319186840250446AC43204640240C400E
:102220002043186030BD0000040400400146C8008F
:10223000014BC218106870470804004010B5C30075
:10224000014C1A19116010BD08040040012806D184
:102250000649096801221143044A116005E0034957
:10226000096849084900014A1160704700040040AC
:1022700010B50720FFF720FF012807D1072000F045
:1022800007F8012802D1072000F012F810BD000065
:1022900001460648806A012212048A401040002844
:1022A00001D0012070470020FCE7000040040040FE
:1022B000012109048140014A9162704740040040B5
:1022C00010B5044620780B2823D120780021FFF791
:1022D00087FF6068FFF7C6FEA068FFF7A3FE60698E
:1022E000FFF74AFE606AFFF7ADFEA06AFFF766FEE1
:1022F000607FFFF773FEA07FFFF782FE2078216AE0
:10230000FFF79CFFE06AFFF7BDFEE07FFFF744FEAA
:102310002FE020780021FFF763FF20786168FFF746
:1023200039FF2078A168FFF711FF2078E168FFF7F7
:10233000FBFE20782169FFF71BFF20786169FFF71A
:1023400063FF2078A169FFF7A5FE217F2078FFF7C2
:1023500033FF617F2078FFF7BFFEA17F2078FFF772
:10236000CFFE2078216AFFF769FFE17F2078FFF731
:1023700037FF10BDFFB581B005460F461E4630073A
:10238000000F002801D005B0F0BD6806400E0828F7
:1023900000DDF8E700240DE0230103981A18680611
:1023A000430D074819182001C0190090FEF7E0FD01
:1023B000601C84B23011A042EEDC00BFE3E70000F5
:1023C00020040020FFB583B00E461C46002001907B
:1023D00003984006400E082801DD07B0F0BD2088B4
:1023E000019001980007000F02900298002812D077
:1023F00010210298081AC7B2002004E00199711850
:102400000F54411CC8B2B842F8DB01980011401CBF
:102410000005000C208000250EE02B0105981A18FD
:1024200003984006430D07481918280180190090A9
:10243000FEF7B4FD681C85B220880011A842ECDCD0
:1024400000BFCAE720040020F0B503460C46042173
:10245000187800282DD10120234D28702348057DB0
:10246000C67C2802304301280BD1002007E000265B
:1024700047001F4D7D192E706E70451CE8B207286D
:10248000F5DB1A48057DC67C28023043174DAE7D2A
:102490006F7D35023D43A8420BDA03211348057DC9
:1024A000C67C28023043401C85B21048C5742D0AF2
:1024B0000575104D68792D790002284306280BDB3D
:1024C0000C4D68792D7900022843801F85B2094898
:1024D00005712D0A457103E0002506480571457117
:1024E000002010800846F0BD710600204B06002039
:1024F000601C0020B0040020F0B597B004460D46E3
:102500002C210BA8FDF791FE2C216846FDF78DFECE
:102510002178CA17120F521812110A235A4308467B
:10252000CB171B0F1B181B111B01CB1AD2187D23B5
:102530001B01D21893B210AA13832978CA17120F5D
:10254000521812110A235A430846CB171B0F1B18A7
:102550001B111B01CB1AD2187D231B01D21893B279
:1025600010AA5383108B5A49401A10906178CA17E9
:10257000120F521812110A235A430846CB171B0F89
:102580001B181B111B01CB1AD218521E0F92A178D7
:10259000CA17120F521812110A235A430846CB17B2
:1025A0001B0F1B181B111B01CB1AD2180E92E178BE
:1025B000CA17120F521812110A235A430846CB1792
:1025C0001B0F1B181B111B01CB1AD2180D9221795E
:1025D000CA17120F521812110A235A430846CB1772
:1025E0001B0F1B181B111B01CB1AD2180C926179FF
:1025F000CA17120F521812110A235A430846CB1752
:102600001B0F1B181B111B01CB1AD2180B9210AAFF
:10261000508B2F49401A05906978CA17120F52182B
:1026200012110A235A430846CB171B0F1B181B1104
:102630001B01CB1AD218521E0492A978CA17120F86
:10264000521812110A235A430846CB171B0F1B18A6
:102650001B111B01CB1AD2180392E978CA17120F6B
:10266000521812110A235A430846CB171B0F1B1886
:102670001B111B01CB1AD21802922979CA17120F0B
:10268000521812110A235A430846CB171B0F1B1866
:102690001B111B01CB1AD21801926979CA17120FAC
:1026A000521812110A235A430846CB171B0F1B1846
:1026B0001B111B01CB1AD21800920BA8FDF756FD77
:1026C00006466846FDF752FD0746F01B17B0F0BD01
:1026D0006C07000010B501211348FFF7B9F900227B
:1026E0000121C902114808F04BFC002240210F488B
:1026F00008F046FC0022012189030C4808F040FC48
:10270000012189020948FFF75BFB0121C902074843
:1027100001F0C9F84021054801F0C7F801218903FB
:10272000024801F0C2F810BD07000001800C004013
:1027300010B501211348FFF78BF900220121C902CE
:10274000114808F01DFC002240210F4808F018FC39
:102750000022012189030C4808F012FC01218902A2
:102760000948FFF72DFB0121C902074801F09DF838
:102770004021054801F097F801218903024801F042
:1027800092F810BD07000001800C0040F8B5064625
:102790000C46174600BF4021174801F084F801217C
:1027A0008903154801F081F800BF03200AF026FFD5
:1027B0002102080E0AF022FF2104080E0AF01EFF73
:1027C000E0B20AF01BFF002505E0FF200AF016FF2B
:1027D0007055681C85B2BD42F7DB00F09BF800BF66
:1027E0004021054801F061F801218903024801F008
:1027F0005CF800BFF8BD0000800C0040F7B584B065
:102800007D2149010698884202DD002007B0F0BD15
:102810000498029000200390059C069D002D0CD08A
:10282000200A461C3002001BA84201D32F4601E0BB
:102830003002071B0120039001E00020039061E0BB
:1028400000BF4021324801F02EF8012189033048B1
:1028500001F02BF800BF06200AF0D0FE00BF402197
:102860002B4801F022F801218903294801F01DF8C5
:1028700000BF00BF4021264801F015F8012189035F
:10288000234801F012F800BF02200AF0B7FE21022F
:10289000080E0AF0B3FE2104080E0AF0AFFEE0B203
:1028A0000AF0ACFE0020019009E002990878491C6A
:1028B00002910AF0A3FE0198401C80B20190019899
:1028C000B842F2D300BF4021114800F0EEFF0121D1
:1028D00089030F4800F0E9FF00BFE419ED1B002D4C
:1028E0000CD0200A461C3002001BA84201D32F4600
:1028F00001E03002071B0120039001E0002003905B
:1029000000F008F8039800289AD100BF7EE7000085
:10291000800C004010B500BF00F006F8C007C00FE3
:102920000028F9D110BD000010B50A200CF06AFF94
:1029300000BF40210E4800F0B6FF012189030C487A
:1029400000F0B3FF00BF05200AF058FEFF200AF098
:1029500055FE044600BF4021054800F0A6FF0121B6
:102960008903034800F0A1FF00BF204610BD00000E
:10297000800C0040FFB583B004460F460020019054
:1029800001AA394620460DF0D7FF002801D107B033
:10299000F0BDE41C6846407E012825D168460079D8
:1029A000082821DB61786846017221784172E1785C
:1029B0008172A178C1720298FDF714FF0546284A7A
:1029C000FDF773FC61796846017221794172E17902
:1029D0008172A179C1720298FDF704FF0546204A71
:1029E000083AFDF762FC39E06846407E022818D1BB
:1029F00068460079082814DB617819483230017183
:102A00002178001D4170E1788170A178C1706179F1
:102A1000001F017021794170E1798170A179C17045
:102A20001CE06846407E032818D1684600790828D3
:102A300014DB61780A481230017721781C3041702C
:102A4000E1788170A178C17061791C3801762179B3
:102A500018304170E1798170A179C170012096E749
:102A6000BE1D002010B501210748FEF7F1FF00222E
:102A70002021064801F017FF0022082103484030BA
:102A800008F07EFA10BD000007000001400D004074
:102A9000FEB5044616460527012019490870194954
:102AA0000870002007E000224300174959180A70F7
:102AB0004A70411CC8B20728F5DB14492046FFF7CD
:102AC0001BFD0546281E01DB014600E041420D4684
:102AD000FF202D3085420BDB60792179E27800926E
:102AE00001910290A2786178207801230AF06AF9B6
:102AF0000021074801714171002030803846FEBD39
:102B00007006002071060020601C0020CC0200200E
:102B1000B004002010B54623034AFF216531034865
:102B20000DF034FF10BD0000643D00002C030020B8
:102B300010B54623064AFF21653106480DF07CFB9F
:102B4000002803D1FFF7E6FF002010BD0120FCE7BD
:102B5000643D00002C03002003B56846C0780628B9
:102B600009D168460079102805D1684640790528C2
:102B700001D1FEF74DFA0CBD10B500BF012189034C
:102B80000B4800F090FE4021094800F08EFE00BF87
:102B900006200AF033FD00BF4021054800F085FE05
:102BA00001218903024800F080FE00BF10BD000033
:102BB000800C00400146054A1068800880008A07A2
:102BC000920F1043014A106070470000001000404F
:102BD000F0B5044600260D46002B08D001208005E4
:102BE000844204D2814202D20013824201DD0020DD
:102BF000F0BD0AE0AC4201D10120F9E7AD18701C2C
:102C00000646044FB84200D901E09E42F2D300BF0D
:102C10000020EDE7FFFF0000F0B5FFB0FFB083B08C
:102C200005460F4614460121FFA841600026880290
:102C3000844204DD00207FB07FB003B0F0BD00BF50
:102C400009F01EFFFFF746FD0121C902274800F0E9
:102C50002AFE00BF01218903244800F024FE402100
:102C6000224800F022FE00BF00BF224639466846D7
:102C700008F0C0F86846017840780002081886B26B
:102C8000A21E00A902311A480FF08CF8B0421DD0E4
:102C900022463946684608F0ADF868460178407823
:102CA0000002081886B2A21E00A9023110480FF0D7
:102CB00079F8B04203D00020FFA948600CE000235F
:102CC0002246294668460CF020FB05E000232246F8
:102CD000294668460CF019FB00BF09F03DFFFFF7DD
:102CE00027FD00BFFFA84068A5E70000800C00405A
:102CF000FFFF0000F8B504460D4616460127324690
:102D00002946204600F00CF8002807D13246294613
:102D1000204600F005F8002800D100273846F8BD0D
:102D200070B5FFB0FFB082B005460E4614460120D4
:102D30008002844204DD00207FB07FB002B070BD0D
:102D400000BF09F09DFEFFF7C5FC0121C902124832
:102D500000F0A9FD00BF012189030F4800F0A3FD89
:102D600040210D4800F0A1FD00BF00BF22463146C2
:102D7000284608F075F822463146684608F03AF8C9
:102D800000BF09F0E9FEFFF7D3FC00BF2246694609
:102D900028460EF0DBFDCFE7800C004010B504465E
:102DA0002403FFF7E9FE00F04DF800BF012189037D
:102DB000114800F078FD40210F4800F076FD00BF7B
:102DC00020200AF01BFC2102080E0AF017FC210447
:102DD000080E0AF013FCE0B20AF010FC00BF40211C
:102DE000054800F062FD01218903034800F05DFD04
:102DF00000BF00F027F810BD800C004010B5002483
:102E000000BF012189030E4800F04DFD40210C4810
:102E100000F04BFD00BF05200AF0F0FBFF200AF098
:102E2000EDFB044600BF4021054800F03EFD0121B6
:102E30008903034800F039FD00BF204610BD0000A3
:102E4000800C004010B500BFFFF7D8FFC007C00FCF
:102E50000028F9D110BDF8B507460E461446F0B269
:102E6000FF2101310D1AAC4200DC254612E02A4652
:102E70003146384600F012F8AC4200D10BE07F1921
:102E80007619601B84B2FF200130844201DD0546C3
:102E900000E02546EBE700BFF8BD0000F8B50646A8
:102EA0000C461746FFF768FE00BF0121890316484C
:102EB00000F0F9FC4021144800F0F7FC00BF0220AC
:102EC0000AF09CFB2102080E0AF098FB2104080E70
:102ED0000AF094FBE0B20AF091FB002504E0705D7B
:102EE0000AF08CFB681C85B2BD42F8DB00BF4021B4
:102EF000054800F0DAFC01218903034800F0D5FC05
:102F000000BFFFF79FFFF8BD800C004010B5002206
:102F100001210903014801F0C6FC10BD800C0040EE
:102F200001460020044A12690A40002A01D001200B
:102F300000E000207047000000FC0140F7B50346A8
:102F40000D460021002207E0012696402E40002E6B
:102F500001D0114602E0521C102AF5D300BF102AFE
:102F600000D1FEBD314FDE1BBB4211D008DC304E1C
:102F70009E19002E09D0402E08D0802E51D106E097
:102F8000402E06D0802E4CD104E000BF00BF00BF11
:102F900000BF00BF254E4036B34203D0234E8036DB
:102FA000B34202D10B2903D93CE00F2900D939E003
:102FB000032901D800200CE0042903D3072901D8F4
:102FC000012006E0082903D30B2901D8022000E0E4
:102FD0000320164E803EB34200D1001D134E403EEA
:102FE000B34200D10830114EB34200D10C300F4E25
:102FF0004036B34200D110300C4E8036B34200D17F
:1030000014300C4E3469029E012E02D186403443A6
:1030100004E0012686402746B7433C46054E34610E
:1030200000E000BF00BF00BF9BE70000C00C0040F5
:1030300000F4FFBFC00D0040F0B502460D4600236E
:103040000027002407E00120A0402840002801D0EC
:10305000234602E0641C102CF5D300BF102C01D1D4
:103060003846F0BD2E4E901BB24211D008DC2D48E0
:103070001018002809D0402808D080284CD106E03C
:10308000402806D0802847D104E000BF00BF00BF21
:1030900000BF00BF22484030824203D02048803029
:1030A000824202D10B2B03D937E00F2B00D934E039
:1030B000032B01D800210CE0042B03D3072B01D8EC
:1030C000012106E0082B03D30B2B01D8022100E0DD
:1030D000032113488038824200D1091D104840382E
:1030E000824200D108310E48824200D10C310C4896
:1030F0004030824200D1103109488030824200D1F4
:1031000014310948406901268E40304001268E4026
:10311000B04200D1012700E000BF00BF3846A0E761
:10312000C00C004000F4FFBFC00D0040F0B50246E7
:103130000C460021002307E001269E402640002E79
:1031400001D0194602E05B1C102BF5D300BF102BF9
:1031500000D1F0BD2D4FD61BBA4211D008DC2C4E49
:103160009619002E09D0402E08D0802E49D106E0B5
:10317000402E06D0802E44D104E000BF00BF00BF27
:1031800000BF00BF214E4036B24203D01F4E8036F2
:10319000B24202D10B2903D934E00F2900D931E022
:1031A000032901D800200CE0042903D3072901D802
:1031B000012006E0082903D30B2901D8022000E0F2
:1031C0000320124E803EB24200D1001D0F4E403E01
:1031D000B24200D108300D4EB24200D10C300B4E3D
:1031E0004036B24200D11030084E8036B24200D193
:1031F0001430084E7569012686403540054E7561CC
:1032000000E000BF00BF00BFA3E70000C00C00400B
:1032100000F4FFBFC00D0040F8B505460E46174646
:103220001C4603223146284600F022F83146284643
:1032300000F0A4F8224631462846FFF77FFE3A46C2
:103240003146284600F014F8C8200CF0DBFA31466D
:103250002846FFF76BFF1E20002805DBC206D20EB2
:1032600001219140014A116000BFF8BD80E200E0F9
:10327000F7B5034615460021002408E00126A640C4
:10328000019F3E40002E01D0214602E0641C102C1C
:10329000F4D300BF102C00D1FEBD354FDE1BBB4266
:1032A00011D008DC334E9E19002E09D0402E08D0D4
:1032B000802E58D106E0402E34D0802E53D132E0FB
:1032C00000BF00BF00BF0F2900D94DE0032901D87E
:1032D00000200CE0042903D3072901D8022006E0CE
:1032E000082903D30B2901D8042000E00620204E32
:1032F000803EB34200D108301D4E403EB34200D163
:1033000010301B4EB34200D118301B4EB26803265A
:1033100086401746B7433A462E4686403243164EFD
:10332000B26021E000BF0B2900D91DE0032901D8BC
:10333000002006E0042903D3072901D8022000E079
:1033400004200B4E8036B34200D108300A4EF2689A
:10335000032686401746B7433A462E4686403243F8
:10336000054EF26000BF00BF00BF00BF94E7000041
:10337000C00C004000F4FFBFC00D0040F0B5024695
:103380000D460020002407E00126A6402E40002E16
:1033900001D0204602E0641C102CF5D300BF102C95
:1033A00000D1F0BD3F4FD61BBA4234D008DC3E4EB0
:1033B0009619002E2CD0402E2BD0802E6ED129E0D5
:1033C000402E02D0802E69D100E000BF0B2800D92A
:1033D00065E0032801D8002106E0042803D307286C
:1033E00001D8022100E004212E4E8036B24200D1E5
:1033F00008318007800F2D4E736803268E401F46CC
:10340000B7433B4606468E403343284E736046E042
:1034100000BF00BF00BF234EC03EB24207D0214EC6
:10342000803EB24203D01F4E403EB24202D10F282E
:1034300000D934E01B4EB24202D10B2800D92EE055
:10344000032801D800210CE0042803D3072801D861
:10345000022106E0082803D30B2801D8042100E04C
:103460000621104E803EB24200D108310D4E403E42
:10347000B24200D110310B4EB24200D11831800758
:10348000800F0A4E336803268E401F46B7433B46E3
:1034900006468E403343054E336000E000BF00BF58
:1034A00000BF7EE7C00C004000F4FFBFC00D00402D
:1034B000F0B504460025002307E001269E400E409B
:1034C0003546002D00D002E05B1C102BF5D300BF69
:1034D000102B36D21D46116026680E403046E8405B
:1034E000012802D10126D67101E00026D671666856
:1034F0000E40EE403046012801D1967101E00026D1
:103500009671A6680E40EE403046012801D15671F2
:1035100001E000265671E6686F00FE40B007800F9C
:10352000002802D1002616710BE0012802D10126E5
:10353000167106E0022802D10226167101E0032668
:103540001671F0BD10B50AF073F94021A548FFF7D8
:1035500073FD012844D14021A248FFF7E7FD012077
:10356000A1490870A148C08800280AD09F48C08897
:10357000401E81B29D48C180002902D101209B4993
:1035800008719A48C08900280AD09848C089401E0E
:1035900081B29648C181002902D101209349087364
:1035A00092484088002809D090484088401E80B248
:1035B0008E494880002801D1012008708C49487B41
:1035C000097B0002084300280AD08949487B097B0F
:1035D00000020843401E80B285490873000A487300
:1035E000012149027F484030FFF726FD01285FD1C5
:1035F00041027C484030FFF799FD0121490279489A
:10360000403000F046F9002852D101218903754865
:10361000803000F03EF9002814D17448C08800289A
:1036200010DD74480078C006C00F002805D071482E
:1036300080780007C00F00283AD1032108460BF01C
:1036400001F835E00121C9036648803000F021F916
:1036500000280ED16548C08800280ADD654800783A
:10366000C006C00F002823D1032101200AF0EAFF81
:103670001EE05E48C088002809D101205E4908701C
:1036800006F064FA01215748803000F00EF900BFBF
:103690001E215648C18000205449087100BF0120F6
:1036A0005649087001F076FD0220554908704870AF
:1036B00040214C488038FFF7BFFC012825D140212C
:1036C00048488038FFF732FD4E48807803280CD1F7
:1036D00040214448803800F0DCF8002815D10BF078
:1036E0009DF80120474988700FE0464880780428FB
:1036F0000BD180213B48803800F0CBF8002804D162
:103700000BF08CF802203F49887001213548FFF703
:1037100093FC012806D101213248FFF707FD012063
:103720003749C87020212F484038FFF785FC012811
:1037300019D120212B484038FFF7F8FC3248C07BD4
:103740008021084080280ED02F488078012803D09F
:103750002D488078032806D101202C4908700121CA
:103760002B48FDF7E8FE20211E488030FFF764FC5F
:10377000012809D120211B488030FFF7D7FC082100
:103780001848C03000F08FF801214903154840382F
:10379000FFF752FC012824D1410312484038FFF7BB
:1037A000C5FC002306221B491B480BF0AEFD19483F
:1037B0008068401C1749886018484078087317488B
:1037C000407948731548C0788873202105488030B7
:1037D00000F05FF80F49C873064840788007C00FB3
:1037E000087410BDC00C0040980200209A0200200E
:1037F000071B0020C00800207A0600207906002060
:10380000DE020020F912002072030020960600203C
:1038100000300140E8110020CC020020AA02002064
:10382000F0B502460B4600210024002500BF2DE024
:1038300001268E4034461E6826403546A54224D1D6
:1038400010680646A6433046DE798E40304310604D
:1038500050680646A64330469E798E4030435060FD
:1038600090680646A64330465E798E4030439060AD
:103870004F000326BE403446D0680646A643304675
:103880001E794F00BE403043D060491C1029CFD371
:10389000F0BD02460020D3690B40002B01D001206F
:1038A00000E0002070478161704741617047026904
:1038B0000A40002A01D0816100E04161704710B5E3
:1038C0001346826A012B03D114460C43224602E0C0
:1038D00014468C432246826210BD0000F8B50446AF
:1038E0000526FE484078002811D1FC48C078002801
:1038F0000DD1FA484079002809D1F94800880528F7
:1039000008DAF7480088401CF549088002E00020EA
:10391000F3490880F348C07817280AD1F1480079A4
:10392000392806D1EF484079392802D1012020708A
:103930006070EC480079392805D1EA4840793A2886
:1039400001D10120A070E078012840D10020E07072
:103950000121E548FFF79DFF002838D100BFE3486B
:1039600000794007C00F002830D1E14800794007B6
:10397000C00F00282AD0DD48007904218843001DAB
:10398000DA490871DB48007904218843001DD949D0
:103990000871122100200DF0E3FBD74800794007A1
:1039A000C00F00280ED01220FDF746FB012809D1D8
:1039B000D248007904218843001DD04908710120B4
:1039C000CF4908701221CF48FDF779FB00BF0120D5
:1039D000FFF7A6FA002840D10A200BF0EBFE0120E9
:1039E000FFF79EFA00284AD100BFC0480079800640
:1039F000C00F002830D1BE4800798006C00F0028D3
:103A00002AD0BA480079202188432030B74908716C
:103A1000B8480079202188432030B6490871152123
:103A200000200DF09DFBB44800798006C00F0028EF
:103A30000ED01520FDF700FB012809D1AF48007911
:103A4000202188432030AD4908710120AC4908701D
:103A50001521AC48FDF733FB11E000BFA348007906
:103A60008006C00F002809D0A04800792021884393
:103A70009E4908711521A348FDF720FB00BF20785F
:103A800000280ED00020207000F064FC0546611D67
:103A9000FCF702FC601DFCF7E7FB0546214606F03B
:103AA000D5FB6078002814D08D480088052810DBED
:103AB0000020607000F0A6FB054621460A31FCF7A5
:103AC000EBFB20460A30FCF7CFFB05462146FDF70D
:103AD000F7FAA078012808D10020A07000F084FC3B
:103AE000054621460F31FCF7D7FB80484078800718
:103AF000C00F002802D1844806F07AFB82480A30C1
:103B0000FCF7B2FB05468048801DFCF7ADFB854203
:103B100002D30020207516E07B48801DFCF7A4FB33
:103B200000907948801DFCF79FFB074676480A30D5
:103B3000FCF79AFB381A6421484305460099FCF7C4
:103B4000D9FA40B22075607A012875D100BF674864
:103B500000798007C00F002830D1654800798007C0
:103B6000C00F00282AD06148007902218843801CB8
:103B70005E4908715F48007902218843801C5D49D5
:103B80000871112100200DF0EBFA5B4800798007E5
:103B9000C00F00280ED01120FDF74EFA012809D1E0
:103BA0005648007902218843801C5449087101203D
:103BB0005349087011215348FDF781FA00BF00BF37
:103BC0004A480079C007C00F002830D14848007922
:103BD000C007C00F00282AD04448007940084000A0
:103BE000401C424908714348007940084000401C8D
:103BF00040490871102100200DF0B2FA3E480079CA
:103C0000C007C00F00280ED01020FDF715FA0128BC
:103C100009D13A48007940084000401C37490871F2
:103C200001203749087010213648FDF748FA00BFD7
:103C300000206075E6E0FFE7607A022866D100BFE9
:103C40002A4800798007C00F002809D0274800794A
:103C5000022188432549087111212A48FDF72EFACF
:103C600000BF00BF21480079C007C00F002830D135
:103C70001F480079C007C00F00282AD01B480079D0
:103C800040084000401C194908711A480079400852
:103C90004000401C17490871102100200DF060FA07
:103CA00015480079C007C00F00280ED01020FDF77E
:103CB000C3F9012809D11148007940084000401C8F
:103CC0000E49087101200E49087010210D48FDF7BA
:103CD000F6F900BFA07D607594E017E0AA0200200D
:103CE000F8020020CC020020C00C0040C0080020D8
:103CF00014000020DA08002022000020CC08002058
:103D000008000020B4020020A8030020207D6428C1
:103D100000D102E014202056401C40B260751520EE
:103D2000205614284ADA00BFFE4800798007C00FE9
:103D3000002809D0FB48007902218843F94908711D
:103D40001121F948FDF7BAF900BF00BFF548007925
:103D5000C007C00F002830D1F4480079C007C00F59
:103D600000282AD0EF48007940084000401CED4967
:103D70000871EF48007940084000401CEC49087188
:103D8000102100200DF0ECF9EA480079C007C00FBF
:103D900000280ED01020FDF74FF9012809D1E64880
:103DA000007940084000401CE34908710120E349C4
:103DB00008701021DC48FDF782F923E000BFD948E4
:103DC00000798007C00F002809D0D6480079022169
:103DD0008843D44908711121D348FDF76FF900BF1A
:103DE00000BFD0480079C007C00F002809D0CD48D7
:103DF000007940084000CB4908711021CA48FDF7FE
:103E00005DF900BFA07B012872D100BFC5480079D1
:103E1000C006C00F002830D1C4480079C006C00FCA
:103E200000282AD0BF480079102188431030BD49AE
:103E30000871BF480079102188431030BC490871CF
:103E4000142100200DF08CF9BA480079C006C00F8B
:103E500000280ED01420FDF7EFF8012809D1B6484C
:103E60000079102188431030B34908710120B3490B
:103E700008701421AC48FDF722F900BF00BFA94823
:103E800000790007C00F002830D1A848007900074A
:103E9000C00F00282AD0A3480079082188430830A1
:103EA000A0490871A2480079082188430830A04938
:103EB0000871132100200DF053F99E480079000786
:103EC000C00F00280ED01320FDF7B6F8012809D145
:103ED00099480079082188430830974908710120E2
:103EE0009649087013219048FDF7E9F872E0FFE762
:103EF000A07B02284AD100BF8A480079C006C00FC3
:103F0000002809D087480079102188438549087125
:103F100014218548FDF7D2F800BF00BF8148007921
:103F20000007C00F002830D1804800790007C00F7B
:103F300000282AD07B480079082188430830794935
:103F400008717B4800790821884308307849087156
:103F5000132100200DF004F9764800790007C00F06
:103F600000280ED01320FDF767F8012809D1724808
:103F700000790821884308306F49087101206F4992
:103F8000087013216848FDF79AF823E000BF6548E0
:103F90000079C006C00F002809D0624800791021BE
:103FA00088436049087114215F48FDF787F800BF16
:103FB00000BF5C4800790007C00F002809D05948AD
:103FC0000079082188435749087113215648FDF7A5
:103FD00075F800BFFEF746FD20215948FFF759FC50
:103FE00000285BD1207617202056052803DAE07DD3
:103FF000401C40B2E0751720205605284DDB49488B
:1040000040788007C00F002847D108214C48403035
:10401000FFF74BFC00BF434840788007C00F0028E3
:104020000AD14048407802218843801C3D494870AD
:1040300000213D48FDF743F800BF01230022202165
:104040003F48FFF7E9F80DF06FFD00203D4988700B
:1040500001203D4908700BF079FB042138484030BD
:10406000FFF721FC314840788007C00F002871D04D
:10407000304840788007C00F00286BD00220FCF742
:10408000DBFF012866D12C48407802218843801C40
:10409000294948700120294908705BE000231A462D
:1040A00020212748FFF7B8F8082125484030FFF7BE
:1040B000FAFB0020E0751B4840788007C00F0028FD
:1040C00048D000BF174840788007C00F002809D0AB
:1040D0001448407802218843124948700021124850
:1040E000FCF7ECFF00BF114840788007C00F0028A4
:1040F00030D00F48407802218843801C0C4948701A
:104100000C4840788007C00F002823D00220FCF71D
:1041100093FF01281ED10848407802218843801C63
:10412000054913E0C0080020B4020020140000205C
:10413000DA08002022000020CC080020080000201F
:10414000400D0040BE0200207A0600204870012089
:1041500001490870F8BD00000800002000B50146C4
:104160000B000AF03EFF091A0C0E11141706080A7C
:104170001A00692000BD9B20FCE79B20FAE79B20EA
:10418000F8E7FF201E30F5E7FF20BE30F2E7FF2002
:10419000EB30EFE74120C000ECE74120C000E9E749
:1041A00070B5002400250120FCF7F2FDFCF7A4FE09
:1041B0000AF0BCFF002803D1FCF72EFE054601E003
:1041C000002070BD28460AF02DFF04462046F8E77F
:1041D00038B50020009000240120FCF7D9FDFCF741
:1041E0008BFE0AF0A3FF002803D1FCF715FE04465E
:1041F00001E0002038BD20460AF066FF00900098DC
:10420000F8E70000F0B587B00026FDF7B3F8FCF73B
:1042100009FE10211C48FFF748FB05200BF0CAFAE5
:1042200013200CF053FB041E27D0082161700021DD
:10423000A1700A202070204600F0EEF807463846AC
:10424000FCF7B5FA0190FCF7A9FB104A104B03915B
:104250000290FCF7C1F905910490FCF7DBFB0546E1
:104260000C492846FCF789F8064610210648FFF756
:104270001AFB20460CF00CF900240020FCF788FD06
:10428000304607B0F0BD0000400D0040FCA9F1D25F
:104290004D62503F10584D401FB50446072202A9F9
:1042A000002007F09BFF6846817B0170417B4170D5
:1042B000017B8170817AC170417A0171017A41710B
:1042C0000199009809F00CFB012814D16846007A86
:1042D00060716846407A20716846807AE07068466E
:1042E000007BA0706846407B60706846807B2070D1
:1042F000012004B010BD072202A9002007F06EFFC4
:104300006846817B0170417B4170017B8170817ABD
:10431000C170417A0171017A41710199009809F0E7
:10432000DFFA012813D16846007A60716846407A46
:1043300020716846807AE0706846007BA07068460D
:10434000407B60706846807B20700120D1E70020B0
:10435000CFE70000F0B587B0002606F0D1F8FCF7F3
:104360008FFD08211C48FFF7A0FA05200BF022FA68
:1043700014200CF0ABFA041E27D008216170002134
:10438000A17005202070204600F046F80746384608
:10439000FCF70DFA0190FCF701FB104A104B03915A
:1043A0000290FCF719F905910490FCF733FB0546E0
:1043B0000C492846FBF7E1FF064608210648FFF7AF
:1043C00072FA20460CF064F800240020FCF7E0FCB0
:1043D000304607B0F0BD0000400D0040FCA9F1D20E
:1043E0004D62503F1B2F4D4070B5FCF795FD1320DB
:1043F0000CF06CFA041E0AD0082161700021A17033
:10440000FFF7CEFE054620460CF042F800240020BF
:10441000FCF7BEFC284670BDFEB5044600200090A7
:10442000002509E0FFF7D4FE0746AA00E01C11189A
:104430003846FBF731FF6D1CA17862780802104303
:10444000A842EFD800252EE06E1C25E0B200E11C4A
:104450005018FBF709FF0746AA00E11C5018FBF7AC
:1044600003FF874217D2B200E11C5018FBF7FCFE95
:104470000190AA00E11C5018FBF7F6FE0746B200B7
:10448000E01C11183846FBF707FFAA00E01C1118C2
:104490000198FBF701FF761CA178627808021043AF
:1044A000B042D3D86D1CA178627808021043A842AC
:1044B000CAD8012002900BE002998A00E11C501832
:1044C000FBF7D2FE0099401800900298401C029021
:1044D000A178627808021043401E02998842EBD806
:1044E000A278637810021843811E0098FBF702FE41
:1044F00000900098FEBD0000F0B599B00120189022
:104500000025002600271B480078012830D1002014
:104510001849087000BF1848417902790E02164305
:10452000801DFBF7A1FE044600BF13E0781C87B294
:104530001248844201D8124C00E0543C54222146D7
:1045400001A8FEF769FB012802D00020189003E0C3
:10455000681C85B2B542E9DB00BF1898002807D176
:10456000179405484179027908021043401B1690C0
:1045700019B0F0BDFD0200201B05002000581400FA
:10458000CC9F150010B508F0F1FB08210C48FFF78F
:104590008AF901200BF036F904210948FFF785F963
:1045A00004200BF02FF904210548FFF77CF90420C3
:1045B0000BF028F908210248FFF777F910BD000039
:1045C000C00C004010B508F0D1FB08210A48FFF7E5
:1045D0006CF901200BF016F904210748FFF765F983
:1045E00004200BF00FF904210348FFF75CF90420C5
:1045F0000BF008F910BD0000C00C004070B5082198
:104600001348FFF752F908F0A1FB80241BE00421B6
:104610000F48FFF74AF901200BF0F4F808210C4885
:10462000FFF737F9012803D128462043054602E069
:104630002846A043054604210548FFF734F9042025
:104640000BF0E0F86410002CE1D1284670BD0000AA
:10465000C00C004010B501210648FDF7F9F9002211
:104660000421054806F08CFC04210348FFF71BF9E0
:1046700010BD000007000001C00C004070B50546E9
:1046800008F074FB80241BE020462840002804D159
:1046900008211448FFF707F903E008211148FFF744
:1046A00004F901200BF0AEF804210E48FFF7FDF8E5
:1046B00004200BF0A7F804210A48FFF7F4F864106F
:1046C000002CE1D104200BF09DF804210548FFF7F0
:1046D000ECF804200BF096F804210248FFF7E3F809
:1046E00070BD0000C00C004010B5FFF7B3FF08F02C
:1046F0003DFB08210A48FFF7D8F804210848FFF7D6
:10470000D4F804200BF07EF808210548FFF7CBF819
:1047100004200BF077F804210148FFF7C4F810BD1E
:10472000C00C004010B508F021FB04210C48FFF735
:10473000BAF808210A48FFF7B6F804200BF062F82F
:1047400004210748FFF7B1F804200BF05BF80821BB
:104750000348FFF7AAF804200BF054F810BD00003E
:10476000C00C0040F8B506460F4614461D467D2095
:10477000C000844201DD0020F8BD39463046FFF715
:1047800088F8A8420ED1002C02DD20460BF012F86A
:1047900039463046FFF77DF8A84201D10120EBE70A
:1047A0000020E9E70020E7E7014802490860704778
:1047B0005A5A34120014014010B501210448FDF783
:1047C00047F9062003494860FFF7EEFF10BD0000DF
:1047D00005000001001401401CB5002000900120DC
:1047E000694608716846FDF7C7F90120FDF79EF894
:1047F0001CBD00000A20054908600548008CC0B2B5
:104800000449C861052001490860704700E0014083
:1048100000FBFF1F00F801401FB5002401211948CB
:10482000FDF716F902211848FCF709FE0421164885
:10483000FCF705FE0120FDF713FA07200002FDF743
:1048400021FA05200AF0B6FF0120FDF74DF805E03A
:1048500019200002844200D304E0641CFDF758F8DC
:104860000028F5D000BF01200090002001900290A8
:104870000120694608736846FDF7E2F903480AF02B
:1048800075FF1FBD07000001400D0040001BB70071
:1048900010B50020FEF78EF9FFF79EFFFFF7AAFF85
:1048A000FFF7BAFF10BD7FB506460D4614466A46AF
:1048B00029463046FEF7FCFD0098A84217D168460D
:1048C000C079012813D16846407901280FD1002C06
:1048D00003D168468079002809D1012C03D16846AC
:1048E0008079012803D168460079002814D0029508
:1048F00001216846C1734173002C03D10020694631
:10490000887302E0012069468873002069460873B5
:1049100002A93046FEF784FF7FBD0000F8B50546CA
:104920000E4600240027FCF737FF002802D10120A3
:10493000FCF73EFF002426E00120A0400746284661
:10494000384000281ED0002E07D1144840680121AD
:10495000A14088431149486006E0104840680121A1
:10496000A14008430D4948600C488168620003205B
:10497000904081430948816000680121A1400843BB
:1049800006490860641C042CD6D3FCF705FF0128F7
:1049900002D10020FCF70CFFF8BD000000FC014034
:1049A000FFB587B015461E4600200490002D01D1AA
:1049B0000BB0F0BD32780192D217130F019A9A18FA
:1049C00012110A235A433178CB171B0F5B181B11A6
:1049D0001B01CB1AD2183C235A4373780293DB177E
:1049E0001F0F029BFB181B110A277B437078C71708
:1049F0003F0F3F183F113F01C71BDB19D21894B27C
:104A000006946A46D27F0192D217130F019A9A1820
:104A100013110A2253436A46D17FCA17120F521844
:104A2000121112018A1A9B183C22534308AA1278C9
:104A30000292D217170F029ABA1812110A277A4354
:104A400008AF3878C7173F0F3F183F113F01C71B0A
:104A5000D2199A1892B20592069C002D06D02946CA
:104A60002D204001FBF75CFB401C00E0012080B2E0
:104A7000039008A84078002816D1049010E005980B
:104A8000844201D1012093E7601984B22D204001B6
:104A9000844201DB201A84B20498401C80B2049046
:104AA000039904988842EADB002081E710B50024CE
:104AB0000A20FCF789FA09240AE000F071FA00F0F4
:104AC000BBFA2046FCF780FA00F00CF8601EC4B276
:104AD000002CF2DC00F064FA00F0AEFA0020FCF7E3
:104AE00073FA10BD30B589B0002008904FE20898E5
:104AF0008000FE490968085C079008988000FB491F
:104B0000096840184078069008988100F7480068C6
:104B100008188078059008988000F44909684018C2
:104B2000C078049007980DF08BFA044607980DF0B2
:104B300087FA03900DF084FA444007980DF080FA4C
:104B400002900DF07DFA03900DF07AFA4440079838
:104B50000DF076FA01900DF073FA02900DF070FAF4
:104B600003900DF06DFA06980DF06AFA0546069866
:104B700045400DF065FA03900DF062FA06980DF0CD
:104B80005FFA02900DF05CFA03900DF059FA45407F
:104B900006980DF055FA01900DF052FA02900DF0C2
:104BA0004FFA03900DF04CFA6C4005980DF048FA5E
:104BB000059805460DF044FA03900DF041FA454082
:104BC00005980DF03DFA02900DF03AFA03900DF0C1
:104BD00037FA454005980DF033FA01900DF030FAA0
:104BE00002900DF02DFA03900DF02AFA6C40049813
:104BF0000DF026FA049805460DF022FA03900DF008
:104C00001FFA04980DF01CFA02900DF019FA0390A7
:104C10000DF016FA454004980DF012FA01900DF0CF
:104C20000FFA02900DF00CFA03900DF009FA6C40A7
:104C300008988000AD4909680C5407980DF000FAF7
:104C4000079804460DF0FCF903900DF0F9F9079868
:104C50000DF0F6F902900DF0F3F903900DF0F0F974
:104C6000444007980DF0ECF901900DF0E9F902903D
:104C70000DF0E6F903900DF0E3F906980DF0E0F978
:104C8000054606980DF0DCF903900DF0D9F9454082
:104C900006980DF0D5F902900DF0D2F903900DF0C1
:104CA000CFF9454006980DF0CBF901900DF0C8F909
:104CB00002900DF0C5F903900DF0C2F96C40059813
:104CC0000DF0BEF90546059845400DF0B9F9039081
:104CD0000DF0B6F905980DF0B3F902900DF0B0F9AA
:104CE00003900DF0ADF9454005980DF0A9F901903C
:104CF0000DF0A6F902900DF0A3F903900DF0A0F9C4
:104D00006C4004980DF09CF9049805460DF098F954
:104D100003900DF095F9454004980DF091F902903B
:104D20000DF08EF903900DF08BF9454004980DF0CD
:104D300087F901900DF084F902900DF081F903904C
:104D40000DF07EF96C4008988000684909684018A9
:104D5000447007980DF074F9079804460DF070F947
:104D600003900DF06DF9444007980DF069F9029039
:104D70000DF066F903900DF063F9444007980DF0CB
:104D80005FF901900DF05CF902900DF059F9039074
:104D90000DF056F906980DF053F9069805460DF0FA
:104DA0004FF903900DF04CF906980DF049F9029077
:104DB0000DF046F903900DF043F9454006980DF0CB
:104DC0003FF901900DF03CF902900DF039F9039094
:104DD0000DF036F96C4005980DF032F9054605984E
:104DE0000DF02EF903900DF02BF9454005980DF0CC
:104DF00027F902900DF024F903900DF021F94540B8
:104E000005980DF01DF901900DF01AF902900DF0C2
:104E100017F903900DF014F96C4004980DF010F997
:104E20000546049845400DF00BF903900DF008F984
:104E300004980DF005F902900DF002F903900DF0C1
:104E4000FFF8454004980DF0FBF801900DF0F8F8DC
:104E500002900DF0F5F803900DF0F2F86C40089810
:104E60008000224A12688018847007980DF0E8F8D4
:104E70000446079844400DF0E3F803900DF0E0F885
:104E800007980DF0DDF802900DF0DAF803900DF0C0
:104E9000D7F8444007980DF0D3F801900DF0D0F802
:104EA00002900DF0CDF803900DF0CAF806980DF0C1
:104EB000C7F8069805460DF0C3F803900DF0C0F84A
:104EC000454006980DF0BCF802900DF0B9F803903B
:104ED0000DF0B6F8454006980DF0B2F801900DF0CF
:104EE000AFF802900DF0ACF8039001E00000002054
:104EF0000DF0A6F86C4005980DF0A2F8059805464F
:104F00000DF09EF803900DF09BF805980DF098F8C1
:104F100002900DF095F803900DF092F84540059839
:104F20000DF08EF801900DF08BF802900DF088F8DE
:104F300003900DF085F86C4004980DF081F805465B
:104F400004980DF07DF803900DF07AF84540049830
:104F50000DF076F802900DF073F803900DF070F8F4
:104F6000454004980DF06CF801900DF069F802903E
:104F70000DF066F803900DF063F86C40089880001F
:104F8000064A12688018C4700898401C0890089857
:104F9000042800DAABE509B030BD000000000020B5
:104FA00024490968487B234909684A7A21490968E4
:104FB0004A73204909684A791E4909684A721D499D
:104FC00009684A781B4909684A711A490968487092
:104FD00018490968887817490968897A154A126852
:104FE00091701449096888721249096888791149D1
:104FF00009688A7B0F4909688A710E4909688873B4
:105000000C490968C8780B490968C979094A1268C6
:10501000D17008490968CA7A06490968CA71054900
:105020000968CA7B03490968CA7202490968C873DA
:10503000704700000000002070B5002413E0002538
:105040000DE0A900094A12688918085D0BF04AFAB8
:10505000A900064A126889180855681CC5B2042DB3
:10506000EFDB601CC4B2042CE9DB70BD0000002043
:10507000F8B500241FE0A00043490968095CA000BE
:10508000424A1154A000401C3F490968095CA00035
:10509000401C1154A000801C3B490968095CA00019
:1050A000801C1154A000C01C37490968095CA0008D
:1050B000C01C1154641C042CDDD362E0002507E001
:1050C000601E800040193149085C694648556D1CD6
:1050D000042DF5D3A007800F002825D16846067857
:1050E0004178017081784170C1788170C6706946DD
:1050F00008780BF0FDF96946087048780BF0F8F96C
:105100006946487088780BF0F3F969468870C8786A
:105110000BF0EEF96946C8700878A1081C4A515C8A
:1051200048406946087000E000BF201F8000174912
:10513000085C694609784840A100144A5054201F71
:105140008000401C1146095C684640784840A10038
:10515000491C5054201F8000801C1146095C684681
:1051600080784840A100891C5054201F8000C01C3A
:105170001146085C6946C9784840A100C91C5054D2
:10518000641C2C2C9AD3F8BD0400002010080020C9
:105190005222010010B50022012149020848FFF700
:1051A00082FB00220121C90305484030FFF77BFB49
:1051B00000220121890302484030FFF774FB10BD33
:1051C000000D004010B501210448FCF741FC00220D
:1051D00020210348FFF767FB10BD00000700000116
:1051E000800C004010B501210348FCF731FC202160
:1051F0000248FCF7E5FD10BD07000001800C0040EF
:1052000004488069C007C00F002801D00120704702
:105210000020FCE70034014010B500F009F8012837
:1052200005D1FFF7EDFF012801D100F00DF810BD09
:105230000448406940210840002801D001207047FF
:105240000020FCE7003401404020014948617047DC
:105250000034014010B501210648FCF7F9FB00229B
:105260000121054805F08CFE01210348FEF71BFBD8
:1052700010BD000007000001000C004010B5012126
:105280000648FCF7E5FB00220221054805F078FE00
:1052900002210348FEF707FB10BD000007000001D4
:1052A000000C00400FB4394880782021084337496A
:1052B00088703748407904210840002832D13348AB
:1052C0004078202108433149487069461520085626
:1052D000002805DD2D484078402108432B494870BF
:1052E000694615200856142805DD28484078802195
:1052F000084326494870694615200856282805DDC8
:10530000224880788021084320498870694615200A
:105310000856462838DD1D488078402108431B493F
:10532000887031E0194840781021084317494870C7
:10533000694616200856002805DD144840784021AB
:10534000084312494870694616200856142805DD9E
:105350000E484078802108430C4948706946162061
:105360000856282805DD0948807880210843074928
:105370008870694616200856462805DD034880785F
:10538000402108430149887004B070479A1C0020EE
:10539000CC020020012801D002281AD1022805D110
:1053A0000C4A927802231A430A4B9A70002908DDAE
:1053B000084A203A527A10231A43064B203B5A726D
:1053C00007E0044A203A127A10231A43014B203B8B
:1053D0001A7270479A1C002010B5012204498420DB
:1053E00004F072FE01210348FEF75DFA10BD0000D3
:1053F00076060020400D004000B5152801D304F0CA
:10540000A1FB43007B449B885B009F449B231400CB
:10541000D40197035A051D07DB089A0A780C380E49
:10542000F40FB41174133415F216DF18D11A931C4B
:10543000561E1920D9210B0009F0D3FD0A06315C54
:1054400087B2DDFEFDFCFBFAFE4A527880231A4348
:10545000FC4B5A701A46927880231A43F94B9A7083
:105460001A46927820231A43F64B9A701A465278BD
:1054700010231A43F34B5A701A46527820231A43CA
:10548000F04B5A701A46527840231A43ED4B5A702B
:105490001A46927840239A43EA4B9A7089E1E94A86
:1054A000527880239A43E74B5A701A4692788023A9
:1054B0001A43E44B9A701A46927820231A43E14B20
:1054C0009A701A46527810239A43DE4B5A701A4645
:1054D000527820239A43DB4B5A701A465278402365
:1054E0009A43D84B5A701A46927840239A43D54B28
:1054F0009A705EE1D34A527880231A43D14B5A7096
:105500001A46927880231A43CE4B9A701A469278A4
:1055100020239A43CB4B9A701A46527810231A4391
:10552000C84B5A701A46527820231A43C54B5A70FA
:105530001A46527840239A43C24B5A701A469278C0
:1055400040231A43BF4B9A7033E1BE4A52788023FE
:105550001A43BC4B5A701A46927880231A43B94BAF
:105560009A701A46927820231A43B64B9A701A46BC
:10557000527810231A43B34B5A701A46527820239C
:105580009A43B04B5A701A46527840239A43AD4B17
:105590005A701A46927840231A43AA4B9A7008E12F
:1055A000A84A527880239A43A64B5A701A4692789A
:1055B00080231A43A34B9A701A46927820231A43E9
:1055C000A04B9A701A46527810239A439D4B5A70FA
:1055D0001A46527820239A439A4B5A701A465278A8
:1055E00040231A43974B5A701A46927840231A4325
:1055F000944B9A70DDE0934A527880231A43914B82
:105600005A701A46927880239A438E4B9A701A46A3
:10561000927820231A438B4B9A701A4652781023A3
:105620001A43884B5A701A46527820239A4304E052
:10563000BEE092E066E03AE00EE0824B5A701A4615
:10564000527840231A437F4B5A701A46927840236F
:105650001A437C4B9A70ACE07A4A527880231A4302
:10566000784B5A701A46927880239A43754B9A70F9
:105670001A46927820231A43724B9A701A4652782F
:1056800010231A436F4B5A701A46527820231A433C
:105690006C4B5A701A46527840231A43694B5A7021
:1056A0001A46927840231A43664B9A7081E0654A05
:1056B000527880231A43634B5A701A46927880239B
:1056C0001A43604B9A701A46927820231A435D4B16
:1056D0009A701A46527810239A435A4B5A701A46B7
:1056E000527820239A43574B5A701A4652784023D7
:1056F0009A43544B5A701A46927840239A43514B1E
:105700009A7056E04F4A527880231A434D4B5A7094
:105710001A46927880231A434A4B9A701A46927816
:1057200020231A43474B9A701A46527810231A4383
:10573000444B5A701A46527820231A43414B5A70F0
:105740001A46527840231A433E4B5A701A469278B2
:1057500040231A433B4B9A702BE03A4A52788023FD
:105760001A43384B5A701A46927880231A43354BA5
:105770009A701A46927820231A43324B9A701A462E
:10578000527810231A432F4B5A701A46527820230E
:105790009A432C4B5A701A46527840231A43294B8D
:1057A0005A701A46927840231A43264B9A7000E0AA
:1057B00000BF00BF23E60B0009F013FC0A06315FAF
:1057C0008AB5E0FEFDFCFBFA1E4AD27880231A431C
:1057D0001C4BDA701A46D27940231A43194BDA71FE
:1057E0001A46D27920231A43164BDA711A46D27818
:1057F00010231A43134BDA701A46927810231A4377
:10580000104B9A701A46D27840231A430D4BDA7027
:105810001A46D27820239A430A4BDA708CE1094A5F
:10582000D27880239A43074BDA701A46D279402304
:105830001A43044BDA711A46D27920231A43014BDA
:10584000DA7101E07A1C00201A46D27810239A43BC
:10585000FE4BDA701A46927810239A43FB4B9A70EB
:105860001A46D27840239A43F84BDA701A46D27817
:1058700020239A43F54BDA705EE1F44AD278802314
:105880001A43F24BDA701A46D27940231A43EF4B8F
:10589000DA711A46D27920239A43EC4BDA711A4610
:1058A000D27810231A43E94BDA701A469278102303
:1058B0001A43E64B9A701A46D27840239A43E34B38
:1058C000DA701A46D27820231A43E04BDA7033E1BB
:1058D000DE4AD27880231A43DC4BDA701A46D2793A
:1058E00040231A43D94BDA711A46D27920231A433E
:1058F000D64BDA711A46D27810231A43D34BDA709A
:105900001A46927810239A43D04B9A701A46D2784E
:1059100040239A43CD4BDA701A46D27820231A439B
:10592000CA4BDA7008E1C94AD27880239A43C74B40
:10593000DA701A46D27940231A43C44BDA711A46F8
:10594000D27920231A43C14BDA711A46D278102338
:105950009A43BE4BDA701A46927810239A43BB4B97
:105960009A701A46D27840231A43B84BDA701A4616
:10597000D27820231A43B54BDA70DDE0B34AD278EF
:1059800080231A43B14BDA701A46D27940239A43E6
:10599000AE4BDA711A46D27920231A43AB4BDA7137
:1059A0001A46D27810231A43A84BDA701A4604E03C
:1059B000C1E095E069E03DE011E0927810239A4360
:1059C000A24B9A701A46D27840231A439F4BDA7042
:1059D0001A46D27820231A439C4BDA70ACE09B4ADB
:1059E000D27880231A43994BDA701A46D279402331
:1059F0009A43964BDA711A46D27920231A43934B75
:105A0000DA711A46D27810231A43904BDA701A468C
:105A1000927810231A438D4B9A701A46D2784023FD
:105A20001A438A4BDA701A46D27820231A43874BDE
:105A3000DA7081E0854AD27880231A43834BDA708A
:105A40001A46D27940231A43804BDA711A46D2792A
:105A500020231A437D4BDA711A46D27810239A43D9
:105A60007A4BDA701A46927810239A43774B9A70E1
:105A70001A46D27840239A43744BDA701A46D27889
:105A800020239A43714BDA7056E0704AD278802313
:105A90001A436E4BDA701A46D27940231A436B4B85
:105AA000DA711A46D27920231A43684BDA711A4602
:105AB000D27810231A43654BDA701A469278102375
:105AC0001A43624B9A701A46D27840231A435F4BAE
:105AD000DA701A46D27820231A435C4BDA702BE036
:105AE0005A4AD27880231A43584BDA701A46D27930
:105AF00040231A43554BDA711A46D27920231A43B0
:105B0000524BDA711A46D27810231A434F4BDA708F
:105B10001A46927810239A434C4B9A701A46D278C0
:105B200040231A43494BDA701A46D27820231A438D
:105B3000464BDA7000E000BF00BF60E40B0009F0E4
:105B400050FA0A06315C8AB5E0FDFCFBFAF93F4ADF
:105B5000D27A80231A433D4BDA721A46D27A402316
:105B60001A433A4BDA721A46D27A20231A43374B39
:105B7000DA721A46D27A10231A43344BDA721A4672
:105B8000927A10231A43314B9A721A46927A402322
:105B90001A432E4B9A721A46927A20239A432B4B21
:105BA0009A728CE1294AD27A80239A43274BDA727F
:105BB0001A46D27A40231A43244BDA721A46D27A12
:105BC00020231A43214BDA721A46D27A10239A43C1
:105BD0001E4BDA721A46927A10239A431B4B9A7222
:105BE0001A46927A40239A43184B9A721A46927A2E
:105BF00020239A43154B9A7261E1144AD27A80238A
:105C00001A43124BDA721A46D27A40231A430F4BC8
:105C1000DA721A46D27A20239A430C4BDA721A4669
:105C2000D27A10231A43094BDA721A46927A102359
:105C30001A43064B9A721A46927A40239A43034BB0
:105C40009A721A46927A20231A4301E07A1C0020A5
:105C5000FE4B9A7233E1FD4AD27A80231A43FB4B02
:105C6000DA721A46D27A40231A43F84BDA721A468D
:105C7000D27A20231A43F54BDA721A46D27A1023CD
:105C80001A43F24BDA721A46927A10239A43EF4B78
:105C90009A721A46927A40239A43EC4B9A721A46A9
:105CA000927A20231A43E94B9A7208E1E74AD27AA2
:105CB00080239A43E54BDA721A46D27A40231A437C
:105CC000E24BDA721A46D27A20231A43DF4BDA7299
:105CD0001A46D27A10239A43DC4BDA721A46927A29
:105CE00010239A43D94B9A721A46927A40231A4348
:105CF000D64B9A721A46927A20231A43D34B9A7241
:105D0000DDE0D24AD27A80231A43D04BDA721A46A7
:105D1000D27A40239A43CD4BDA721A46D27A2023A4
:105D20001A43CA4BDA721A46D27A10231A43C74B67
:105D3000DA7204E0C2E096E06AE03EE012E01A4661
:105D4000927A10239A43C14B9A721A46927A402350
:105D50001A43BE4B9A721A46927A20231A43BB4BBF
:105D60009A72ACE0B94AD27A80231A43B74BDA72FE
:105D70001A46D27A40239A43B44BDA721A46D27A40
:105D800020231A43B14BDA721A46D27A10231A43EF
:105D9000AE4BDA721A46927A10231A43AB4B9A72C0
:105DA0001A46927A40231A43A84B9A721A46927A5C
:105DB00020231A43A54B9A7281E0A44AD27A802309
:105DC0001A43A24BDA721A46D27A40231A439F4BE7
:105DD000DA721A46D27A20231A439C4BDA721A4698
:105DE000D27A10239A43994BDA721A46927A102388
:105DF0009A43964B9A721A46927A40239A43934B4F
:105E00009A721A46927A20239A43904B9A7256E0DD
:105E10008E4AD27A80231A438C4BDA721A46D27A8F
:105E200040231A43894BDA721A46D27A20231A4346
:105E3000864BDA721A46D27A10231A43834BDA72EF
:105E40001A46927A10231A43804B9A721A46927A13
:105E500040231A437D4B9A721A46927A20231A43A2
:105E60007A4B9A722BE0794AD27A80231A43774B85
:105E7000DA721A46D27A40231A43744BDA721A46FF
:105E8000D27A20231A43714BDA721A46D27A10233F
:105E90001A436E4BDA721A46927A10239A436B4B6E
:105EA0009A721A46927A40231A43684B9A721A469B
:105EB000927A20231A43654B9A7200E000BF00BF1C
:105EC00078E40B0009F08DF80A06315C87B2E0FE39
:105ED000FDFCFBFA5D4AD27A01231A435B4BDA726E
:105EE0001A46927A02231A43584B9A721A46927AA9
:105EF00008231A43554B9A721A46D27A08231A433A
:105F0000524BDA721A46D27A04231A434F4BDA7292
:105F10001A46D27A02231A434C4BDA721A46927A04
:105F200004239A43494B9A728CE1484AD27A520828
:105F30005200464BDA721A46927A02231A43434BB6
:105F40009A721A46927A08231A43404B9A721A465A
:105F5000D27A08239A433D4BDA721A46D27A042346
:105F60009A433A4BDA721A46D27A02239A43374B53
:105F7000DA721A46927A04239A43344B9A7261E198
:105F8000324AD27A01231A43304BDA721A46927A95
:105F900002231A432D4B9A721A46927A08239A4387
:105FA0002A4B9A721A46D27A08231A43274BDA727E
:105FB0001A46D27A04231A43244BDA721A46D27A4A
:105FC00002239A43214BDA721A46927A04231A4327
:105FD0001E4B9A7236E11D4AD27A01231A431B4B9B
:105FE000DA721A46927A02231A43184B9A721A46A8
:105FF000927A08231A43154B9A721A46D27A0823CA
:106000001A43124BDA721A46D27A04239A430F4B80
:10601000DA721A46D27A02239A430C4BDA721A4683
:10602000927A04231A43094B9A720BE1074AD27AF7
:1060300052085200054BDA721A46927A02231A432A
:10604000024B9A721A46927A082301E07A1C0020C9
:106050001A43FB4B9A721A46D27A08239A43F84B9A
:10606000DA721A46D27A04239A43F54BDA721A4648
:10607000D27A02231A43F24BDA721A46927A042336
:106080001A43EF4B9A72DDE0ED4AD27A01231A43AC
:10609000EB4BDA721A46927A02239A43E84B9A72D1
:1060A0001A46927A08231A43E54B9A721A46D27A14
:1060B00008231A43E24BDA721A4604E0C1E095E085
:1060C00069E03DE011E0D27A04239A43DC4BDA72B6
:1060D0001A46D27A02231A43D94BDA721A46927AB6
:1060E00004231A43D64B9A72ACE0D54AD27A0123E4
:1060F0001A43D34BDA721A46927A02239A43D04B50
:106100009A721A46927A08231A43CD4B9A721A460B
:10611000D27A08231A43CA4BDA721A46D27A042377
:106120001A43C74BDA721A46D27A02231A43C44B77
:10613000DA721A46927A04231A43C14B9A7281E0AA
:10614000BF4AD27A01231A43BD4BDA721A46927AB9
:1061500002231A43BA4B9A721A46927A08231A43B8
:10616000B74B9A721A46D27A08239A43B44BDA7222
:106170001A46D27A04239A43B14BDA721A46D27A7B
:1061800002239A43AE4BDA721A46927A04239A4358
:10619000AB4B9A7256E0AA4AD27A01231A43A84B13
:1061A000DA721A46927A02231A43A54B9A721A4659
:1061B000927A08231A43A24B9A721A46D27A08237B
:1061C0001A439F4BDA721A46D27A04231A439C4B25
:1061D000DA721A46D27A02231A43994BDA721A46B5
:1061E000927A04231A43964B9A722BE0944AD27AFD
:1061F00001231A43924BDA721A46927A02231A4307
:106200008F4B9A721A46927A08231A438C4B9A72D1
:106210001A46D27A08231A43894BDA721A46D27A7E
:1062200004239A43864BDA721A46D27A02231A431F
:10623000834BDA721A46927A04231A43804B9A727D
:1062400000E000BF00BF78E40B0008F0CAFE0A06B9
:10625000315B85B0DAFFFEFDFCFB794A52780823FA
:106260001A43774B5A701A46927804231A43744B98
:106270009A701A46927801231A43714B9A701A4603
:10628000527801231A436E4B5A701A4652780223F1
:106290001A436B4B5A701A46527804231A43684BC0
:1062A0005A701A46927802239A43654B9A7087E196
:1062B000634A527808239A43614B5A701A4692787F
:1062C00004231A435E4B9A701A46927801231A43AC
:1062D0005B4B9A701A465278520852005A701A460E
:1062E000527802239A43564B5A701A465278042326
:1062F0009A43534B5A701A46927802239A43504B52
:106300009A705DE14E4A527808231A434C4B5A70FA
:106310001A46927804231A43494B9A701A46927887
:10632000520852009A701A46527801231A43444B7D
:106330005A701A46527802231A43414B5A701A4631
:10634000527804239A433E4B5A701A46927802239D
:106350001A433B4B9A7033E1394A527808231A4367
:10636000374B5A701A46927804231A43344B9A706A
:106370001A46927801231A43314B9A701A46527882
:1063800001231A432E4B5A701A46527802239A431D
:106390002B4B5A701A46527804239A43284B5A7052
:1063A0001A46927802231A43254B9A7008E1244A30
:1063B000527808239A43224B5A701A469278042343
:1063C0001A431F4B9A701A46927801231A431C4BAA
:1063D0009A701A465278520852005A701A465278E9
:1063E00002239A43164B5A701A46527804231A43D2
:1063F000134B5A701A46927802231A43104B9A7024
:10640000DEE00F4A527808231A430D4B5A701A46A1
:10641000927804239A430A4B9A701A469278012381
:106420001A43074B9A701A46527801231A43044BB9
:106430005A701A46527802239A43014B5A7006E06A
:106440007A1C0020BBE08FE063E038E00CE01A46E5
:10645000527804231A43F84B5A701A469278022352
:106460001A43F54B9A70ABE0F34A527808231A436B
:10647000F14B5A701A46927804239A43EE4B9A7065
:106480001A46927801231A43EB4B9A701A465278B7
:1064900001231A43E84B5A701A46527802231A43D2
:1064A000E54B5A701A46527804231A43E24B5A704D
:1064B0001A46927802231A43DF4B9A7080E0DE4A34
:1064C000527808231A43DC4B5A701A4692780423F8
:1064D0001A43D94B9A701A46927801231A43D64B25
:1064E0009A701A465278520852005A701A465278D8
:1064F00002239A43D04B5A701A46527804239A4387
:10650000CD4B5A701A46927802239A43CA4B9A701E
:1065100056E0C94A527808231A43C74B5A701A46A4
:10652000927804231A43C44B9A701A469278012336
:106530001A43C14B9A701A46527801231A43BE4B34
:106540005A701A46527802231A43BB4B5A701A46A5
:10655000527804231A43B84B5A701A469278022391
:106560001A43B54B9A702BE0B34A527808231A436A
:10657000B14B5A701A46927804231A43AE4B9A7064
:106580001A46927801231A43AB4B9A701A465278F6
:1065900001231A43A84B5A701A46527802239A4391
:1065A000A54B5A701A46527804231A43A24B5A70CC
:1065B0001A46927802231A439F4B9A7000E000BF5C
:1065C00000BF7DE40B0008F00CFD0A06315B86B1CC
:1065D000DBFDFCFBFAF9984AD27908231A43964B63
:1065E000DA711A46D27904231A43934BDA711A46A8
:1065F000D27902231A43904BDA711A46D2790123D9
:106600001A438D4BDA711A46D27802231A438A4B09
:10661000DA701A46D27808231A43874BDA701A4682
:10662000D27804239A43844BDA7088E1824AD27983
:1066300008239A43804BDA711A46D27904231A430D
:106640007D4BDA711A46D27902231A437A4BDA71FA
:106650001A46D27952085200DA711A46D2780223C9
:106660009A43754BDA701A46D27808239A43724BD4
:10667000DA701A46D27804239A436F4BDA705EE1DF
:106680006D4AD27908231A436B4BDA711A46D279D4
:1066900004231A43684BDA711A46D27902239A43CB
:1066A000654BDA711A46D27901231A43624BDA71CB
:1066B0001A46D27802231A435F4BDA701A46D27810
:1066C00008239A435C4BDA701A46D27804231A43A3
:1066D000594BDA7033E1584AD27908231A43564BA2
:1066E000DA711A46D27904231A43534BDA711A46E7
:1066F000D27902231A43504BDA711A46D279012318
:106700001A434D4BDA711A46D27802239A434A4B08
:10671000DA701A46D27808239A43474BDA701A4641
:10672000D27804231A43444BDA7008E1424AD27902
:1067300008239A43404BDA711A46D27904231A434C
:106740003D4BDA711A46D27902231A433A4BDA7179
:106750001A46D27952085200DA711A46D2780223C8
:106760009A43354BDA701A46D27808231A43324BD3
:10677000DA701A46D27804231A432F4BDA70DEE01F
:106780002D4AD27908231A432B4BDA711A46D27953
:1067900004239A43284BDA711A46D27902231A430A
:1067A000254BDA711A46D27901231A43224BDA714A
:1067B0001A46D27802239A431F4B04E0BEE092E0CF
:1067C00066E03BE00DE0DA701A46D27808231A43FF
:1067D000194BDA701A46D27804231A43164BDA7032
:1067E000ADE0154AD27908231A43134BDA711A46E1
:1067F000D27904239A43104BDA711A46D2790223D4
:106800001A430D4BDA711A46D27901231A430A4B07
:10681000DA711A46D27802231A43074BDA701A4605
:10682000D27808231A43044BDA701A46D27804232C
:106830001A43014BDA7082E07A1C0020FE4AD279BA
:1068400008231A43FC4BDA711A46D27904231A43FF
:10685000F94BDA711A46D27902231A43F64BDA71F0
:106860001A46D27952085200DA711A46D2780223B7
:106870009A43F14BDA701A46D27808239A43EE4BCA
:10688000DA701A46D27804239A43EB4BDA7056E05A
:10689000E94AD27908231A43E74BDA711A46D279CA
:1068A00004231A43E44BDA711A46D27902231A43BD
:1068B000E14BDA711A46D27901231A43DE4BDA71C1
:1068C0001A46D27802231A43DB4BDA701A46D27882
:1068D00008231A43D84BDA701A46D27804231A4395
:1068E000D54BDA702BE0D44AD27908231A43D24B25
:1068F000DA711A46D27904231A43CF4BDA711A4659
:10690000D27902231A43CC4BDA711A46D279012389
:106910001A43C94BDA711A46D27802239A43C64BFE
:10692000DA701A46D27808231A43C34BDA701A4633
:10693000D27804231A43C04BDA7000E000BF00BFD6
:1069400081E40B0008F04DFB0A0634618FBDF0EEC8
:10695000EDECEBEAB84AD27F08231A43B64BDA775C
:106960001A46927F08231A43B34B9A771A46D27F6E
:1069700002231A43B04BDA771A46D27F01231A4317
:10698000AD4BDA771A462032127802231A43AA4B0B
:1069900020331A701A46127808231A43A64B203364
:1069A0001A70A54AD27F04239A43A34BDA77A4E155
:1069B000A14AD27F08239A439F4BDA771A46927FE7
:1069C00008231A439C4B9A771A46D27F02231A4314
:1069D000994BDA771A46D27F52085200DA771A4674
:1069E0002032127802239A43934B20331A701A46AE
:1069F000127808239A43904B20331A708E4AD27F24
:106A000004239A438C4BDA7777E18B4AD27F0823B1
:106A10001A43894BDA771A46927F08231A43864B2A
:106A20009A771A46D27F02239A43834BDA771A4623
:106A3000D27F01231A43804BDA771A46203212782C
:106A400002231A437C4B20331A701A46127808230B
:106A50009A43794B20331A70774AD27F04231A4322
:106A6000754BDA7749E1744AD27F08231A43724B97
:106A7000DA771A46927F08231A436F4B9A771A46A1
:106A8000D27F02231A436C4BDA771A46D27F012356
:106A90001A43694BDA771A462032127802239A4356
:106AA000654B20331A701A46127808239A43624BBA
:106AB00020331A70604AD27F04231A435E4BDA7780
:106AC0001BE15D4AD27F08239A435B4BDA771A4673
:106AD000927F08231A43584B9A771A46D27F022393
:106AE0001A43554BDA771A46D27F52085200DA77AA
:106AF0001A462032127802239A434F4B20331A70E1
:106B00001A46127808231A434B4B20331A704A4A0C
:106B1000D27F04231A43484BDA77EEE0ECE0BDE085
:106B20008EE05DE02EE0FFE7434AD27F08231A4360
:106B3000414BDA771A46927F08239A433E4B9A7765
:106B40001A46D27F02231A433B4BDA771A46D27F8A
:106B500001231A43384BDA771A462032127802237F
:106B60009A43354B20331A701A46127808231A4379
:106B7000314B20331A70304AD27F04231A432E4BF4
:106B8000DA77BAE02C4AD27F08231A432A4BDA7705
:106B90001A46927F08239A43274B9A771A46D27F48
:106BA00002231A43244BDA771A46D27F01231A4371
:106BB000214BDA771A462032127802231A431E4BF1
:106BC00020331A701A46127808231A431A4B2033BE
:106BD0001A70194AD27F04231A43174BDA778CE0D4
:106BE000154AD27F08231A43134BDA771A46927F4D
:106BF00008231A43104B9A771A46D27F02231A436E
:106C00000D4BDA771A46D27F52085200DA771A46CD
:106C10002032127802239A43074B20331A701A4607
:106C2000127808239A43044B20331A70024AD27F09
:106C300004239A43004B01E07A1C0020DA775CE0E1
:106C4000FE4AD27F08231A43FC4BDA771A46927F1A
:106C500008231A43F94B9A771A46D27F02231A4324
:106C6000F64BDA771A46D27F01231A43F34BDA77D1
:106C70001A462032127802231A43F04B20331A703E
:106C80001A46127808231A43EC4B20331A70EB4A49
:106C9000D27F04231A43E94BDA772EE0E74AD27F0A
:106CA00008231A43E54BDA771A46927F08231A43E2
:106CB000E24B9A771A46D27F02231A43DF4BDA77E8
:106CC0001A46D27F01231A43DC4BDA771A46203268
:106CD000127802239A43D94B20331A701A4612783D
:106CE00008231A43D54B20331A70D44AD27F042389
:106CF0001A43D24BDA7700E000BF00BF61E40B001B
:106D000008F06FF90A06315B86B1DBFEFDFCFBFA89
:106D1000CA4A527F08231A43C84B5A771A46127F31
:106D200004231A43C54B1A771A46127F02231A43CB
:106D3000C24B1A771A46527F01231A43BF4B5A7728
:106D40001A46927F02231A43BC4B9A771A46527F07
:106D500004231A43B94B5A771A46527F02239A43A7
:106D6000B64B5A7789E1B54A527F08239A43B34B11
:106D70005A771A46127F04231A43B04B1A771A46E1
:106D8000127F02231A43AD4B1A771A46527F5208DC
:106D900052005A771A46927F02239A43A74B9A775A
:106DA0001A46527F04239A43A44B5A771A46527FBD
:106DB00002239A43A14B5A775FE1A04A527F0823EE
:106DC0001A439E4B5A771A46127F04231A439B4B51
:106DD0001A771A46127F02239A43984B1A771A465B
:106DE000527F01231A43954B5A771A46927F02230A
:106DF0001A43924B9A771A46527F04239A438F4B39
:106E00005A771A46527F02231A438C4B5A7734E141
:106E10008A4A527F08231A43884B5A771A46127FB0
:106E200004231A43854B1A771A46127F02231A430A
:106E3000824B1A771A46527F01231A437F4B5A77A7
:106E40001A46927F02239A437C4B9A771A46527FC6
:106E500004239A43794B5A771A46527F02231A43E6
:106E6000764B5A7709E1754A527F08239A43734B50
:106E70005A771A46127F04231A43704B1A771A4620
:106E8000127F02231A436D4B1A771A46527F52081B
:106E900052005A771A46927F02239A43674B9A7799
:106EA0001A46527F04231A43644B5A771A46527F7C
:106EB00002231A43614B5A77DFE0604A527F08236E
:106EC0001A435E4B5A771A46127F04239A435B4B50
:106ED0001A771A46127F02231A43584B1A771A461A
:106EE000527F01231A43554B5A771A46927F022349
:106EF0009A43524B9A7704E0BEE08FE063E038E0BB
:106F00000CE01A46527F04231A434C4B5A771A4618
:106F1000527F02231A43494B5A77AEE0474A527FC9
:106F200008231A43454B5A771A46127F04239A4383
:106F3000424B1A771A46127F02231A433F4B1A77A5
:106F40001A46527F01231A433C4B5A771A46927FC6
:106F500002231A43394B9A771A46527F04231A4365
:106F6000364B5A771A46527F02231A43334B5A77CD
:106F700083E0324A527F08231A43304B5A771A462D
:106F8000127F04231A432D4B1A771A46127F0223CD
:106F90001A432A4B1A771A46527F520852005A77E0
:106FA0001A46927F02239A43244B9A771A46527FBD
:106FB00004239A43214B5A771A46527F02239A435D
:106FC0001E4B5A7759E01D4A527F08231A431B4B28
:106FD0005A771A46127F04231A43184B1A771A4617
:106FE000127F02231A43154B1A771A46527F012348
:106FF0001A43124B5A771A46927F02231A430F4BB9
:107000009A771A46527F04231A430C4B5A771A4632
:10701000527F02231A43094B5A772EE0074A527FC8
:1070200008231A43054B5A771A46127F04231A4342
:10703000024B1A771A46127F022301E07A1C0020C5
:107040001A43FE4B1A771A46527F01231A43FB4B11
:107050005A771A46927F02239A43F84B9A771A4638
:10706000527F04231A43F54B5A771A46527F022364
:107070001A43F24B5A7700E000BF00BF60E40B00F8
:1070800007F0AFFF0A06315B85B0DAFEFDFCFBFAC4
:10709000EA4AD27E08231A43E84BDA761A46927EF1
:1070A00004231A43E54B9A761A46927E01231A432B
:1070B000E24B9A761A46D27E01231A43DF4BDA76E8
:1070C0001A46D27E02231A43DC4BDA761A46D27E67
:1070D00004231A43D94BDA761A46927E02239A4346
:1070E000D64B9A7685E1D54AD27E08239A43D34B74
:1070F000DA761A46927E04231A43D04B9A761A46C1
:10710000927E01231A43CD4B9A761A46D27E5208BC
:107110005200DA761A46D27E02239A43C74BDA76B9
:107120001A46D27E04239A43C44BDA761A46927EDC
:1071300002239A43C14B9A765BE1C04AD27E082370
:107140001A43BE4BDA761A46927E04231A43BB4B8F
:107150009A761A46927E520852009A761A46D27E43
:1071600001231A43B54BDA761A46D27E02231A431C
:10717000B24BDA761A46D27E04239A43AF4BDA76C4
:107180001A46927E02231A43AC4B9A7631E1AB4AFF
:10719000D27E08231A43A94BDA761A46927E04233C
:1071A0001A43A64B9A761A46927E01231A43A34BA2
:1071B0009A761A46D27E01231A43A04BDA761A46F3
:1071C000D27E02239A439D4BDA761A46D27E04235E
:1071D0009A439A4BDA761A46927E02231A43974BC9
:1071E0009A7606E1954AD27E08239A43934BDA7643
:1071F0001A46927E04231A43904B9A761A46927E40
:1072000001231A438D4B9A761A46D27E52085200B9
:10721000DA761A46D27E02239A43884BDA761A46E9
:10722000D27E04231A43854BDA761A46927E0223D5
:107230001A43824B9A76DCE0804AD27E08231A43B6
:107240007E4BDA761A46927E04239A437B4B9A76DB
:107250001A46927E01231A43784B9A761A46D27EBA
:1072600001231A43754BDA761A46D27E02239A43DB
:10727000724BDA761A4604E0BAE08EE062E037E05C
:107280000BE0D27E04231A436C4BDA761A46927EC8
:1072900002231A43694B9A76ABE0684AD27E0823F0
:1072A0001A43664BDA761A46927E04239A43634B5E
:1072B0009A761A46927E01231A43604B9A761A46B2
:1072C000D27E01231A435D4BDA761A46D27E022320
:1072D0001A435A4BDA761A46D27E04231A43574B86
:1072E000DA761A46927E02231A43544B9A7680E04D
:1072F000524AD27E08231A43504BDA761A46927EBF
:1073000004231A434D4B9A761A46927E01231A4360
:107310004A4B9A761A46D27E52085200DA761A46BC
:10732000D27E02239A43454BDA761A46D27E042354
:107330009A43424BDA761A46927E02239A433F4B97
:107340009A7656E03D4AD27E08231A433B4BDA76C2
:107350001A46927E04231A43384B9A761A46927E36
:1073600001231A43354B9A761A46D27E01231A43DB
:10737000324BDA761A46D27E02231A432F4BDA7644
:107380001A46D27E04231A432C4BDA761A46927E92
:1073900002231A43294B9A762BE0284AD27E0823EF
:1073A0001A43264BDA761A46927E04231A43234B5D
:1073B0009A761A46927E01231A43204B9A761A46F1
:1073C000D27E01231A431D4BDA761A46D27E02235F
:1073D0009A431A4BDA761A46D27E04231A43174B85
:1073E000DA761A46927E02231A43144B9A7600E00C
:1073F00000BF00BF82E40B0007F0F3FD0A06345E15
:1074000089B4DEFEFDFCFBFA0C4A127E08231A4307
:107410000A4B1A761A46127E04231A43074B1A7631
:107420001A46127E02231A43044B1A761A46127E1B
:1074300001231A43014B1A761A4601E07A1C0020F8
:10744000527E02231A43FB4B5A761A46527E082379
:107450001A43F84B5A761A46527E04239A43F54B48
:107460005A7686E1F34A127E08239A43F14B1A7644
:107470001A46127E04231A43EE4B1A761A46127EDF
:1074800002231A43EB4B1A761A46127E5208520018
:107490001A761A46527E02239A43E64B5A761A46C9
:1074A000527E08239A43E34B5A761A46527E0423AF
:1074B0009A43E04B5A765CE1DE4A127E08231A4377
:1074C000DC4B1A761A46127E04231A43D94B1A76DD
:1074D0001A46127E02239A43D64B1A761A46127E19
:1074E00001231A43D34B1A761A46527E02231A43BB
:1074F000D04B5A761A46527E08239A43CD4B5A7681
:107500001A46527E04231A43CA4B5A7631E1C94ABD
:10751000127E08231A43C74B1A761A46127E04239A
:107520001A43C44B1A761A46127E02231A43C14BE1
:107530001A761A46127E01231A43BE4B1A761A4651
:10754000527E02239A43BB4B5A761A46527E082338
:107550009A43B84B5A761A46527E04231A43B54BC7
:107560005A7606E1B34A127E08239A43B14B1A7643
:107570001A46127E04231A43AE4B1A761A46127E1E
:1075800002231A43AB4B1A761A46127E5208520057
:107590001A761A46527E02239A43A64B5A761A4608
:1075A000527E08231A43A34B5A761A46527E04236E
:1075B0001A43A04B5A76DCE09E4A127E08231A43F7
:1075C0009C4B1A761A46127E04239A43994B1A76DC
:1075D0001A46127E02231A43964B1A761A46127ED8
:1075E00001231A43934B1A761A46527E022304E073
:1075F000BEE092E066E03BE00FE09A438D4B5A76A6
:107600001A46527E08231A438A4B5A761A46527EED
:1076100004231A43874B5A76ABE0864A127E08232E
:107620001A43844B1A761A46127E04239A43814BDE
:107630001A761A46127E02231A437E4B1A761A468F
:10764000127E01231A437B4B1A761A46527E02237E
:107650001A43784B5A761A46527E08231A43754BC2
:107660005A761A46527E04231A43724B5A7680E0A9
:10767000704A127E08231A436E4B1A761A46127EFF
:1076800004231A436B4B1A761A46127E02231A43BE
:10769000684B1A761A46127E520852001A761A461B
:1076A000527E02239A43634B5A761A46527E08232F
:1076B0009A43604B5A761A46527E04239A435D4B96
:1076C0005A7656E05B4A127E08231A43594B1A76C3
:1076D0001A46127E04231A43564B1A761A46127E15
:1076E00002231A43534B1A761A46127E01231A4379
:1076F000504B1A761A46527E02231A434D4B5A7645
:107700001A46527E08231A434A4B5A761A46527E2C
:1077100004231A43474B5A762BE0464A127E08232D
:107720001A43444B1A761A46127E04231A43414BDD
:107730001A761A46127E02231A433E4B1A761A46CE
:10774000127E01231A433B4B1A761A46527E0223BD
:107750009A43384B5A761A46527E08231A43354BC1
:107760005A761A46527E04231A43324B5A7600E068
:1077700000BF00BF82E40B0007F033FC0A06315E55
:1077800089B4DEFEFDFCFBFA2A4A927D08231A43E7
:10779000284B9A751A46527D08231A43254B5A7571
:1077A0001A46927D02231A43224B9A751A46927DFD
:1077B00001231A431F4B9A751A46D27D02231A439E
:1077C0001C4BDA751A46D27D08231A43194BDA7519
:1077D0001A46927D04239A43164B9A7589E1154AFD
:1077E000927D08239A43134B9A751A46527D0823BB
:1077F0001A43104B5A751A46927D02231A430D4BB9
:107800009A751A46927D520852009A751A46D27D90
:1078100002239A43074BDA751A46D27D08239A430E
:10782000044BDA751A46927D04239A43014B9A75EC
:107830005FE100007A1C0020FE4A927D08231A4373
:10784000FC4B9A751A46527D08231A43F94B5A7518
:107850001A46927D02239A43F64B9A751A46927DF8
:1078600001231A43F34B9A751A46D27D02231A4319
:10787000F04BDA751A46D27D08239A43ED4BDA7540
:107880001A46927D04231A43EA4B9A7531E1E94A7C
:10789000927D08231A43E74B9A751A46527D0823B6
:1078A0001A43E44B5A751A46927D02231A43E14B60
:1078B0009A751A46927D01231A43DE4B9A751A4631
:1078C000D27D02239A43DB4BDA751A46D27D082318
:1078D0009A43D84BDA751A46927D04231A43D54B46
:1078E0009A7506E1D34A927D08239A43D14B9A7543
:1078F0001A46527D08231A43CE4B5A751A46927D7A
:1079000002231A43CB4B9A751A46927D52085200B5
:107910009A751A46D27D02239A43C64BDA751A46E7
:10792000D27D08231A43C34BDA751A46927D04238D
:107930001A43C04B9A75DCE0BE4A927D08231A4375
:10794000BC4B9A751A46527D08239A43B94B5A7517
:107950001A46927D02231A43B64B9A751A46927DB7
:1079600001231A43B34B9A751A46D27D022304E0D1
:10797000BEE092E066E03BE00FE09A43AD4BDA7583
:107980001A46D27D08231A43AA4BDA751A46927D0D
:1079900004231A43A74B9A75ABE0A64A927D0823AD
:1079A0001A43A44B9A751A46527D08239A43A14B59
:1079B0005A751A46927D02231A439E4B9A751A46AF
:1079C000927D01231A439B4B9A751A46D27D02235E
:1079D0001A43984BDA751A46D27D08231A43954B01
:1079E000DA751A46927D04231A43924B9A7580E009
:1079F000904A927D08231A438E4B9A751A46527DFF
:107A000008231A438B4B5A751A46927D02231A4358
:107A1000884B9A751A46927D520852009A751A46FA
:107A2000D27D02239A43834BDA751A46D27D08230E
:107A30009A43804BDA751A46927D04239A437D4B14
:107A40009A7556E07B4A927D08231A43794B9A75C2
:107A50001A46527D08231A43764B5A751A46927D70
:107A600002231A43734B9A751A46927D01231A43D7
:107A7000704B9A751A46D27D02231A436D4BDA7504
:107A80001A46D27D08231A436A4BDA751A46927D4C
:107A900004231A43674B9A752BE0664A927D0823AC
:107AA0001A43644B9A751A46527D08231A43614B58
:107AB0005A751A46927D02231A435E4B9A751A46EE
:107AC000927D01231A435B4B9A751A46D27D02239D
:107AD0009A43584BDA751A46D27D08231A43554B00
:107AE000DA751A46927D04231A43524B9A7500E0C8
:107AF00000BF00BF7EE40B0007F073FA0A06315B9B
:107B000086B4DEFEFDFCFBFA4A4A127D08231A43C6
:107B1000484B1A751A46D27C04231A43454BDA7433
:107B20001A46D27C02231A43424BDA741A46127D5B
:107B300001231A433F4B1A751A46527D02231A43FA
:107B40003C4B5A751A46127D04231A43394B1A7559
:107B50001A46127D02239A43364B1A7589E1354A3B
:107B6000127D08239A43334B1A751A46D27C04239C
:107B70001A43304BDA741A46D27C02231A432D4B37
:107B8000DA741A46127D520852001A751A46527D4E
:107B900002239A43274B5A751A46127D04239A43AF
:107BA000244B1A751A46127D02239A43214B1A75EB
:107BB0005FE1204A127D08231A431E4B1A751A46AC
:107BC000D27C04231A431B4BDA741A46D27C02235C
:107BD0009A43184BDA741A46127D01231A43154B47
:107BE0001A751A46527D02231A43124B5A751A46C9
:107BF000127D04239A430F4B1A751A46127D0223F5
:107C00001A430C4B1A7534E10A4A127D08231A43B1
:107C1000084B1A751A46D27C04231A43054BDA74B2
:107C20001A46D27C02231A43024BDA741A46127D9A
:107C3000012301E07A1C00201A43FD4B1A751A46F5
:107C4000527D02239A43FA4B5A751A46127D042339
:107C50009A43F74B1A751A46127D02231A43F44BC6
:107C60001A7506E1F24A127D08239A43F04B1A7501
:107C70001A46D27C04231A43ED4BDA741A46D27C9E
:107C800002231A43EA4BDA741A46127D5208520054
:107C90001A751A46527D02239A43E54B5A751A46C5
:107CA000127D04231A43E24B1A751A46127D0223F1
:107CB0001A43DF4B1A75DCE0DD4A127D08231A43B4
:107CC000DB4B1A751A46D27C04239A43D84BDA74DC
:107CD0001A46D27C02231A43D54BDA741A46127D17
:107CE00001231A43D24B1A751A46527D022304E02F
:107CF000BEE092E066E03BE00FE09A43CC4B5A7561
:107D00001A46127D04231A43C94B1A751A46127D6E
:107D100002231A43C64B1A75ABE0C54A127D0823ED
:107D20001A43C34B1A751A46D27C04239A43C04B9C
:107D3000DA741A46D27C02231A43BD4BDA741A460F
:107D4000127D01231A43BA4B1A751A46527D02233B
:107D50001A43B74B5A751A46127D04231A43B44B83
:107D60001A751A46127D02231A43B14B1A7580E028
:107D7000AF4A127D08231A43AD4B1A751A46D27CBE
:107D800004231A43AA4BDA741A46D27C02231A43FC
:107D9000A74BDA741A46127D520852001A751A4619
:107DA000527D02239A43A24B5A751A46127D042330
:107DB0009A439F4B1A751A46127D02239A439C4B95
:107DC0001A7556E09A4A127D08231A43984B1A7581
:107DD0001A46D27C04231A43954BDA741A46D27C95
:107DE00002231A43924BDA741A46127D01231A4376
:107DF0008F4B1A751A46527D02231A438C4B5A75C3
:107E00001A46127D04231A43894B1A751A46127DAD
:107E100002231A43864B1A752BE0854A127D0823EC
:107E20001A43834B1A751A46D27C04231A43804B9B
:107E3000DA741A46D27C02231A437D4BDA741A464E
:107E4000127D01231A437A4B1A751A46527D02237A
:107E50009A43774B5A751A46127D04231A43744B82
:107E60001A751A46127D02231A43714B1A7500E0E7
:107E700000BF00BF7EE40B0007F0B3F80A06315BD9
:107E800085B0DCFEFDFCFBFA694A927C08231A43AC
:107E9000674B9A741A46527C04231A43644B5A74F3
:107EA0001A46527C01231A43614B5A741A46927C3B
:107EB00001231A435E4B9A741A46927C02231A439A
:107EC0005B4B9A741A46927C04231A43584B9A745B
:107ED0001A46527C02239A43554B5A7487E1544AFE
:107EE000927C08239A43524B9A741A46527C04237C
:107EF0001A434F4B5A741A46527C01231A434C4B77
:107F00005A741A46927C520852009A741A46927C0D
:107F100002239A43464B9A741A46927C04239A434E
:107F2000434B9A741A46527C02239A43404B5A742C
:107F30005DE13F4A927C08231A433D4B9A741A46EE
:107F4000527C04231A433A4B5A741A46527C520804
:107F500052005A741A46927C01231A43344B9A7485
:107F60001A46927C02231A43314B9A741A46927C29
:107F700004239A432E4B9A741A46527C02231A43C6
:107F80002B4B5A7433E12A4A927C08231A43284B1C
:107F90009A741A46527C04231A43254B5A741A4683
:107FA000527C01231A43224B5A741A46927C0123B5
:107FB0001A431F4B9A741A46927C02239A431C4B15
:107FC0009A741A46927C04239A43194B9A741A465F
:107FD000527C02231A43164B5A7408E1144A927CCD
:107FE00008239A43124B9A741A46527C04231A436C
:107FF0000F4B5A741A46527C01231A430C4B5A7485
:108000001A46927C520852009A741A46927C0223B5
:108010009A43074B9A741A46927C04231A43044BE2
:108020009A741A46527C02231A43014B5A74DEE0BA
:108030007A1C0020FE4A927C08231A43FC4B9A7457
:108040001A46527C04239A43F94B5A741A46527CBE
:1080500001231A43F64B5A741A46927C01231A43A1
:10806000F34B9A741A46927C02239A43F04B04E035
:10807000BCE090E064E039E00DE09A741A46927C2E
:1080800004231A43EA4B9A741A46527C02231A4379
:10809000E74B5A74ABE0E64A927C08231A43E44B60
:1080A0009A741A46527C04239A43E14B5A741A4636
:1080B000527C01231A43DE4B5A741A46927C0123E8
:1080C0001A43DB4B9A741A46927C02231A43D84B0C
:1080D0009A741A46927C04231A43D54B9A741A4612
:1080E000527C02231A43D24B5A7480E0D04A927CCD
:1080F00008231A43CE4B9A741A46527C04231A431F
:10810000CB4B5A741A46527C01231A43C84B5A74FB
:108110001A46927C520852009A741A46927C0223A4
:108120009A43C34B9A741A46927C04239A43C04BD9
:108130009A741A46527C02239A43BD4B5A7456E0F5
:10814000BB4A927C08231A43B94B9A741A46527C54
:1081500004231A43B64B5A741A46527C01231A431D
:10816000B34B5A741A46927C01231A43B04B9A744B
:108170001A46927C02231A43AD4B9A741A46927C9B
:1081800004231A43AA4B9A741A46527C02231A43B8
:10819000A74B5A742BE0A64A927C08231A43A44B9F
:1081A0009A741A46527C04231A43A14B5A741A46F5
:1081B000527C01231A439E4B5A741A46927C012327
:1081C0001A439B4B9A741A46927C02239A43984B0B
:1081D0009A741A46927C04231A43954B9A741A4651
:1081E000527C02231A43924B5A7400E000BF00BF36
:1081F00080E40B0006F0F5FE0A06356493C2F7F53D
:10820000F4F3F2F18A4AD27F10231A43884BDA77CB
:108210001A46D27F20231A43854BDA771A46D27F3B
:1082200040231A43824BDA771A46D27F80231A43BF
:108230007F4BDA771A462032127880231A437C4B20
:1082400020331A701A46127820231A43784B2033B1
:108250001A701A46127840239A43754B20331A70CD
:10826000B2E1734AD27F10239A43714BDA771A46F0
:10827000D27F20231A436E4BDA771A46D27F4023EF
:108280001A436B4BDA771A46D27F80239A43684BA6
:10829000DA771A462032127880239A43644B2033CF
:1082A0001A701A46127820239A43614B20331A70B1
:1082B0001A46127840239A435D4B20331A7083E1AB
:1082C0005B4AD27F10231A43594BDA771A46D27F82
:1082D00020231A43564BDA771A46D27F40239A431B
:1082E000534BDA771A46D27F80231A43504BDA7702
:1082F0001A462032127880231A434D4B20331A70CD
:108300001A46127820239A43494B20331A701A4692
:10831000127840231A43464B20331A7054E1444AE2
:10832000D27F10231A43424BDA771A46D27F20239A
:108330001A433F4BDA771A46D27F40231A433C4B0D
:10834000DA771A46D27F80231A43394BDA771A46F6
:108350002032127880239A43354B20331A701A4604
:10836000127820239A43324B20331A701A4612781F
:1083700040231A432E4B20331A7025E12C4AD27F1A
:1083800010239A432A4BDA771A46D27F20231A43C6
:10839000274BDA771A46D27F40231A43244BDA77E9
:1083A0001A46D27F80239A43214BDA771A4620322D
:1083B000127880239A431E4B20331A701A46127883
:1083C00020231A431A4B20331A701A46127840237E
:1083D0001A43174B20331A70F6E0F4E0C3E092E042
:1083E00061E030E0FFE7124AD27F10231A43104BBE
:1083F000DA771A46D27F20239A430D4BDA771A4652
:10840000D27F40231A430A4BDA771A46D27F802361
:108410001A43074BDA771A462032127880239A43A0
:10842000034B20331A701A46127820231A4301E0B6
:108430007A1C0020FE4B1A701A46127840231A4309
:10844000FB4B1A70C0E0FA4A203AD27F10231A433D
:10845000F74B203BDA771A46D27F20239A43F44B1E
:10846000203BDA771A46D27F40231A43F04B203B59
:10847000DA771A46D27F80231A43ED4B203BDA7716
:10848000EB4A127880231A43E94B1A701A46127885
:1084900020231A43E64B1A701A46127840231A43D7
:1084A000E34B1A7090E0E24A203AD27F10231A433D
:1084B000DF4B203BDA771A46D27F20231A43DC4B6E
:1084C000203BDA771A46D27F40231A43D84B203B11
:1084D000DA771A46D27F80239A43D54B203BDA774E
:1084E000D34A127880239A43D14B1A701A461278D5
:1084F00020239A43CE4B1A701A46127840239A438F
:10850000CB4B1A7060E0CA4A203AD27F10231A433C
:10851000C74B203BDA771A46D27F20231A43C44B3D
:10852000203BDA771A46D27F40231A43C04B203BC8
:10853000DA771A46D27F80231A43BD4B203BDA7785
:10854000BB4A127880231A43B94B1A701A46127824
:1085500020231A43B64B1A701A46127840231A4346
:10856000B34B1A7030E0B24A203AD27F10231A433C
:10857000AF4B203BDA771A46D27F20231A43AC4B0D
:10858000203BDA771A46D27F40231A43A84B203B80
:10859000DA771A46D27F80231A43A54B203BDA773D
:1085A000A34A127880239A43A14B1A701A46127874
:1085B00020231A439E4B1A701A46127840231A43FE
:1085C0009B4B1A7000E000BF00BF53E40B0006F0A5
:1085D00008FD0A06396C9FD2FEFDFCFBFAF9944AAD
:1085E000203A527F10231A43914B203B5A771A4668
:1085F000127F10231A438E4B203B1A771A46527F64
:1086000040231A438A4B203B5A771A46527F8023D5
:108610001A43874B203B5A771A46927F40231A43CE
:10862000834B203B9A771A46927F10231A43804B44
:10863000203B9A771A46527F20239A437C4B203B5B
:108640005A77B3E17A4A203A527F10239A43784B03
:10865000203B5A771A46127F10231A43744B203B53
:108660001A771A46527F40231A43714B203B5A77A0
:108670001A46527F80239A436D4B203B5A771A4605
:10868000927F40239A436A4B203B9A771A46927F07
:1086900010239A43664B203B9A771A46527F202339
:1086A0009A43634B203B5A7780E1614A203A527FDC
:1086B00010231A435E4B203B5A771A46127F102331
:1086C0001A435B4B203B1A771A46527F40239A434A
:1086D000574B203B5A771A46527F80231A43544BFC
:1086E000203B5A771A46927F40231A43504B203B37
:1086F0009A771A46927F10239A434D4B203B9A77E4
:108700001A46527F20231A43494B203B5A774DE1AA
:10871000474A203A527F10231A43454B203B5A7751
:108720001A46127F10231A43414B203B1A771A46F0
:10873000527F40231A433E4B203B5A771A46527FC2
:1087400080231A433A4B203B5A771A46927F4023A4
:108750009A43374B203B9A771A46927F10239A43CD
:10876000334B203B9A771A46527F20231A43304BD3
:10877000203B5A771AE12E4A203A527F10239A431F
:108780002B4B203B5A771A46127F10231A43284B53
:10879000203B1A771A46527F40231A43244B203B32
:1087A0005A771A46527F80239A43214B203B5A77AF
:1087B0001A46927F40239A431D4B203B9A771A46D4
:1087C000927F05E0F1E0C5E099E06DE041E00CE06A
:1087D00010231A43164B203B9A771A46527F2023C8
:1087E0001A43134B203B5A77E0E0114A203A527F5C
:1087F00010231A430E4B203B5A771A46127F102340
:108800009A430B4B203B1A771A46527F40231A4358
:10881000074B203B5A771A46527F80231A43044B5A
:10882000203B5A771A46927F40239A43004B01E03F
:108830009A1C0020203B9A771A46927F10231A43F5
:10884000F94B9A771A46527F20231A43F64B5A77F0
:10885000ACE0F54A527F10231A43F34B5A771A467D
:10886000127F10239A43F04B1A771A46527F402307
:108870001A43ED4B5A771A46527F80231A43EA4B2C
:108880005A771A46927F40231A43E74B9A771A4643
:10889000927F10231A43E44B9A771A46527F202383
:1088A0001A43E14B5A7781E0DF4A527F10231A4383
:1088B000DD4B5A771A46127F10231A43DA4B1A7788
:1088C0001A46527F40231A43D74B5A771A46527F93
:1088D00080239A43D44B5A771A46927F40239A4377
:1088E000D14B9A771A46927F10239A43CE4B9A77B0
:1088F0001A46527F20239A43CB4B5A7756E0CA4AF6
:10890000527F10231A43C84B5A771A46127F1023FE
:108910001A43C54B1A771A46527F40231A43C24B5B
:108920005A771A46527F80231A43BF4B5A771A460A
:10893000927F40231A43BC4B9A771A46927F1023AA
:108940001A43B94B9A771A46527F20231A43B64BE3
:108950005A772BE0B44A527F10231A43B24B5A770E
:108960001A46127F10231A43AF4B1A771A46527FCA
:1089700040231A43AC4B5A771A46527F80231A433E
:10898000A94B5A771A46927F40239A43A64B9A776F
:108990001A46927F10231A43A34B9A771A46527FA6
:1089A00020231A43A04B5A7700E000BF00BF1FE40A
:1089B0000B0006F016FB0A06315C87B2DDFDFCFBFE
:1089C000FAF9994AD27E10231A43974BDA761A465F
:1089D000927E20231A43944B9A761A46927E402325
:1089E0001A43914B9A761A46D27E80231A438E4BB5
:1089F000DA761A46127F40231A438B4B1A771A46AF
:108A0000D27E20231A43884BDA761A46D27E402340
:108A10009A43854BDA768BE1834AD27E10239A43C0
:108A2000814BDA761A46927E20231A437E4B9A7641
:108A30001A46927E40231A437B4B9A761A46D27E80
:108A400080239A43784BDA761A46127F40239A4362
:108A5000754B1A771A46D27E20239A43724BDA76E8
:108A60001A46D27E40239A436F4BDA7660E16E4A13
:108A7000D27E10231A436C4BDA761A46927E20235C
:108A80001A43694B9A761A46927E40239A43664B64
:108A90009A761A46D27E80231A43634BDA761A46B8
:108AA000127F40231A43604B1A771A46D27E202346
:108AB0009A435D4BDA761A46D27E40231A435A4BCC
:108AC000DA7635E1584AD27E10231A43564BDA76CD
:108AD0001A46927E20231A43534B9A761A46927E68
:108AE00040231A43504B9A761A46D27E80231A436B
:108AF0004D4BDA761A46127F40239A434A4B1A7737
:108B00001A46D27E20239A43474BDA761A46D27E03
:108B100040231A43444BDA760AE1434AD27E1023BB
:108B20009A43414BDA761A46927E20231A433E4BF3
:108B30009A761A46927E40231A433B4B9A761A46FF
:108B4000D27E80239A43384BDA761A46127F40232E
:108B50009A43354B1A771A46D27E20231A43324B5A
:108B6000DA761A46D27E40231A432F4BDA76DFE0BC
:108B70002D4AD27E10231A432B4BDA761A46927E68
:108B800020239A43284B9A761A46927E40231A4312
:108B9000254B9A761A46D27E80231A43224BDA76E8
:108BA0001A46127F402304E0C1E095E069E03DE011
:108BB0000FE09A431C4B1A771A46D27E20231A43A1
:108BC000194BDA761A46D27E40231A43164BDA76D0
:108BD000AEE0154AD27E10231A43134BDA761A46BA
:108BE000927E20239A43104B9A761A46927E402317
:108BF0001A430D4B9A761A46D27E80231A430A4BAB
:108C0000DA761A46127F40231A43074B1A771A4620
:108C1000D27E20231A43044BDA761A46D27E4023B2
:108C20001A43014BDA7683E07A1C0020FE4AD27E9A
:108C300010231A43FC4BDA761A46927E20231A43FD
:108C4000F94B9A761A46927E40231A43F64B9A764F
:108C50001A46D27E80239A43F34BDA761A46127F65
:108C600040239A43F04B1A771A46D27E20239A4328
:108C7000ED4BDA761A46D27E40239A43EA4BDA76F7
:108C800056E0E94AD27E10231A43E74BDA761A46B9
:108C9000927E20231A43E44B9A761A46927E402312
:108CA0001A43E14B9A761A46D27E80231A43DE4B52
:108CB000DA761A46127F40231A43DB4B1A771A469C
:108CC000D27E20231A43D84BDA761A46D27E40232E
:108CD0001A43D54BDA762BE0D34AD27E10231A43BF
:108CE000D14BDA761A46927E20231A43CE4B9A76DF
:108CF0001A46927E40231A43CB4B9A761A46D27E6E
:108D000080231A43C84BDA761A46127F40239A43CF
:108D1000C54B1A771A46D27E20231A43C24BDA7605
:108D20001A46D27E40231A43BF4BDA7600E000BFDA
:108D300000BF4AE40B0006F054F90A06315C87B222
:108D4000DDFDFCFBFAF9B84A527E10231A43B64BFC
:108D50005A761A46127E20231A43B34B1A761A46C5
:108D6000127E80231A43B04B1A761A46527E802315
:108D70001A43AD4B5A761A46527E40231A43AA4BE9
:108D80005A761A46527E20231A43A74B5A761A4621
:108D9000127E40239A43A44B1A768CE1A24A527E5B
:108DA00010239A43A04B5A761A46127E20231A4368
:108DB0009D4B1A761A46127E80231A439A4B1A76D6
:108DC0001A46527E80239A43974B5A761A46527E11
:108DD00040239A43944B5A761A46527E20239A4354
:108DE000914B5A761A46127E40239A438E4B1A763E
:108DF00061E18D4A527E10231A438B4B5A761A46F4
:108E0000127E20231A43884B1A761A46127E80233C
:108E10009A43854B1A761A46527E80231A43824B18
:108E20005A761A46527E40231A437F4B5A761A4688
:108E3000527E20239A437C4B5A761A46127E402358
:108E40001A43794B1A7636E1774A527E10231A4339
:108E5000754B5A761A46127E20231A43724B1A76A5
:108E60001A46127E80231A436F4B1A761A46527E98
:108E700080231A436C4B5A761A46527E40239A43FB
:108E8000694B5A761A46527E20239A43664B5A768D
:108E90001A46127E40231A43634B1A760BE1624A4C
:108EA000527E10239A43604B5A761A46127E202334
:108EB0001A435D4B1A761A46127E80231A435A4B88
:108EC0001A761A46527E80239A43574B5A761A4690
:108ED000527E40239A43544B5A761A46527E2023A0
:108EE0001A43514B5A761A46127E40231A434E4B70
:108EF0001A76E0E04C4A527E10231A434A4B5A76C7
:108F00001A46127E20239A43474B1A761A46127E3F
:108F100080231A43444B1A761A46527E80231A4302
:108F2000414B5A761A46527E402304E0C2E096E056
:108F300067E03BE00FE09A433B4B5A761A46527E7D
:108F400020231A43384B5A761A46127E40231A437E
:108F5000354B1A76AFE0344A527E10231A43324B17
:108F60005A761A46127E20239A432F4B1A761A46B7
:108F7000127E80231A432C4B1A761A46527E802387
:108F80001A43294B5A761A46527E40231A43264BDF
:108F90005A761A46527E20231A43234B5A761A4693
:108FA000127E40231A43204B1A7684E01E4A527EDA
:108FB00010231A431C4B5A761A46127E20231A435A
:108FC000194B1A761A46127E80231A43164B1A76CC
:108FD0001A46527E80239A43134B5A761A46527E83
:108FE00040239A43104B5A761A46527E20239A43C6
:108FF0000D4B5A761A46127E40239A430A4B1A7634
:1090000059E0094A527E10231A43074B5A761A46F2
:10901000127E20231A43044B1A761A46127E8023AE
:109020001A43014B1A7601E07A1C00201A46527E40
:1090300080231A43FE4B5A761A46527E40231A4327
:10904000FB4B5A761A46527E20231A43F84B5A7627
:109050001A46127E40231A43F54B1A762BE0F44A47
:10906000527E10231A43F24B5A761A46127E202360
:109070001A43EF4B1A761A46127E80231A43EC4BA2
:109080001A761A46527E80231A43E94B5A761A46BC
:10909000527E40239A43E64B5A761A46527E20234C
:1090A0001A43E34B5A761A46127E40231A43E04B8A
:1090B0001A7600E000BF00BF79E40B0005F091FFD5
:1090C0000A06315C87B2DDFEFDFCFBFAD84A927DD0
:1090D00010231A43D64B9A751A46927D20231A43C1
:1090E000D34B9A751A46927D40231A43D04B9A75FA
:1090F0001A46927D80231A43CD4B9A751A46D27D2B
:1091000040231A43CA4BDA751A46D27D10231A43FC
:10911000C74BDA751A46D27D20239A43C44BDA75C1
:109120008CE1C34A927D10239A43C14B9A751A462B
:10913000927D20231A43BE4B9A751A46927D402396
:109140001A43BB4B9A751A46927D80239A43B84BBB
:109150009A751A46D27D40239A43B54BDA751A4662
:10916000D27D10239A43B24BDA751A46D27D202362
:109170009A43AF4BDA7561E1AD4A927D10231A43F1
:10918000AB4B9A751A46927D20231A43A84B9A75C9
:109190001A46927D40239A43A54B9A751A46927DB2
:1091A00080231A43A24B9A751A46D27D40231A4354
:1091B0009F4BDA751A46D27D10239A439C4BDA7581
:1091C0001A46D27D20231A43994BDA7536E1984A24
:1091D000927D10231A43964B9A751A46927D20234E
:1091E0001A43934B9A751A46927D40231A43904B2B
:1091F0009A751A46927D80231A438D4B9A751A46AA
:10920000D27D40239A438A4BDA751A46D27D1023C9
:109210009A43874BDA751A46D27D20231A43844B32
:10922000DA750BE1824A927D10239A43804B9A753E
:109230001A46927D20231A437D4B9A751A46927DD9
:1092400040231A437A4B9A751A46927D80239A439B
:10925000774B9A751A46D27D40239A43744BDA7540
:109260001A46D27D10231A43714BDA751A46D27D05
:1092700020231A436E4BDA75E0E06D4A927D10238D
:109280001A436B4B9A751A46927D20239A43684B7A
:109290009A751A46927D40231A43654B9A751A4671
:1092A000927D80231A43624B9A751A46D27D4023E1
:1092B0009A4304E0C1E092E066E03AE00EE05C4BE5
:1092C000DA751A46D27D10231A43594BDA751A46BD
:1092D000D27D20231A43564BDA75AFE0544A927D73
:1092E00010231A43524B9A751A46927D20239A43B3
:1092F0004F4B9A751A46927D40231A434C4B9A75F0
:109300001A46927D80231A43494B9A751A46D27D9C
:1093100040231A43464BDA751A46D27D10231A436E
:10932000434BDA751A46D27D20231A43404BDA7537
:1093300084E03F4A927D10231A433D4B9A751A46AA
:10934000927D20231A433A4B9A751A46927D402308
:109350001A43374B9A751A46927D80239A43344BB1
:109360009A751A46D27D40239A43314BDA751A46D4
:10937000D27D10239A432E4BDA751A46D27D2023D4
:109380009A432B4BDA7559E0294A927D10231A43F0
:10939000274B9A751A46927D20231A43244B9A75BF
:1093A0001A46927D40231A43214B9A751A46927DA4
:1093B00080231A431E4B9A751A46D27D40231A43C6
:1093C0001B4BDA751A46D27D10231A43184BDA75F7
:1093D0001A46D27D20231A43154BDA752EE0144A23
:1093E000927D10231A43124B9A751A46927D2023C0
:1093F0001A430F4B9A751A46927D40231A430C4B21
:109400009A751A46927D80231A43094B9A751A461B
:10941000D27D40239A43064BDA751A46D27D10233B
:109420001A43034BDA751A46D27D20231A4301E012
:109430007A1C0020FC4BDA7500E000BF00BF81E31E
:109440000B0005F0CEFD0A06315C87B2DDFDFCFBAA
:10945000FAF9F54A127D10231A43F34B1A751A468E
:10946000D27C10231A43F04BDA741A46127D402343
:109470001A43ED4B1A751A46127D80231A43EA4BA4
:109480001A751A46527D40231A43E74B5A751A46FD
:10949000527D10231A43E44B5A751A46127D20233D
:1094A0009A43E14B1A7589E1DF4A127D10239A43F2
:1094B000DD4B1A751A46D27C10231A43DA4BDA7444
:1094C0001A46127D40231A43D74B1A751A46127D4D
:1094D00080239A43D44B1A751A46527D40239A43EF
:1094E000D14B5A751A46527D10239A43CE4B5A756A
:1094F0001A46127D20239A43CB4B1A755EE1CA4A65
:10950000127D10231A43C84B1A751A46D27C1023B9
:109510001A43C54BDA741A46127D40239A43C24B54
:109520001A751A46127D80231A43BF4B1A751A46C4
:10953000527D40231A43BC4B5A751A46527D102364
:109540009A43B94B5A751A46127D20231A43B64BDB
:109550001A7533E1B44A127D10231A43B24B1A75BF
:109560001A46D27C10231A43AF4BDA741A46127D86
:1095700040231A43AC4B1A751A46127D80231A43B6
:10958000A94B1A751A46527D40239A43A64B5A7529
:109590001A46527D10239A43A34B5A751A46127DE0
:1095A00020231A43A04B1A7508E19F4A127D10230D
:1095B0009A439D4B1A751A46D27C10231A439A4B34
:1095C000DA741A46127D40231A43974B1A751A46CD
:1095D000127D80239A43944B1A751A46527D40237C
:1095E0009A43914B5A751A46527D10231A438E4B5B
:1095F0005A751A46127D20231A438B4B1A75DDE0EB
:10960000894A127D10231A43874B1A751A46D27C59
:1096100010239A43844BDA741A46127D40231A436E
:10962000814B1A751A46127D80231A437E4B1A7598
:109630001A46527D402304E0BFE093E067E03BE040
:109640000FE09A43784B5A751A46527D10231A43FD
:10965000754B5A751A46127D20231A43724B1A75A0
:10966000ACE0714A127D10231A436F4B1A751A46EB
:10967000D27C10239A436C4BDA741A46127D402335
:109680001A43694B1A751A46127D80231A43664B9A
:109690001A751A46527D40231A43634B5A751A466F
:1096A000527D10231A43604B5A751A46127D2023AF
:1096B0001A435D4B1A7581E05B4A127D10231A43F1
:1096C000594B1A751A46D27C10231A43564BDA743A
:1096D0001A46127D40231A43534B1A751A46127DBF
:1096E00080239A43504B1A751A46527D40239A4361
:1096F0004D4B5A751A46527D10239A434A4B5A7560
:109700001A46127D20239A43474B1A7556E0464A63
:10971000127D10231A43444B1A751A46D27C10232B
:109720001A43414BDA741A46127D40231A433E4BCA
:109730001A751A46127D80231A433B4B1A751A4636
:10974000527D40231A43384B5A751A46527D1023D6
:109750001A43354B5A751A46127D20231A43324B51
:109760001A752BE0304A127D10231A432E4B1A75BE
:109770001A46D27C10231A432B4BDA741A46127DF8
:1097800040231A43284B1A751A46127D80231A4328
:10979000254B1A751A46527D40239A43224B5A751F
:1097A0001A46527D10231A431F4B5A751A46127DD2
:1097B00020231A431C4B1A7500E000BF00BFC1E113
:1097C0000B0005F00EFC0A06335E89B4DFFDFCFBDE
:1097D000FAF9154A927C10231A43134B9A741A46CD
:1097E000527C20231A43104B5A741A46527C802311
:1097F0001A430D4B5A741A46927C80231A430A4B23
:109800009A741A46D27C40231A43074BDA741A46DC
:10981000927C20231A43044B9A741A46927C40236C
:109820009A43014B9A748BE17A1C0020C64A927CC1
:1098300010239A43C44B9A741A46527C20231A432D
:10984000C14B5A741A46527C80231A43BE4B5A7439
:109850001A46927C80239A43BB4B9A741A46D27C58
:1098600040239A43B84BDA741A46927C20239A43D9
:10987000B54B9A741A46927C40239A43B24B9A7421
:109880005EE1B14A927C10231A43AF4B9A741A4698
:10989000527C20231A43AC4B5A741A46527C8023C4
:1098A0009A43A94B5A741A46927C80231A43A64BBA
:1098B0009A741A46D27C40231A43A34BDA741A4690
:1098C000927C20239A43A04B9A741A46927C4023A0
:1098D0001A439D4B9A7433E19B4A927C10231A439E
:1098E000994B9A741A46527C20231A43964B5A7409
:1098F0001A46527C80231A43934B5A741A46927C20
:1099000080231A43904B9A741A46D27C40239A4380
:109910008D4BDA741A46927C20239A438A4B9A74B0
:109920001A46927C40231A43874B9A7408E1864A70
:10993000927C10239A43844B9A741A46527C2023BB
:109940001A43814B5A741A46527C80231A437E4B29
:109950005A741A46927C80239A437B4B9A741A4617
:10996000D27C40239A43784BDA741A46927C2023A7
:109970001A43754B9A741A46927C40231A43724BD1
:109980009A74DDE0704A927C10231A436E4B9A74ED
:109990001A46527C20239A436B4B5A741A46527CC7
:1099A00080231A43684B5A741A46927C80231A43C8
:1099B000654B9A741A4604E0C1E095E069E03DE029
:1099C00011E0D27C40239A435F4BDA741A46927CB2
:1099D00020231A435C4B9A741A46927C40231A4304
:1099E000594B9A74ACE0584A927C10231A43564B58
:1099F0009A741A46527C20239A43534B5A741A463F
:109A0000527C80231A43504B5A741A46927C80230E
:109A10001A434D4B9A741A46D27C40231A434A4B40
:109A2000DA741A46927C20231A43474B9A741A46DA
:109A3000927C40231A43444B9A7481E0424A927CC0
:109A400010231A43404B9A741A46527C20231A431F
:109A50003D4B5A741A46527C80231A433A4B5A742F
:109A60001A46927C80239A43374B9A741A46D27CCA
:109A700040239A43344BDA741A46927C20239A434B
:109A8000314B9A741A46927C40239A432E4B9A7417
:109A900056E02D4A927C10231A432B4B9A741A4697
:109AA000527C20231A43284B5A741A46527C802336
:109AB0001A43254B5A741A46927C80231A43224B30
:109AC0009A741A46D27C40231A431F4BDA741A4602
:109AD000927C20231A431C4B9A741A46927C402392
:109AE0001A43194B9A742BE0174A927C10231A439D
:109AF000154B9A741A46527C20231A43124B5A74FF
:109B00001A46527C80231A430F4B5A741A46927C91
:109B100080231A430C4B9A741A46D27C40239A43F2
:109B2000094BDA741A46927C20231A43064B9A7426
:109B30001A46927C40231A43034B9A7400E000BFFC
:109B400000BF00BF00BF00BD7A1C002010B501217E
:109B50000648F7F77DFF00220121054801F010FAC1
:109B600001210348F9F79FFE10BD00000700000126
:109B7000400D004010B501220249842000F0A4FAF3
:109B800010BD00007806002010B58AB03948C079B1
:109B90004007C00F002805D13748807810210843BE
:109BA0003549887034482038C0791021084332493B
:109BB0002039C8710846007A082108432E49203907
:109BC000087209222D496846F6F716FB19222B491F
:109BD000103903A8F6F710FB03A80FC8FBF762FBC8
:109BE000274840788007C00F002807D02248203837
:109BF000407A01210843204920394872214BDA7804
:109C00001C46637A247A1B02234319461D4B98781D
:109C100000F056F81C4C237862781C4C21791C4CBF
:109C2000E07800F097F91B4841791B48007800F074
:109C3000E9F81A4A51790F4AD2791206900FFBF7C8
:109C4000A9FB0F480078C006C00F002805D00A48BD
:109C50008078042108430849887030220649203959
:109C6000002000F04AFA302103482038F6F7DDFAE8
:109C70000AB010BD0A0000209A1C0020EE0200204D
:109C8000C0080020F9120020181C0020071B00202B
:109C9000AA020020CC020020B8020020A21200205C
:109CA00010B5FFF753FF01210448F9F7FEFD01202D
:109CB00005F080FDFFF75EFF10BD0000400D004085
:109CC000F7B582B005460C462B0005F08AF906046C
:109CD00005121F3245524DE04848007820210843C4
:109CE00046490870084600788021084343490870B7
:109CF00040E0424800782021084340490870084667
:109D00000078102108433D49087033E03B48007853
:109D1000202108433949087039484079C007C00FED
:109D2000002805D10846007880210843334908708F
:109D300020E032480078202108433049087030483C
:109D40004079C007C00F002805D1084600781021CF
:109D500008432A4908700DE029484079C007C00F20
:109D6000002805D1254800782021084323490870A0
:109D700000E000BF00BF0498012805D11F4800780B
:109D8000402108431D4908700121C903204688432A
:109D90000446022D2FD1FF2C2DDCE117090F0919E4
:109DA00009110A2251432646E217120F9219121185
:109DB0001201A21A88180A21F6F7B2F9C0B20146B8
:109DC00001900120FBF718FBE117090F0919091190
:109DD0000A2251432646E217120F9219121112015C
:109DE000A21A88180A21F6F79BF9C8B20146019019
:109DF0000220FBF701FB05B0F0BD00007A1C00203B
:109E0000CC020020FEB504460D4600200290012041
:109E1000029049480668E807C00F002835D0002E98
:109E200033D046480078A8423AD0444805704448A8
:109E30000078A0420DD04248047060B241490870D9
:109E4000052C03DD601F4049087002E000203E49F8
:109E500008703C480078401E40B23A4908703A49C0
:109E60000978884203DA601E40B236490870002043
:109E700002E07668411CC8B2324900228A569042FC
:109E8000F7DB3088314908800AE0002E08D12C48E1
:109E90000078002804D000202C490880284804704D
:109EA0002A480088002845D028480088FF2841DC3F
:109EB0002748807A802108432549887223490988E8
:109EC0000191C9170A0F0199511809110A2251432A
:109ED0001E4A1788FA17120FD21912111201BA1A54
:109EE00088180A21F6F71CF9C0B200900299891C63
:109EF000C8B20099FBF780FA144909880191C91783
:109F00000A0F0199511809110A2251430F4A178863
:109F1000FA17120FD21912111201BA1A88180A214F
:109F2000F6F7FEF8C8B200900299C91CC8B20099B1
:109F3000FBF762FAFEBD0000B4020020810600209B
:109F4000820600208406002083060020860600206A
:109F50007A1C002030B51C461311042B05D1584B38
:109F60001B7A80252B43564D2B72012878D1544BF8
:109F7000DB7980252B43524DEB71524B1B785B1CD8
:109F8000504D2B702B461D782B0005F02AF80664E7
:109F9000040B182B44644A4B1B7A40252B43484D35
:109FA0002B725CE0464B1B7A40252B43444D2B72B1
:109FB0002B461B7A20252B43414D2B724FE0404B03
:109FC0001B7A40252B433E4D2B722B461B7A2025B6
:109FD0002B433B4D2B722B465B7A20252B43384D70
:109FE0006B723CE0364B1B7A40252B43344D2B7271
:109FF0002B461B7A20252B43314D2B722B465B7A47
:10A0000020252B432E4D6B722B465B7A40252B432C
:10A010002B4D6B7223E02A4B1B7A40252B43284D96
:10A020002B722B461B7A20252B43254D2B722B465A
:10A030005B7A20252B43224D6B722B465B7A4025A1
:10A040002B431F4D6B722B465B7A80252B431C4D97
:10A050006B7204E004E000231A4D2B7000BF2DE06A
:10A0600001292BD1164BDB7980252B43144DEB7145
:10A070002B461B7A40252B43114D2B72032C05DDFB
:10A080002B461B7A20252B430D4D2B720A2C05DD08
:10A090000B4B5B7A20252B43094D6B720F2C05DD92
:10A0A000074B5B7A40252B43054D6B72192C05DD60
:10A0B000034B5B7A80252B43014D6B7230BD000052
:10A0C0007A1C002088060020F8B507460D46164683
:10A0D0000024FAF709FB7C20FAF7D0FA3846FAF7A1
:10A0E000CDFA00BF04E0285DFAF7C8FA601CC4B2DC
:10A0F000B442F8DBFAF716FBF8BDF8B507460D4693
:10A1000016460024FAF7F0FA7C20FAF7B7FA802016
:10A11000FAF7B4FA3846FAF7B1FA00BF04E0285D5E
:10A12000FAF7ACFA601CC4B2B442F8DBFAF7FAFAF8
:10A13000F8BD0000FEB506460024002700250020DB
:10A14000019000BF0AE0705D412805D1681C305CB9
:10A15000412801D1741903E0681C85B2642DF2DB3B
:10A1600000BF002C40D00027002504E0605DC0192E
:10A17000C7B2681C85B2592DF8DB5920005DB84282
:10A1800032D104F0E3FBA07801282BD10190E078D4
:10A19000012806D0E078392803DAE07813490870FE
:10A1A00002E0002011490870002314220F491131E8
:10A1B000201D05F0AAF8207E0C49487000230F22CC
:10A1C000891C20461B3005F0A0F808482530F6F71A
:10A1D0004BF8002302220146009020462C3005F067
:10A1E00094F801E0002001900198FEBD181C0020A9
:10A1F00070B5044620460E30F6F736F8451C214669
:10A200000E312846F6F748F820460E30F6F72CF8BF
:10A21000E1210901884215D321460E310020F6F7CD
:10A220003BF820460A30F6F71FF80749884209D262
:10A2300020460A30F6F718F8451C21460A31284610
:10A24000F6F72AF870BD000030560100F3B58DB066
:10A250000C46A249C878F6F7C5FA0546A04AA14BB4
:10A26000F6F7BAF90B910A900D98F6F797FB09915A
:10A2700008900B9B0A9AF6F7A5FB02D201206072A8
:10A280005FE09649C878F6F7ADFA0546944A954BD3
:10A29000F6F7A2F9924A944B07910690F6F7E8F880
:10A2A0000B910A900D98F6F779FB099108900B9B9A
:10A2B0000A9AF6F787FB07D2607A012801D160720B
:10A2C0003FE0022060723CE084498878F6F78AFA21
:10A2D0000546834A834BF6F77FF90B910A900D9858
:10A2E000F6F75CFB099108900B9B0A9AF6F76AFB5C
:10A2F00002D20220607224E078498878F6F772FA78
:10A300000546774A774BF6F767F9754A764B07911A
:10A310000690F6F7ADF80B910A900D98F6F73EFB14
:10A32000099108900B9B0A9AF6F74CFB07D2607ACA
:10A33000022801D1607204E00020607201E0002078
:10A340006072607A012802D10020E074C3E0607A74
:10A35000022852D1614880786049C978884249DD35
:10A360005E4989785D4AD278881AF6F727FA054659
:10A370005B4A5C4BF6F730F90991089057498878A9
:10A38000F6F730FA0546564A564BF6F725F903918B
:10A3900002900D98F6F702FB01910090039B029A40
:10A3A000F6F70BF90022514B05910490F6F714F9DA
:10A3B00007910690099B089AF6F776F90B910A9097
:10A3C000F6F728FB07463846F6F7E8FA0546002276
:10A3D000464BF6F70BFB01D2454F05E0002138460E
:10A3E000F6F734FB00D200273846F6F71FFA40B2E2
:10A3F000E07470E00020E0746DE038498878F6F78A
:10A40000F1F9374A374B0B910A90F6F7E5F8054614
:10A4100003229207374BF6F7D5FA5AD22F4988789C
:10A42000F6F7E0F905462E4A2E4BF6F7D5F803224B
:10A430009207304B05910490F6F7C5F80991089002
:10A4400026498878F6F7CEF90546254A254BF6F7D2
:10A45000C3F8039102900D98F6F7A0FA01910090CD
:10A46000039B029AF6F7A9F80022234B059104906A
:10A47000F6F7B2F807910690099B089AF6F714F9D7
:10A480000B910A90F6F7C6FA07463846F6F786FAB1
:10A4900005460022184BF6F7A9FA01D2174F09E03A
:10A4A0003846F6F77BFA054600221346F6F78AFA95
:10A4B00000D200273846F6F771FA054600220B4B0A
:10A4C000F5F7D6FF0B910A90F6F7DEF940B2E0748B
:10A4D00001E01420E0740FB0F0BD0000A8030020DC
:10A4E0009A9999999999B93F9999C93F000034402F
:10A4F0000000A041CCCC1C40000054400000A04211
:10A5000010B501210848F7F7A3FA40210748F6F7EC
:10A5100096FF012240210548F9F7D1F900220821D0
:10A52000024800F02DFD10BD07000001400D004065
:10A5300010B5012400215E488170C170011D200505
:10A54000F5F7AAFE00215A480176417601461A31F4
:10A5500081204003F5F7A0FE002155482230017309
:10A56000417301460E3143208003F5F795FE00212B
:10A570004F48403001714171811D4E48F5F78CFE06
:10A5800000204D498870C870091D6005F5F784FEEC
:10A5900000214A488170C170011D4948F5F77CFED1
:10A5A000002146480176417601461A314548F5F7C3
:10A5B00073FE0021414822300173417301460E3180
:10A5C0004148F5F769FE002140488170C170011DC6
:10A5D0003F48F5F761FE00213C480176417601468F
:10A5E0001A313C48F5F758FE0021384822300173F3
:10A5F000417301460E313848F5F74EFE00213348CD
:10A60000403001714171811D3448F5F745FE00214C
:10A610002E4842300176417601461A313048F5F72E
:10A620003BFE00212948603001744174014612311B
:10A630002C48F5F731FE0021244882300171417128
:10A64000811D2948F5F728FE002120488030017738
:10A65000417701461E312548F5F71EFE5A23244A4C
:10A660002449134806F092F9002800D10024182349
:10A670001F4A6E321F496E310F4806F087F90028D5
:10A6800000D1002444231A4A9A321A499A310B48BD
:10A6900006F07CF9002800D10024B223164A17499D
:10A6A0000A4806F073F9002800D10024204610BDA6
:10A6B000DB04002000581400350500204D05002063
:10A6C0000078200000882000008A200091050020EA
:10A6D00000C820006ACC2000EECF200032D220003B
:10A6E00006DB2000DAE32000BEE6200062ED200059
:10A6F000984C0000981000000E4E00000E12000052
:10A7000010B501245A236B4A6B496C4805F094FD3F
:10A7100000282BD1002169488170C170011D2005DE
:10A72000F5F7BAFD00206549087648761A31812090
:10A730004003F5F7B1FD00216048223001734173F9
:10A7400001460E3143208003F5F7A6FD00215B484A
:10A75000403001714171811D5948F5F79DFD5A2323
:10A76000544A5549554806F011F900241823514A16
:10A770006E3251496E31534805F05EFD002810D10C
:10A7800050498870C870091D01204005F5F784FD07
:10A790001823484A6E3248496E314A4806F0F6F8A6
:10A7A00000244423434A9A3243499A31464805F0EB
:10A7B00043FD002823D1002143488170C170011D51
:10A7C0004248F5F769FD00213F4801764176014690
:10A7D0001A313F48F5F760FD00213B4822300173F4
:10A7E000417301460E313B48F5F756FD4423314A8B
:10A7F0009A3231499A31344806F0C8F80024B2231D
:10A80000354A3649364805F017FD00284FD13449FE
:10A810008870C870091D3348F5F73EFD00203049A7
:10A82000087648761A313048F5F736FD00212C4875
:10A8300022300173417301460E312C48F5F72CFD8F
:10A8400000212748403001714171811D2848F5F7EA
:10A8500023FD0021224842300176417601461A311B
:10A860002448F5F719FD00211D486030017441743A
:10A87000014612312048F5F70FFD002118488230BB
:10A8800001714171811D1D48F5F706FD0021144835
:10A8900080300177417701461E311948F5F7FCFCFD
:10A8A000B2230D4A0D490E4806F070F800242046E8
:10A8B00010BD0000984C000098100000DB04002040
:10A8C00000581400350500204D05002000782000B8
:10A8D00000882000008A20000E4E00000E120000AA
:10A8E0009105002000C820006ACC2000EECF200097
:10A8F00032D2200006DB2000DAE32000BEE6200092
:10A9000062ED20000FB410B53748C078062867D133
:10A9100035480079372863D13348407900285FD122
:10A9200008A8807900285BDD30484079012814D1DF
:10A9300000202F49087000BF2E4880784006C00FC5
:10A94000002809D02B488078402188432949887005
:10A9500097212948F6F7B2FB42E0254801780078B4
:10A96000401C234A107008A88079814238DB00BF60
:10A97000204880784006C00F002830D11F488078DA
:10A980004006C00F00282AD01A488078402188430A
:10A990004030184988701A488078402188434030F8
:10A9A000174988709721002006F0DAFB1548807857
:10A9B0004006C00F00280ED09720F6F73DFB012877
:10A9C00009D1114880784021884340300E49887071
:10A9D00001200E49087097210748F6F770FB00BF69
:10A9E00010BC08BC04B01847CC020020071B002094
:10A9F0004A060020C0080020B402002014000020F5
:10AA0000DA08002022000020CC08002008000020E6
:10AA100010B501210448F7F71BF800220421034870
:10AA2000F9F741FF10BD000007000001400C004095
:10AA300010B501210348F7F70BF804210248F7F796
:10AA4000BFF910BD07000001400C004010B505F033
:10AA50005BFE80210C48F8F71CFF012809D10B4848
:10AA6000007802280EDA09480078401C074908706F
:10AA700008E006480078002804D004480078401E0A
:10AA80000249087010BD0000800D0040FC0200204B
:10AA9000F8B5002488E0A000454909680F5CA000D3
:10AAA00043490968085CA100414A1268891849783D
:10AAB0004840A1003E4A1268891889784840A100A0
:10AAC0003B4A12688918C97805464D40A0003849AC
:10AAD0000968085CA100364A12688918497848401C
:10AAE0000646304607F0ACFA0646A0003049096831
:10AAF000085C314669404840A1002D4A1268505414
:10AB0000A0002B49096840184078A100284A126823
:10AB10008918897848400646304607F091FA06467B
:10AB2000A0002349096840184078314669404840F0
:10AB3000A1001F4A126889184870A0001C490968C2
:10AB400040188078A1001A4A12688918C9784840CC
:10AB50000646304607F074FA0646A0001449096814
:10AB600040188078314669404840A100104A126878
:10AB700089188870A0000E4909684018C07878408C
:10AB80000646304607F05CFA0646A0000849096808
:10AB90004018C078314669404840A100044A126814
:10ABA0008918C870601CC4B2042C00DA73E7F8BDC1
:10ABB0000000002010B50022FF210131044800F000
:10ABC000DFF9002201214902014800F0D9F910BD46
:10ABD000400C004010B5002240210448F9F763FE04
:10ABE000002280210148F9F75EFE10BD400C0040B4
:10ABF00010B540210348F7F7E3F880210148F7F743
:10AC0000DFF810BD400C004070470000002805DB55
:10AC1000C206D20E01219140014A11607047000026
:10AC200080E100E0002805DBC206D20E0121914040
:10AC3000014A11607047000080E100E0002805DB58
:10AC4000C206D20E01219140014A116070470000F6
:10AC500000E100E0002805DBC206D20E0121914090
:10AC6000014A11607047000000E100E010B50028C3
:10AC700019DB1A4A03231B02D21883089B00D258FF
:10AC80008307DC0EFF23A3409A438B071B0E840728
:10AC9000E40EA3401A43114B032424021B19840819
:10ACA000A4001A5118E00E4A03071B0F083B9B082B
:10ACB0009B00D2588307DC0EFF23A3409A438B07E7
:10ACC0001B0E8407E40EA3401A43054B0407240F10
:10ACD000083CA408A4001A5110BD000000E100E0E7
:10ACE0001CED00E010B5002819DB1A4A03231B02F3
:10ACF000D21883089B00D2588307DC0EFF23A340A1
:10AD00009A438B071B0E8407E40EA3401A43114B92
:10AD1000032424021B198408A4001A5118E00E4AC7
:10AD200003071B0F083B9B089B00D2588307DC0ED0
:10AD3000FF23A3409A438B071B0E8407E40EA34016
:10AD40001A43054B0407240F083CA408A4001A5119
:10AD500010BD000000E100E01CED00E010B500288F
:10AD600019DB1A4A03231B02D21883089B00D2580E
:10AD70008307DC0EFF23A3409A438B071B0E840737
:10AD8000E40EA3401A43114B032424021B19840828
:10AD9000A4001A5118E00E4A03071B0F083B9B083A
:10ADA0009B00D2588307DC0EFF23A3409A438B07F6
:10ADB0001B0E8407E40EA3401A43054B0407240F1F
:10ADC000083CA408A4001A5110BD000000E100E0F6
:10ADD0001CED00E010B505F087FCFF2101310448AF
:10ADE000F8F765FD03F0CAF8FFF730FE10BD00006C
:10ADF000C00C0040F8B506460C46174600BF0121BE
:10AE000089031648F8F74FFD40211448F8F74DFD27
:10AE100000BF032002F0F2FB2102080E02F0EEFB5D
:10AE20002104080E02F0EAFBE0B202F0E7FB002585
:10AE300005E0FF2002F0E2FB7055681C85B2BD42C0
:10AE4000F7DB00BF40210548F8F72FFD01218903FA
:10AE50000248F8F72AFD00BFF8BD0000800C004052
:10AE6000F7B5434B9D440F4615460121090368463B
:10AE7000F5F7DBF9781901218905884202D93D4BA4
:10AE80009D44F0BD390B3C48684441603805000DD5
:10AE9000394969440860086837490C1AA54200DC42
:10AEA0002C4656E03448684440680103324A6846FC
:10AEB000FFF7A0FF00260AE02F48684400688019C9
:10AEC0006946085CFF2800D003E0701C86B2A642E9
:10AED000F2DB00BFA6421DDA274868444068F7F756
:10AEE0005DFF00260BE0244868448068815D2248AD
:10AEF0006844006830186A461154701C86B2A64235
:10AF0000F1DB1D486844406801031B4A6846F7F7B7
:10AF1000A2FF06E022463946174868448068F7F7E2
:10AF20009AFFA54200D115E0134868444068411CCF
:10AF300011486844416000210160816809198160FD
:10AF40003F19281B85B20C48854201DD044600E00C
:10AF50002C46A7E700BF00BF40210848F8F7A5FC32
:10AF6000012189030548F8F7A0FC00BF00BF86E770
:10AF7000F8EFFFFF1410000000100000800C0040EC
:10AF80007FB506460D4614466A4629463046F8F710
:10AF90008FFA0098A84217D16846C079002813D1CB
:10AFA000002C03D16846407900280DD1012C03D133
:10AFB00068464079012807D168468079002803D186
:10AFC00068460079012813D0029500206946C873AD
:10AFD000002C01D1487302E001206946487300212A
:10AFE000684681730121017302A93046F8F718FC05
:10AFF0007FBD0000FEB5F9F7ADF90446D449F5F779
:10B000004BF9D449C878F5F7EDFB0646D24AD34B45
:10B01000F5F7E2FA01910090CD48F5F725F90646DB
:10B02000F5F7BCFC0446019B009AF5F7CBFC25D252
:10B0300000BFCB4800798007C00F00280AD1C8485C
:10B04000007902218843801CC54908711121C54837
:10B05000F6F735F800BF00BFC1480079C007C00F40
:10B0600000280AD1BE48007940084000401CBC4975
:10B0700008711021BB48F6F722F860E0B5498878DE
:10B08000F5F7B0FB0646B44AB44BF5F7A5FA04460B
:10B090000D46AF48F5F7E8F80646F5F77FFC22467F
:10B0A0002B4601910090F5F78DFC24D200BFAC48EF
:10B0B00000798007C00F002809D0A9480079022133
:10B0C0008843A74908711121A648F5F7F7FF00BF8B
:10B0D00000BFA3480079C007C00F00280AD1A048CC
:10B0E000007940084000401C9D49087110219D488E
:10B0F000F5F7E5FF23E000BF994800798007C00F0E
:10B10000002809D0964800790221884394490871A3
:10B1100011219448F5F7D2FF00BF00BF9048007995
:10B12000C007C00F002809D08D48007940084000B2
:10B130008B49087110218B48F5F7C0FF00BFF9F764
:10B1400061F804468249491DF5F7A6F88149487916
:10B15000F5F748FB0446804A804BF5F73DFA064672
:10B160000F467B48401DF5F77FF80446F5F716FCBF
:10B1700032463B4601910090F5F724FC25D200BFF2
:10B1800077480079C006C00F00280AD174480079BA
:10B190001021884310307249087114217148F5F765
:10B1A0008EFF00BF00BF6E4800790007C00F002867
:10B1B0000AD16B4800790821884308306849087132
:10B1C00013216848F5F77BFF61E062490879F5F7DC
:10B1D00009FB0446604A614BF5F7FEF906460F4647
:10B1E0005B48401DF5F740F80446F5F7D7FB3246BB
:10B1F0003B4601910090F5F7E5FB24D200BF58488B
:10B200000079C006C00F002809D0554800791021E8
:10B2100088435349087114215248F5F74FFF00BF86
:10B2200000BF4F4800790007C00F00280AD14C48E2
:10B230000079082188430830494908711321494899
:10B24000F5F73DFF23E000BF45480079C006C00F79
:10B25000002809D0424800791021884340490871EC
:10B2600014214048F5F72AFF00BF00BF3C48007991
:10B270000007C00F002809D0394800790821884309
:10B280003749087113213748F5F718FF00BFF7F762
:10B29000E9FB20213448F8F7FCFA002840D10A20C5
:10B2A00004F088FA20213048F8F7F3FA002820D17A
:10B2B00008212D484030F8F7F8FA00BF28484078B8
:10B2C0008007C00F00280AD1254840780221884312
:10B2D000801C2349487000212248F5F7F0FE00BF8A
:10B2E0000123002220212048F7F796FF06F01CFCDE
:10B2F0002DE008211C484030F8F7D5FA00BF184867
:10B3000040788007C00F002809D0154840780221F6
:10B3100088431349487000211248F5F7CFFE16E024
:10B32000082111484030F8F7BEFA00BF0C484078B9
:10B330008007C00F002809D00948407802218843BF
:10B340000749487000210748F5F7B8FE00BFFEBD69
:10B35000E3020020A80300209A9999999999B93F8E
:10B36000C0080020B4020020400D004010B50121AB
:10B370001E48F6F76DFB002208211D48FFF700FE6E
:10B38000002201211A488038F9F78DFA0022102195
:10B390001748FFF7F5FD00210120F9F7BFFA10214A
:10B3A0001348F8F780FA08211148F8F77CFA0022D0
:10B3B00004210F484030FFF7E3FD002208210C482C
:10B3C0004030FFF7DDFD042109484030F8F76BFA03
:10B3D000082107484030F8F766FA002201214903A6
:10B3E0000348C038F9F75FFA10BD000007000001FC
:10B3F000400D0040F7B582B006460F4600240025F8
:10B40000002001900BA13046F4F71AFF0446002CEF
:10B410000DD009A12046F4F713FF0546002D06D0F4
:10B4200039462846049A01F0CBFD05B0F0BD042052
:10B43000FBE700002B5200002C00000010B5F9487B
:10B44000C07B8021084080282ED1F9F703FFF64801
:10B4500040790007C00F00281FD0F9F7B3FE012183
:10B46000F248F8F722FA012004F0A4F901231A4661
:10B470002021EE488030F9F775F9012809D1EC4810
:10B480000078FA280BDAEA480078401CE84908708E
:10B4900005E00020E649087001E0F9F7A3FE01216C
:10B4A000E248F8F700FA51E0DE488078012803D03E
:10B4B000DC488078032841D1F9F7CCFEF9F782FE09
:10B4C0000121DA48F8F7F1F9D648C07BF0210840AD
:10B4D00000283BD1D3480179C27808021043D549EE
:10B4E000884227D0CF480179C27808021043D14959
:10B4F000491C88421ED0CB480179C278080210430B
:10B50000CD49884216D0002301222021C74880302F
:10B51000F9F728F9012809D1C5480078FA2815DA81
:10B52000C3480078401CC24908700FE00020C049A1
:10B5300008700BE00020BE49087007E0F9F78AFEAA
:10B54000F9F750FE0121B948F8F7ADF9B548C07BCD
:10B55000F021084020282BD1B34840790007C00FC4
:10B56000002825D002F0F6FC02F082FD0421AF484D
:10B57000F8F79BF9012004F01DF901231A46082170
:10B58000AA484030F9F7EEF8012809D1A848007818
:10B59000FA2808DAA6480078401CA549087002E09D
:10B5A0000020A34908700421A048F8F77CF932E094
:10B5B0009D480079C009002825D002F0CBFC02F09C
:10B5C00057FD04219948F8F770F9012004F0F2F8CA
:10B5D00000230122082195484030F9F7C3F80128DB
:10B5E00009D196480078FA2808DA94480078401C77
:10B5F0009249087002E000209049087004218B48AD
:10B60000F8F751F907E002F0A5FC02F041FD042132
:10B610008648F8F748F989480078032835DB00BFE9
:10B6200087480079C00900282ED17F480079C009D9
:10B63000002829D0824800798021884380308049C1
:10B640000871804800798021884380307D490871E5
:10B650008121002005F084FD7B480079C009002885
:10B660000ED08120F5F7E8FC012809D17748007950
:10B670008021884380307549087101207449087021
:10B6800081217448F5F71BFD00BF6648C07BF0219F
:10B69000084010282BD1644840790007C00F0028CB
:10B6A00025D0F9F7EBFDFFF7B3F902215F48F8F772
:10B6B000FCF8012004F07EF801231A4604215B48BF
:10B6C0004030F9F74FF8012809D159480078FA2895
:10B6D00008DA57480078401C5549087002E00020FD
:10B6E0005349087002215148F8F7DDF833E04E481D
:10B6F00000794006C00F002825D0F9F7BFFDFFF7FD
:10B7000087F902214948F8F7D0F8012004F052F8EF
:10B7100000230122042145484030F9F723F801288D
:10B7200009D14D480078FA2808DA4B480078401CC7
:10B730004949087002E000204749087004213B484D
:10B74000F8F7B1F807E0F9F799FDFFF771F9022171
:10B750003648F8F7A8F840480078032838DB00BFDF
:10B76000374800794006C00F002830D12E480079B4
:10B770004006C00F00282AD0314800794021884374
:10B7800040302F4908712F480079402188434030CC
:10B790002C4908718021002005F0E2FC2A4800793C
:10B7A0004006C00F00280ED08020F5F745FC012888
:10B7B00009D1264800794021884340302349087147
:10B7C00001202349087080212248F5F778FC00BF4A
:10B7D0001448C07BF0210840402847D112484079E6
:10B7E0000007C00F002841D0F6F7BAFAF6F704FBBD
:10B7F00008210E48F8F759F8012003F0DBFF012378
:10B800001A4659030948F8F7ADFF012826D1084820
:10B810000078FA2825DA06480078401C04490870A8
:10B820001FE000007203002014000020000C004004
:10B830009C06002001070000011300009E06002066
:10B84000C0080020DA08002022000020CC080020D8
:10B8500008000020B40200209D060020002061495D
:10B86000087008216048F8F71EF831E05F48407919
:10B87000C009002824D0F6F773FAF6F7BDFA0821BC
:10B880005948F8F712F8012003F094FF0023012231
:10B8900051035548F8F766FF012809D1544800784C
:10B8A000FA2808DA52480078401C5149087002E032
:10B8B00000204F49087008214B48F7F7F4FF07E0D4
:10B8C000F6F74EFAF6F7A8FA08214748F7F7EBFF24
:10B8D00047480078032835DB00BF46484079C00957
:10B8E00000282ED141484079C009002829D041487C
:10B8F00040798021884380303E4948713E484079F4
:10B900008021884380303C4948718721002005F020
:10B9100027FC3A484079C00900280ED08720F5F767
:10B920008BFB012809D1364840798021884380303B
:10B930003349487101203349087087213248F5F7AF
:10B94000BEFB00BF27480078032838DB00BF29482A
:10B9500040790007C00F002830D124484079000703
:10B96000C00F00282AD02348407908218843083096
:10B9700020494871204840790821884308301E49F1
:10B9800048718221002005F0EBFB1C48407900073C
:10B99000C00F00280ED08220F5F74EFB012809D1F8
:10B9A000174840790821884308301549487101201B
:10B9B0001449087082211448F5F781FB11E000BF9B
:10B9C0000C4840790007C00F002809D00948407989
:10B9D000082188430749487182210B48F5F76EFB1F
:10B9E00000BF10BD9C060020000C00401400002089
:10B9F0009F060020C0080020DA0800202200002056
:10BA0000CC08002008000020B402002010B5FC483B
:10BA1000C07B80210840802845D1F9F71BFCF948FC
:10BA200040790007C00F002836D0F9F7CBFB012181
:10BA3000F548F7F73AFF012003F0BCFE01231A4650
:10BA40002021F1488030F8F78DFE012812D100BF87
:10BA5000EE4840790007C00F00280AD1EB48407932
:10BA6000082188430830E94948718221E848F5F700
:10BA700026FB13E000BFE54840790007C00F00280F
:10BA800009D0E248407908218843E0494871822181
:10BA9000DF48F5F713FB01E0F9F7A4FB0121DA48D1
:10BAA000F7F701FF7DE0D6488078012803D0D4481D
:10BAB000807803286DD1F9F7CDFBF9F783FB0121DD
:10BAC000D148F7F7F2FECE48C07BF02108400028AD
:10BAD00059D1CB480179C27808021043CD49884238
:10BAE0003FD0C7480179C27808021043C949491CB0
:10BAF000884236D0C2480179C27808021043C6494C
:10BB000088422ED00023FF22F6322021BE4880300A
:10BB1000F8F728FE012812D100BFBC484079000781
:10BB2000C00F00280AD1B94840790821884308305D
:10BB3000B64948718221B648F5F7C1FA23E000BF43
:10BB4000B24840790007C00F002809D0AF484079BB
:10BB500008218843AD4948718221AD48F5F7AEFA16
:10BB600011E000BFA94840790007C00F002809D0A4
:10BB7000A648407908218843A44948718221A448F5
:10BB8000F5F79CFA00BFA54AF021A548F5F796FD08
:10BB900007E0F9F75FFBF9F725FB01219A48F7F772
:10BBA00082FE9748C07BF0210840202843D1954869
:10BBB00040790007C00F00283DD002F0CBF902F019
:10BBC00057FA04219048F7F770FE012003F0F2FDC8
:10BBD00001231A4608218C484030F8F7C3FD01289C
:10BBE00012D100BF894840790007C00F00280AD150
:10BBF0008648407908218843083084494871822169
:10BC00008348F5F75CFA11E000BF804840790007EF
:10BC1000C00F002809D07D484079082188437B491E
:10BC2000487182217A48F5F749FA00BF0421764825
:10BC3000F7F739FE33E073480079C009002826D0B1
:10BC400002F088F902F014FA04216F48F7F72DFE8C
:10BC5000012003F0AFFD0023012208216A48403093
:10BC6000F8F780FD012807D16848007980218843D2
:10BC700080306649087105E0644800798021884376
:10BC80006249087104216048F7F70DFE07E002F0F1
:10BC900061F902F0FDF904215B48F7F704FE58480A
:10BCA000C07BF0210840102843D156484079000756
:10BCB000C00F00283DD0F9F7E1FAFEF7A9FE0221F6
:10BCC0005148F7F7F2FD012003F074FD01231A46F5
:10BCD00004214D484030F8F745FD012812D100BF3E
:10BCE0004A4840790007C00F00280AD147484079E8
:10BCF0000821884308304549487182214448F5F7B6
:10BD0000DEF911E000BF414840790007C00F00286C
:10BD100009D03E484079082188433C494871822136
:10BD20003B48F5F7CBF900BF02213748F7F7BBFDD9
:10BD300034E0344800794006C00F002826D0F9F7D7
:10BD40009DFAFEF765FE02212F48F7F7AEFD0120B0
:10BD500003F030FD0023012204212B484030F8F786
:10BD600001FD012807D1294800794021884340304E
:10BD70002649087105E02548007940218843234978
:10BD8000087104212048F7F78EFD07E0F9F776FAED
:10BD9000FEF74EFE02211C48F7F785FD1848C07BD0
:10BDA000F0210840402854D1164840790007C00FC0
:10BDB00000284ED0F5F7D4FFF6F71EF808211248F8
:10BDC000F7F773FD012003F0F5FC01231A46590330
:10BDD0000D48F8F7C7FC012824D100BF0B48407973
:10BDE0000007C00F00280AD108484079082188437D
:10BDF00008300649487182210548F5F760F923E0CB
:10BE00007203002014000020000C0040C008002035
:10BE1000B40200200107000001130000DC0500004F
:10BE20000030014000BF0F4840790007C00F0028D4
:10BE300009D00C484079082188430A494871822179
:10BE40000948F5F73BF900BF08210848F7F72BFD33
:10BE500007E0F5F785FFF5F7DFFF08210348F7F75F
:10BE600022FD10BDC0080020B4020020000C0040DC
:10BE7000F7B586B004460F4600BF00BF0020385E0D
:10BE80007D21C900884209DC0020385E4942884291
:10BE900004DB64490898F4F7E3FD02D2002009B0FE
:10BEA000F0BD0020385EF4F777FC02900899F4F7B3
:10BEB00064FA0390F4F772FD05460E4600203880C0
:10BEC000214639310A461378194653781B02194323
:10BED00093781B041943D278120611430846F4F7ED
:10BEE00081FC514A514B01910090F4F775FB2A46B1
:10BEF000334603910290F4F76FFB059104900820FC
:10BF00002218002001461378184353781B02184367
:10BF100093781B041843D3781B06184313791943ED
:10BF200053791B02194393791B041943D2791206E2
:10BF300011432A46334603910290F4F799FA20728E
:10BF4000020A6272020CA272000EE0722173080AE9
:10BF50006073080CA073080EE073204638300D2182
:10BF60004218002108461378194353781B021943DD
:10BF700093781B041943D3781B061943137918438C
:10BF800053791B02184393791B041843D279120684
:10BF9000104302910390084603A90EC9F4F768FA0A
:10BFA000224638325073030A9373030CD373000E86
:10BFB00010745174080A9074080CD074080E10752F
:10BFC000521D002108461378194353781B02194368
:10BFD00093781B041943D3781B061943137918432C
:10BFE00053791B02184393791B041843D279120624
:10BFF000104302910390084603A90EC9F4F7DDFA35
:10C00000224638325071030A9371030CD371000E2B
:10C0100010725172080A9072080CD072080E1073D8
:10C0200001203CE700007A442D431CEBE2361A3F26
:10C0300010B5F9F70FF9F9F7D5F8F9F71FF9FEF789
:10C04000F7FC01F087FF02F023F8F5F789FEF5F71A
:10C05000E3FE10BDF7B596B004460F4604201490D9
:10C060000023082212A9A01D03F04FF90023082283
:10C0700010A920460E3003F048F9002304220FA92E
:10C080002046163003F041F9A07E0E904D480F99DE
:10C0900041700A0A82700A0CC270090E01712030C8
:10C0A0000E9941710246503A002001461378184318
:10C0B00053781B02184393781B041843D3781B064C
:10C0C00018431379194353791B02194393791B04BD
:10C0D0001943D2791206114300223B4B0B910A906F
:10C0E000F4F77AFA0D910C90F4F710FC05460E4621
:10C0F00013991298401BB14143DA0F98F4F772FB81
:10C10000079106903046139A1299691A904100914E
:10C11000019008460199F4F773FB2C4A2C4B0391CC
:10C120000290F4F759FA05910490079B069AF4F7E8
:10C1300053FA264A264B09910890F4F74DFA0D91CF
:10C140000C9011991098F4F75BFB224A224B09914D
:10C150000890F4F741FA0B910A900D9B0C9AF4F7B2
:10C160002CFA184A5071030A9371030CD371000E14
:10C1700010725172080A9072080CD072080E107377
:10C1800018E011991098F4F73BFB124A124B0D91ED
:10C190000C90F4F721FA0B4A5071030A9371030CC7
:10C1A000D371000E10725172080A9072080CD0728E
:10C1B000080E10730020387001211898018014981F
:10C1C00019B0F0BD821200200088C3402D431CEB43
:10C1D000E2361A3FFCA9F1D24D62503FF8B507464E
:10C1E0000D4616460024F8F77FFA6420F8F746FA61
:10C1F0003846F8F743FAF8F777FA6520F8F73EFA89
:10C2000000BF06E0F8F7FAF92855F8F7BBF9601C0B
:10C21000C4B2701EA042F5DCF8F7F0F92855F8F723
:10C22000D1F9F8F77FFAF8BDF8B507460D4616467E
:10C23000F8F75AFA6420F8F721FA3846F8F71EFAA8
:10C24000002404E0285DF8F719FA601CC4B2B44277
:10C25000F8DBF8F767FAF8BD0146064A506806238E
:10C2600002469A43104606220A401043014A506093
:10C270007047000000280040012806D1064949689F
:10C2800001221143044A516005E003494968490805
:10C290004900014A5160704700280040012806D13A
:10C2A0000649096801221143044A116005E0034967
:10C2B000096849084900014A116070470028004098
:10C2C00070B586B0044600BF00BF20463830372125
:10C2D0004218002001461378184353781B02184374
:10C2E00093781B041843D3781B061843137919431A
:10C2F00053791B02194393791B041943D27912060F
:10C30000114303910290082022180020014613785F
:10C31000184353781B02184393781B041843D378AF
:10C320001B0618431379194353791B021943937958
:10C330001B041943D2791206114301910090039B0B
:10C34000029AF4F73FFB02D2002006B070BD2046EF
:10C3500038303721421800210846137819435378A2
:10C360001B02194393781B041943D3781B06194306
:10C370001379184353791B02184393791B0418430C
:10C38000D27912061043029103900820221800204F
:10C3900001461378184353781B02184393781B0403
:10C3A0001843D3781B0618431379194353791B029A
:10C3B000194393791B041943D27912061143019151
:10C3C0000090039B029AF4F7F8F805460E462146C2
:10C3D00039310A461378194653781B02194393786A
:10C3E0001B041943D278120611430846F4F7FAF9F0
:10C3F000504A514B01910090F4F7EEF82A4633462B
:10C4000003910290F4F7E8F80591049008202218AF
:10C41000002108461378194353781B021943937877
:10C420001B041943D3781B06194313791843537916
:10C430001B02184393791B041843D2791206104348
:10C440002A4633460291039008460399F4F710F800
:10C450002072020A6272020CA272000EE072217354
:10C46000080A6073080CA073080EE0732046383089
:10C470000D214218002001461378184353781B02FF
:10C48000184393781B041843D3781B061843137979
:10C49000194353791B02194393791B041943D27929
:10C4A0001206114303910290059B049AF3F7E0FFF3
:10C4B000224638325073030A9373030CD373000E71
:10C4C00010745174080A9074080CD074080E10751A
:10C4D000521D002001461378184353781B0218435D
:10C4E00093781B041843D3781B0618431379194318
:10C4F00053791B02194393791B041943D27912060D
:10C50000114303910290059B049AF4F756F82246D2
:10C5100038325071030A9371030CD371000E1072FC
:10C520005172080A9072080CD072080E1073012024
:10C530000BE700002D431CEBE2361A3F10B500213B
:10C540000548F5F785FA02210448F5F739FC012181
:10C550000248F5F735FC10BD09000003400C00400F
:10C5600010B5002204212D48F8F79DF90022012181
:10C57000C9032B48FEF704FD002201218903284846
:10C58000FEF7FEFC00220121C90225484030FEF7DB
:10C59000F7FC00220121090321484030FEF7F0FC9E
:10C5A0000022012149031E484030FEF7E9FC002229
:10C5B000012189031A484030FEF7E2FC00220121E4
:10C5C000C90317484030FEF7DBFC0121C9031448BA
:10C5D000F7F769F9012189031148F7F764F9012197
:10C5E000C9020F484030F7F75EF9012109030C48F2
:10C5F0004030F7F758F90121490309484030F7F76F
:10C6000052F90121890306484030F7F74CF901211E
:10C61000C90303484030F7F746F910BD000D00404C
:10C62000000C004000B58DB001211448F5F710FA58
:10C630000120F5F70BFE032168460171012040033C
:10C640000390801004900802059000200690FF20BF
:10C6500002900B48099000200790002108A8417023
:10C6600081700121C1701520FEF7D0FA0320F5F783
:10C670001FFE01A8F5F724FE0DB000BD0400000266
:10C68000E808002010B50320F5F712FE0021032072
:10C69000F5F7A6FDFF2101310548F3F7C6FD044972
:10C6A0000320F5F7CBFD01210320F5F799FD10BD1F
:10C6B000E808002070B500260320F5F7B7FD054611
:10C6C0001848854216D0022003F074F80CE00320CD
:10C6D000F5F7ACFD0546022003F06CF83046711CFE
:10C6E0008EB2642800DD04E00320F5F79FFDA84228
:10C6F000EDD100E070BD0B48281A84B2002C0FD099
:10C70000FF2C00DC00DDF5E707480480002322460B
:10C71000C11FF939034802F0F8FD01210248817078
:10C7200000BFE7E7E8080020AA1D002070B58AB026
:10C7300006460C46154601212548F5F789F90022E1
:10C7400002212448F4F728FE002201212148F4F7B1
:10C7500023FE00200990079608A84470002C03D1FE
:10C76000012008A9087002E0022008A9087008A8A2
:10C7700085706846F5F728F86A4607A9164801F05B
:10C78000DDF90A20FEF742FAFF21134801F0C6FB4B
:10C79000114801F09BFB01210F4801F063FB0121CF
:10C7A0000D4801F006FB02210A20FEF79BFA0A2041
:10C7B000FEF744FA0121084801F0E3FA0121064896
:10C7C00001F011FB044801F072FB0AB070BD0000DB
:10C7D00007000001400C00400068014010B5F7F769
:10C7E00039FF002240210248F8F75DF810BD000033
:10C7F000C00C00407047000070B50646FEF7EAF92D
:10C80000002E04DD652E02DA304602F0D3FF40210F
:10C810000D48F7F73EF8054680210B48F7F739F841
:10C820000446002D02D1012C00D170BD012D03D191
:10C83000002C01D10220F8E7012D03D1012C01D1F8
:10C840000520F2E70520F0E7400C0040F0B58DB080
:10C8500004460F460020069006AA3946204604F0FA
:10C860006BF8002801D10DB0F0BD6846007E22288B
:10C8700077DBE41C002306227E49204602F045FDBA
:10C88000012304220BA9A01D02F03FFD0123022277
:10C890000AA920460A3002F038FD6846008DF3F7F9
:10C8A000A1FF754A754B01910090F3F795FE039136
:10C8B00002900B98F3F796FF0546039B029AF3F755
:10C8C000D7FD6C4A0E3205910490F3F7EEFC01237C
:10C8D00004220BA920460C3002F017FD012302228E
:10C8E0000AA92046103002F010FD6846008DF3F7CB
:10C8F00079FF614A614B01910090F3F76DFE05915C
:10C9000004900B98F3F76EFF03910290059B049A35
:10C91000F3F7AEFD0546574A921DF3F7C6FC012317
:10C92000042254493C312046123002F0EEFC01232F
:10C930000422504938312046163002F0E6FC01232B
:10C9400004224C49403120461A3002F0DEFC01231B
:10C9500004224849443120461E3002F0D6FC02E051
:10C96000FFE700207FE76846007E622867DB01233F
:10C9700004220BA92046223002F0C7FC0123022228
:10C980000AA92046263002F0C0FC6846008DF3F765
:10C9900029FF394A394B01910090F3F71DFE0391AD
:10C9A00002900B98F3F71EFF0546039B029AF3F7DC
:10C9B0005FFD304A2E3205910490F3F776FC012397
:10C9C00004220BA92046283002F09FFC01230222FA
:10C9D0000AA920462C3002F098FC6846008DF3F737
:10C9E00001FF0546244A254BF3F7F6FD039102901B
:10C9F0000B98F3F7F7FE01910090039B029AF3F76F
:10CA000037FD1C4A263205910490F3F74EFC0123B2
:10CA1000082218491E312046463002F076FC0123D8
:10CA200008221449163120464E3002F06EFC0023D5
:10CA30000C2207A92046563002F067FC17E00D4A89
:10CA40002E3200200146F3F730FC0A4A263200203D
:10CA50000146F3F72AFC074A1E3200200146F3F78D
:10CA600024FC044A163200200146F3F71EFC012084
:10CA7000F9E60000B01D00207B14AE47E17A843F48
:10CA800010B501213048F4F7E3FF002280212F4840
:10CA9000F4F782FC0022FF2101312C48F4F77CFCE2
:10CAA0000022012149022948F4F776FC0121284897
:10CAB000F4F7CEFF0021274800F08DF8FF21013167
:10CAC000244800F0A1F80021224800F0AAF808212B
:10CAD000204800F05FF800211E4800F089F800218E
:10CAE0001C4800F06CF800211A4800F05FF80021A3
:10CAF000184800F0E1F80021164800F0B8F80021CD
:10CB0000144800F09AF80021124800F0A3F8002120
:10CB1000104800F0C5F800210E4800F0D9F80021B7
:10CB20000C4800F0E1F80B4800F0F0F8094800F07C
:10CB3000E7F8084800F0E7F8064800F0EAF80121B5
:10CB4000044800F0A1F810BD07000001800C00406F
:10CB500003000003004C014010B500210A48F4F71F
:10CB600077FF0021094800F08FF880210848F5F789
:10CB700027F9FF2101310648F5F722F90121490281
:10CB80000348F5F71DF910BD03000003004C0140F8
:10CB9000800C004010B50A46016838240B46A343B8
:10CBA0001946382313401943016010BD0A46016835
:10CBB00049084900D307DB0F19430160704710B5DE
:10CBC0000A46016802240B46A34319460223134078
:10CBD0001943016010BD10B50A4601680124E40242
:10CBE0000B46A3431946234613401943016010BD69
:10CBF00010B50A46016804240B46A34319460423D2
:10CC000013401943016010BD10B50A460168FF24A6
:10CC100001340B46A34319462346134019430160D0
:10CC200010BD10B50A460168C0240B46A34319463F
:10CC3000C02313401943016010BD10B50A46416876
:10CC4000032464020B46A3431946234613401943A9
:10CC5000416010BD10B50A464168FF2401340B46FF
:10CC6000A3431946234613401943416010BD0129CF
:10CC700004D14268CB021A43426004E042680123B7
:10CC8000DB029A4342607047012904D142680123C4
:10CC90001A43426003E04268520852004260704703
:10CCA00010B50A46416820240B46A34319462023A9
:10CCB00013401943416010BD012904D14268022389
:10CCC0001A43426003E0426802239A43426070477D
:10CCD000012904D1426810231A43426003E04268EC
:10CCE00010239A4342607047012904D14268082307
:10CCF0001A43426003E0426808239A434260704747
:10CD000002218160704704218160704701218160A8
:10CD1000704708218160704701460869C007C00F4D
:10CD2000002801D0012070470020FCE70146086977
:10CD300002221040002801D0012070470020FCE7AB
:10CD400001468869704741617047000010B50121B4
:10CD50000448F4F77DFE002208210348F7F7A3FDFD
:10CD600010BD000007000001C00C004010B50121FB
:10CD70000448F4F76DFE002208210348FEF700F98D
:10CD800010BD000007000001C00C004010B50346B4
:10CD9000042000240C700124148010BDF8B5064650
:10CDA0000C4615460427002380220549304602F030
:10CDB000ACFA00202070012028803846F8BD000021
:10CDC00030040020FFB585B004460D4616460E9F80
:10CDD00014A103C9049103906846047145718671DA
:10CDE000C7710F99017269461098487202990198AB
:10CDF00000F076FD012813D1694610980873684643
:10CE00000F99417387730899C173067445748474CC
:10CE1000072203A90020FFF707FA012009B0F0BD9F
:10CE20000020FBE700000000010115001CB50021F7
:10CE3000684601704170022181700021C17060213B
:10CE40000171052269460B20FFF7EEF91CBD0000B9
:10CE500070B592B000262E480088002808D02D48D2
:10CE6000F3F702FA0446224629492B48FFF700F857
:10CE70002A480078012808D100202849087026484F
:10CE8000FFF71EFA012800D101262248401F8078B2
:10CE900001280BD1224908790521F3F741F900292E
:10CEA00004D11F484079002800D10126012E00D16D
:10CEB00000BF1D221B496846F3F79EF9164A3D3212
:10CEC000002001461378184353781B0218439378C7
:10CED0001B041843D3781B0618431379194353795D
:10CEE0001B02194393791B041943D279120611438B
:10CEF00004460D4625220B49083908A8F3F77CF9AA
:10CF000020462946099B089A02F020FA12B070BD0B
:10CF100094060020770300204A120020FA02002025
:10CF2000CC020020BE040020244909684878234927
:10CF300009684979214A12685170204909684A7A7A
:10CF40001E4909684A711D4909684A7B1B490968DD
:10CF50004A721A4909684873184909688878174954
:10CF60000968897A154A12689170144909688872AB
:10CF7000124909688879114909688A7B0F4909684B
:10CF80008A710E49096888730C490968C8780B4989
:10CF90000968C97B094A1268D17008490968CA7AC8
:10CFA00006490968CA7305490968CA7903490968C5
:10CFB000CA7202490968C871704700000000002069
:10CFC000F7B58EB00D461646002400200D900420C3
:10CFD0000390002002900D900E98841C0AE00D989A
:10CFE000401C80B20D90641C0D980A2802DD0420BC
:10CFF00011B0F0BD20786828F1D100231A2206A9CB
:10D00000204602F082F96846018E20461A30081840
:10D010000123022205A9019002F077F96846008EEB
:10D0200002461A3221466D4804F0BCFE07466946A6
:10D03000898A8F4264D101F089FC08A8C07B8021D5
:10D040000840802809D16846038E08A8C07B224684
:10D050001A3211460190F5F78DF908A8817A427AC3
:10D0600008021043FF220532811A90422BD008DCBF
:10D07000FF38023800280BD0012812D002283DD1F9
:10D0800018E0FD2928D0FF39FF39002936D12CE0DE
:10D0900002AA29461A3120461A30F5F7D5F903902D
:10D0A0002DE002AA29461A3120461A30F5F7F0FC85
:10D0B000039024E002AA29461A3120461A30FFF7CD
:10D0C0006DFE03901BE002AA29461A3120461A3051
:10D0D000FEF7C0FF039012E002AA29461A3120464B
:10D0E0001A30FEF7B7FF039009E002AA29461A3169
:10D0F00020461A30FFF74AFE039000E000BF00BF51
:10D1000068460089002865DD002306223449354839
:10D1100002F0FBF8012132480A38C1740021017580
:10D12000012141750021817508A8817A427A08029F
:10D1300010432B490A394874000A887408A8C07B38
:10D14000C87508A8C07B80210840802810D108A895
:10D15000C07B02AB2A461A3211460190F5F732F92C
:10D16000684601891E480A380176090A417606E0B8
:10D17000684601891A480A380176090A417600236F
:10D180001A22294616480A3802F0BFF814490A390B
:10D19000487E097E000208431A3080B20490294676
:10D1A0000E48049A04F0FEFD0F490870000A48700A
:10D1B0001620887004982918002303220A4802F0D8
:10D1C000A4F807490A39487E097E000208431D3049
:10D1D000308001E000203080039809E7FFFF000065
:10D1E00055060020CC02002065060020F0B597B05F
:10D1F00004460020159000230622A649A64802F006
:10D2000084F800201CE04200A4495218517812789A
:10D21000090211434200A24BD3185A781B7812021C
:10D220001A43114343009D4A9A181170090A51701C
:10D23000002142009A4BD21811705170411CC8B2A3
:10D240000728E0DB012193480A38417500218175E8
:10D250000121C174002101757B208E490A390876AD
:10D260000020487601218D48401C017600230822C9
:10D2700004A9894802F049F88A48F2F7FFFF002222
:10D28000894B01910090F3F7A7F90546F3F766FB88
:10D2900005AA023203910290F3F707F8814808309B
:10D2A000F2F7ECFF054600227F4BF3F795F9019169
:10D2B0000090F3F753FB07AA023203910290F2F7B2
:10D2C000F4FF7849891F886B7849F3F756F80646CA
:10D2D000F3F7ACFA054609A90231F2F7DDFF71490F
:10D2E000891FC86B7149F3F748F80646F3F79EFAB1
:10D2F00005460AA90231F2F7CFFF6A49891F486C37
:10D300000BA90231F2F7C8FF6649891F086C0CA906
:10D310000231F2F7C1FF664A00210846137819432B
:10D3200053781B02194393781B041943D3781B06C7
:10D3300019431379184353791B02184393791B043B
:10D340001843D279120610430D4601460022594B6C
:10D350002846F3F741F901910090F3F7D7FA0DAAA7
:10D36000023203910290F2F7A0FF514A121F137884
:10D37000194653781B02194393781B041943D2783A
:10D380001206114308460FA90231F2F785FF4A48F9
:10D39000F2F76AFF06464949F2F7EFFF0546F3F751
:10D3A0005EFAC1B210A881704348401F417D10A8A9
:10D3B000C1704148401DF2F757FF06463F49F2F75A
:10D3C000DCFF0546F3F74BFAC1B210A801713A48E9
:10D3D000401F817D10A8417100230C22811D384817
:10D3E00001F093FF002342222146533104A801F0AB
:10D3F0008CFF0023392221461A3128481F3801F0BA
:10D4000084FF24480A38C07D80210840802816D136
:10D4100020490A39487E097E0002084315901D49BB
:10D420000A39C87D15AB22461A321146F4F7CAFFF5
:10D4300010A9898A17480A380176090A417600231B
:10D440001A22214613480A3801F05FFF11490A39B0
:10D45000487E097E000208431A3087B23A462146C8
:10D46000184804F09FFC18490870000A48701620FC
:10D470008870E11900230322134801F046FF054993
:10D480000A39487E097E000208431D3080B217B079
:10D49000F0BD000055060020CC020020601C0020DA
:10D4A000CC080020B61D00200088C34000401C4668
:10D4B0008712002000408F40E3020020000020413E
:10D4C000C0080020FFFF00006506002010B541489D
:10D4D000417D027D080210433F498871000AC871EE
:10D4E00000203E4908703B48C01E417D027D080275
:10D4F00010433C21484380B237490873000A4873FF
:10D5000068203749087000230822491C354801F07B
:10D51000FCFE55203249487242200874FF21023136
:10D520002F484174090A817480202D49C8752D48FF
:10D530000830407980302C4908702A481838807D9E
:10D54000487025480078887000231422C91C274899
:10D5500001F0DBFE2548113800782349C8750846DC
:10D56000C07D142802DD012008760AE01E48C07D37
:10D570000F2803DD02201C49087602E003201A4927
:10D5800008761A4811384078174948760023042253
:10D590001A31174801F0B9FE16480078C006C00FCE
:10D5A000114988771449487A097A000208430E49DC
:10D5B00021310873000A487300210B482030C175DF
:10D5C000012107484175002181750121C1740021A5
:10D5D000017510BD0A040020071B00207006002002
:10D5E0004B06002044030020411C0020291C002081
:10D5F0000D120020C0080020F912002010B50446CA
:10D6000021460A48FFF79FFB00BF0848FFF78EFB43
:10D610000028FAD000BF0548FFF77EFB0028FAD0AB
:10D620000248FFF78DFB0446E0B210BD004C0140FC
:10D6300070B5002413E000250DE0A900094A126826
:10D640008918085D02F054FFA900064A126889187B
:10D650000855681CC5B2042DEFDB601CC4B2042C55
:10D66000E9DB70BD000000207CB56B48017868469E
:10D67000017069484178684641706748817868461A
:10D6800081706548C1786846C17063480179684611
:10D690000171614841796846417101990098F5F737
:10D6A0005BFA5E480078012802D100205B490870CF
:10D6B00000249FE0E000201859494118C878897873
:10D6C0000002084300114000564941184878097883
:10D6D00000020843E1006118514A8A18D178927813
:10D6E000090211430907090F0841C007C00F0028AC
:10D6F0007BD0E00020184A49411848790979000296
:10D700000843001140004849411848780978000250
:10D710000843E1006118424A8A18517912790902D6
:10D7200011430907090F08410646B607B60F032E35
:10D7300040D10221084600F085FF3C49487A097A29
:10D74000000208430121C9030840884222D1374919
:10D75000487A097A000208430121C90305468D432E
:10D76000902D42D1912D40D1922D3ED1932D3CD17F
:10D77000942D3AD1E00020182949411848780978B9
:10D78000000208430121C903084328490872000A1E
:10D7900048722AE0E00020182149411848780978A9
:10D7A000000208430121C903084320490872000A06
:10D7B00048721AE0012E18D10221012000F042FF28
:10D7C0001A49487A097A00020843F103084088425E
:10D7D0000BD0E0002018124941184878097800025F
:10D7E000084312490872000A4872C82C00DD04E0A0
:10D7F000601C84B2422C00D25CE700BF002407E02A
:10D8000000206100074A891808704870601C84B2C3
:10D81000072CF5D37CBD0000CC02002008000020BE
:10D8200046000020DA08002030000020F912002015
:10D830001FB500240120F4F713FA07200002F4F7C3
:10D8400021FA032001F0B6FF0120F4F74DF805E0BE
:10D8500019200002844200D304E0641CF4F758F855
:10D860000028F5D000BF0120009000200190029018
:10D870000120694608736846F4F7E2F9014801F0AF
:10D8800075FF1FBD001BB7000148024908607047C3
:10D8900000127A007007002010B572B6F6F78CFF00
:10D8A0000D4801F063FF0A2001F084FFF6F7F0FF56
:10D8B0000120FEF7F3FC0620FEF7CEFC0020FEF769
:10D8C000DBFCF4F753FB01210448F4F7C1F8F6F749
:10D8D0006BFF62B610BD000000127A000700000165
:10D8E000F3B582B06E46337ADE17360FF61837116D
:10D8F0000A2677436E46307AC617360F3618361129
:10D900003601861BBE19F2B26E46737ADE17360FE9
:10D91000F61837110A2677436E46707AC617360F07
:10D92000361836113601861BBE19F4B26E46B37A2C
:10D93000DE17360FF61837110A2677436E46B07A8F
:10D94000C617360F361836113601861BBE19F1B2CE
:10D950006E46F37ADE17360FF61837110A2677432C
:10D960006E46F07AC617360F361836113601861B0A
:10D97000BE19F5B26E46337BDE17360FF618371137
:10D980000A2677436E46307BC617360F3618361197
:10D990003601861BBE19F6B201966E46737BDE1702
:10D9A000360FF61836110A277E436F46787BC71765
:10D9B0003F0F3F183F113F01C71BF619F6B2009603
:10D9C000322A11DC142A0FDB0C2C0DDC002C0BD0BE
:10D9D0001F2909DC002907D0172D05DC01983B28F9
:10D9E00002DC00983B2802DD002004B0F0BDA01E40
:10D9F000030001F0F6FA0A0E1E061E071E1E081E80
:10DA0000091E00BF00BF00BF1E2901DD0020ECE79A
:10DA100000BF9007800F002803D01C2901DD0020E3
:10DA2000E3E79007800F002802D11D2900DDDCE725
:10DA300000E000BF00BF0120D7E7000010B5064896
:10DA400000F039FA012806D1034800F03FFA01201E
:10DA500002494870087010BD00680140BE020020F5
:10DA6000F3B585B00F460598F2F7A1FE0546384696
:10DA7000F2F79DFE06462946F2F7BCFC04907F2192
:10DA8000C9050498F2F7ECFF13D20498F2F786FF69
:10DA900005460022094BF2F790FD0022084B019148
:10DAA0000090F2F7E5FC03910290F2F711FF0446B3
:10DAB00000E00024204607B0F0BD00000000F03F69
:10DAC0000000E03F30B505460C462846616800F08E
:10DAD0003DF92846A16800F048F92846E16800F0C1
:10DAE00038F92846616900F071F9617C284600F038
:10DAF000ACF9217C284600F0B5F92178284600F0E1
:10DB000097F96178284600F0BAF9A178284600F024
:10DB1000C2F9A17E284600F040F9E17E284600F0D7
:10DB20007BF9A17C284600F02CF9217E284600F0E4
:10DB30005AF9617E284600F062F930BD70B588B0B0
:10DB400006460C4615467A48864228D1A068F3F767
:10DB50004DFF0120F3F736FF01217648F3F778FFF8
:10DB6000A068002804D0012808D0022815D10EE0B2
:10DB7000A9682068FFF774FF02900FE00120F3F717
:10DB8000DDFFE9682068FFF76BFF029006E0296877
:10DB90002068FFF765FF029000E000BF63E0664881
:10DBA000864229D1A068F3F743FF0120F3F72CFF49
:10DBB00001216048401CF3F74BFFA068002804D007
:10DBC000042808D0082815D10EE0A9682068FFF7BE
:10DBD00047FF02900FE00120F3F7B0FFE9682068EB
:10DBE000FFF73EFF029006E029682068FFF738FF44
:10DBF000029000E000BF36E0504886420AD1012181
:10DC00004C48801CF3F724FFA9682068FFF728FF21
:10DC1000029028E04A4886420AD101214548C01CAA
:10DC2000F3F716FFA9682068FFF71AFF02901AE0C1
:10DC3000444886420AD101213E48001DF3F708FFFF
:10DC4000A9682068FFF70CFF02900CE03E4886426E
:10DC500009D101213748401DF3F7FAFEA968206871
:10DC6000FFF7FEFE02902079012810D1402003909A
:10DC70006079012802D1102004903FE060790228E9
:10DC800002D12020049039E00020049036E0207971
:10DC9000022810D1802003906079012802D1102041
:10DCA00004902BE06079022802D12020049025E026
:10DCB0000020049022E0207900280FD103906079A1
:10DCC000012802D11020049018E06079022802D1C6
:10DCD0002020049012E0002004900FE0C020039068
:10DCE0006079012802D11020049007E060790228B1
:10DCF00002D12020049001E000200490A0790028A7
:10DD000001D1069002E0FF20013006900021684614
:10DD1000017141718171417501758177C17781759B
:10DD20000177417701A93046FFF7CCFE08B070BDFE
:10DD3000002001400800000300680140006C014021
:10DD40000070014000740140007801408AB2826195
:10DD5000704710B50A46016830240B46A3431946A4
:10DD6000302313401943016010BD10B50A46016805
:10DD7000C0240B46A3431946C02313401943016036
:10DD800010BD012904D1026802231A43026003E096
:10DD9000026802239A4302607047012904D1026895
:10DDA00008231A43026003E0026808239A430260D2
:10DDB0007047012904D102680B041A43026004E091
:10DDC000026801231B049A430260704710B50A469B
:10DDD0000168FF2401340B46A34319462346134030
:10DDE0001943016010BD012904D1026801231A43BF
:10DDF000026003E002685208520002607047012985
:10DE000004D102684B041A43026004E00268012353
:10DE10005B049A4302607047012904D1026804231D
:10DE20001A43026003E0026804239A4302607047C9
:10DE3000012904D142680B021A43426004E042689F
:10DE4000FF2301339A4342607047012904D142689D
:10DE50008B021A43426004E0426801239B029A430A
:10DE600042607047012904D14268CB021A434260E4
:10DE700004E042680123DB029A43426070470129B3
:10DE800004D1426802231A43426003E0426802233D
:10DE90009A4342607047012904D1426801231A4322
:10DEA000426003E042685208520042607047FF211E
:10DEB000013181607047014688680122D20210401A
:10DEC000002801D0012070470020FCE70121C90291
:10DED0008160704701468868C007C00F002801D0E4
:10DEE000012070470020FCE701460869C005C00D0D
:10DEF0007047F8B507460D46164600240BE0295D2D
:10DF0000384600F013F800BF3846FFF7E3FF00285B
:10DF1000FAD0601C84B2B442F1DBF8BD0A46C16895
:10DF2000090A0902D3B21943C1607047CA05D20D6C
:10DF30004261704710B501210448F3F789FD0022C2
:10DF400002210348F6F7AFFC10BD000007000001F6
:10DF5000C00C004010B501210648F3F779FD0022FE
:10DF600004210548FDF70CF804210348F5F79BFC54
:10DF700010BD000007000001000C004010B5FFF7C5
:10DF8000D9FF02213148F5F784FC012842D13048FD
:10DF90000078022838DB00BF2E4840780007C00F09
:10DFA000002830D12C4840780007C00F00282AD024
:10DFB0002848407808218843083026494870274877
:10DFC0004078082188430830244948700321002004
:10DFD00003F0C6F8224840780007C00F00280ED092
:10DFE0000320F3F729F8012809D11E4840780821B9
:10DFF000884308301B49487001201B4908700321E1
:10E000001A48F3F75CF820E011480078401C1049EA
:10E0100008701AE00E480078002811D100BF0D48A2
:10E0200040780007C00F002809D00A48407808212E
:10E0300088430849487003210C48F3F73FF804E08F
:10E0400003480078401E0249087010BDC00C004013
:10E05000FB020020C008002014000020DA08002085
:10E0600022000020CC08002008000020B40200207C
:10E0700010B501210448F3F7EBFC00220821034806
:10E08000F6F711FC10BD000007000001400C004035
:10E0900010B501210348F3F7DBFC08210248F3F730
:10E0A0008FFE10BD07000001400C0040F8B504468B
:10E0B0000D460126E17821488078814205D12179F9
:10E0C0001E48801C4078814200D00226A078642837
:10E0D00009D0A078012806D0A078022803D0A07823
:10E0E000032800D00026012E08D100BFE12109013C
:10E0F0001348C18100201249087300BFF2F724F8C9
:10E1000007466421F2F70CF80F02F2F71DF86421BC
:10E110000090F2F705F80F43B9B20A480180E9719F
:10E12000090A29720120A8720020E872E87AA97A07
:10E13000000208430B302E543046F8BD4C0300203B
:10E140009A0200204806002010B50446204600F040
:10E1500043F810BDF8B504460D461D480078012867
:10E1600034D1217AE279080210431A490988884299
:10E170002CD1607B217B000208432873000A68735E
:10E18000607B217B000208430006060C607B227B3B
:10E1900000021043FF2212021040001206432746DD
:10E1A0000E37012E02D02D2E0ED106E0607A2B46BE
:10E1B0003A463146F3F776FD07E0607A2B463A4659
:10E1C0003146F3F789FD00E000BF00BFF8BD000055
:10E1D000440600204806002070B5044600BFE07ADF
:10E1E000A17A000208430C3085B2E07AA17A0002DD
:10E1F00008430006010CE07AA27A00021043FF22D5
:10E200001202104000120143A172080AE0722A466D
:10E2100021460C4803F0C6FD064630126055681CC6
:10E220002654012189020848F5F73FFBA81C82B259
:10E2300021460648FFF75DFE012189020248F5F7F5
:10E2400032FB70BDFFFF0000000C00400078014071
:10E25000012806D10649496A01221143044A516244
:10E2600005E00349496A49084900014A516270477B
:10E2700000F801400146064A506A0E2302469A43BE
:10E2800010460E220A401043014A506270470000B7
:10E2900000F8014000B507484368180CD94389B21B
:10E2A000884203D1D8B200F019F802E01F2000F034
:10E2B00015F800BD40FBFF1F012806D1064949693A
:10E2C00080221143044A516105E0034949698022D3
:10E2D0009143014A5161704700F801400146054AE7
:10E2E0005069800980018A06920E1043014A5061EC
:10E2F0007047000000F8014070B505460C46C7485D
:10E300008079012814D1002301228021C448F4F728
:10E3100083FF0020FEF770FA012805D00320C149D1
:10E32000887000F07BFA02E00120BE49887070BD61
:10E33000BA480078032839D10020FEF75DFA012899
:10E3400011D100F06BFA0120B64988700020B34962
:10E3500088800A4611785078002203F0F6F80020F1
:10E36000AE490870ACE060780128FBD0E078012865
:10E37000F8D02846F5F7F2FEA849488000F03CFAAC
:10E380000320A8498870A54A11785078002203F02C
:10E39000DCF80020A14908700A2001F00BFA0123E3
:10E3A0001A4640219E48F4F737FF89E09B480078E1
:10E3B000012803D099480078022858D10020FEF7A0
:10E3C0001BFA022821D100F029FA02209549887011
:10E3D0000020924948809348C078002806D108461A
:10E3E0000078022802D101208E49C8708D4E737AC0
:10E3F000367A1B0233431A46884B1978587803F053
:10E40000A4F80020854908705AE06078012857D0A8
:10E41000E078012854D02846F5F7A0FE7F4988808F
:10E4200000F0B8F904207F4988700846C0780028B9
:10E4300005D17A480078022801D10120C870794EB0
:10E44000737A367A1B0233431A46744B197858781C
:10E4500003F07BF80020714908700A2001F0AAF946
:10E4600001231A4680216E48F4F7D6FE28E06B4857
:10E470000078042810D16B48C078002808D101200A
:10E480006849C870654A11785078002203F05DF839
:10E4900000206249087013E06048007805280FD119
:10E4A0006048C078012808D100205E49C8705B4AE6
:10E4B00011785078002203F048F80020574908707E
:10E4C0005848807803281AD10020FEF795F90128D2
:10E4D00005D100F0A3F90120524988702DE04F4882
:10E4E0004088002805D100F099F905204D49887031
:10E4F00023E04A484088401E484948801DE049487A
:10E500008078042819D10020FEF776F9022805D179
:10E5100000F084F90220434988700EE03F4880886B
:10E52000002805D100F07AF905203E49887004E002
:10E530003A488088401E394988803A4880780328C4
:10E5400003D038488078042802D10121617101E0AC
:10E55000002161713348C078002806D132488078A4
:10E56000082188433049887006E02F4880780821C8
:10E57000884308302C4988702A48807805283FD184
:10E58000294880784007400F052844D027488078E4
:10E59000C007C00F00282BD000BF25488078C007D7
:10E5A000C00F002823D02348807840084000401C3A
:10E5B000204988707021002002F0D2FD1B4880782D
:10E5C000C007C00F00280ED07020F2F735FD0128DB
:10E5D00009D11948807840084000401C16498870CD
:10E5E00001201649087070211548F2F768FD00BF38
:10E5F0001048807840084000401C0E4988700AE0AE
:10E60000084989784807400F07498978C908C9002F
:10E610000143054A917000BF89E60000D602002040
:10E62000400C0040F9120020C00800202200002009
:10E6300014000020DA080020CC0800200800002088
:10E64000B402002000B5024632484170130000F0C9
:10E65000C8FC0604293D0558535D58E02E48007952
:10E660008006C00F002805D12B480079C006C00FD6
:10E67000002806D0284840788007C00F002800D125
:10E6800000BD2648807802280BD1224880790028D6
:10E6900007D103201F4B18700420214B5870012014
:10E6A000EEE734E01D48807802280DD01B488078C2
:10E6B000042809D017488079002805D10120154B7E
:10E6C00018700420164B58700120D9E70420114B14
:10E6D00018701248807802280CD0104880780428DE
:10E6E00008D018468079002804D102201870042030
:10E6F0000B4B58700120C3E70520064B1870012012
:10E70000BEE70420034B18700120B9E700BF00BF2B
:10E710000020B5E7D6020020C0080020F912002032
:10E72000DE02002010B50024F4F7F0FB01210903FC
:10E730001648F5F7AEF801280AD1052001F03AF89D
:10E74000012109031148F5F7A4F8012800D101249B
:10E75000012C0CD10E48807901280FD001200C49E2
:10E76000887100220621052002F0EFFE06E008482D
:10E770008079012802D100200549887104488079F8
:10E78000012802D10020FEF737F810BD800C0040B0
:10E79000D602002010B5154800798006C00F002869
:10E7A00005D112480079C006C00F00280ED00F48CE
:10E7B00040788007C00F002808D100F0C7FF04216F
:10E7C0000B48F5F772F8012000F0F4FFFCF7F2F9BE
:10E7D000FCF700FAFF2101310648F5F764F8012142
:10E7E00049020448F5F761F810BD0000C008002098
:10E7F000800D0040400C004010B5FCF7DBF9FCF741
:10E80000E9F9FF2101310448F5F74FF801214902E8
:10E810000148F5F748F810BD400C004010B5FCF772
:10E82000C9F9FCF7E5F90023012240210C48F4F76F
:10E83000F3FC0023012280210948F4F7EDFCFF21BD
:10E8400001310748F5F72FF8012149020448F5F78F
:10E850002AF800F07BFF04210248F5F724F810BDE8
:10E86000400C0040800D004010B50446012C02D041
:10E87000022C07D100E000BF0020FDF7BDFF0349D7
:10E88000887000E000BF00BF10BD0000F91200203A
:10E8900010B5FCF78FF9FF2101310548F5F703F8B2
:10E8A000012149020248F4F7FEFFFCF7A1F910BD6F
:10E8B000400C004010B5002240210A48FCF760FBE4
:10E8C000002280210748FCF75BFB20210548F3F775
:10E8D00077FA80210348F4F7E6FF40210148F4F776
:10E8E000E2FF10BD000D004000B58DB001211448BD
:10E8F000F3F7AEF80120F3F7A9FC03216846017194
:10E90000012040030390801004900802059000202D
:10E9100006900C4802900C480990002007900021B6
:10E9200008A8417081700121C1701520FCF76EF9B3
:10E930000320F3F7BDFC01A8F3F7C2FC0DB000BD46
:10E9400004000002FF030000E80D002010B50320C2
:10E95000F3F7AEFC00210320F3F742FC012189020A
:10E960000548F1F762FC04490320F3F767FC012135
:10E970000320F3F735FC10BDE80D0020F8B505467F
:10E9800000270320F3F752FC06461C48864216D0A7
:10E99000022000F00FFF0CE00320F3F747FC0646CF
:10E9A000022000F007FF3846791C8FB2642800DD92
:10E9B00004E00320F3F73AFCB042EDD100E0F8BDEB
:10E9C0000E48301A84B2002C15D0FF2C03DC012035
:10E9D0008002844200DBF2E7E81DF9300470210A6E
:10E9E0004170002322462946044800F08EFC012194
:10E9F000FF200330415500BFE1E70000E80D002093
:10EA000070B58AB006460C46154601212548F3F735
:10EA10001FF8002210212448F2F7BEFC0022082132
:10EA20002148F2F7B9FC00200990079608A8447025
:10EA3000002C03D1012008A9087002E0022008A9D7
:10EA4000087008A885706846F2F7BEFE6A4607A9F6
:10EA50001648FFF773F80A20FCF7D8F8FF2113488F
:10EA6000FFF75CFA1148FFF731FA01210F48FFF771
:10EA7000F9F901210D48FFF79CF902210A20FCF762
:10EA800031F90A20FCF7DAF801210848FFF779F993
:10EA900001210648FFF7A7F90448FFF708FA0AB072
:10EAA00070BD000007000001000D0040006801403B
:10EAB00010B590B00446A07801280DD160790028E7
:10EAC0000AD16078002807D1A07023484078002838
:10EAD00002D10120204948701F484078030000F00F
:10EAE00080FA0604050A0F14191E19E000F0DCF87C
:10EAF0001949487014E000F0B3F8174948700FE066
:10EB000000F078F9144948700AE000F0B9F91249A8
:10EB1000487005E000F024F80F49487000E000BF9D
:10EB200000BF0D484078002802D10021E17001E0CB
:10EB30000121E170152209496846F1F75DFB2522A4
:10EB40000649103906A8F1F757FB06A80FC8FBF7CE
:10EB5000D9FE10B010BD0000071B0020C604002025
:10EB60001CB537A103C90191009037480078374997
:10EB7000087137480078012800D101E03348007956
:10EB8000324948710020324908703049487A097A80
:10EB900000020843401C81B22C480172090A4172EC
:10EBA0000146487A097A0002084301280DD100BFC6
:10EBB000072269462748FFF79CF90A2000F022FE49
:10EBC000FFF792FE00BF05201CBD2049487A097A54
:10EBD0000002084303280CD140211F48F4F763FECC
:10EBE0000A2000F00FFE80211B48F4F75CFE052090
:10EBF000EAE71649487A097A0002084308281CDB2C
:10EC000040211548F4F74FFE80211348F4F74BFEDE
:10EC10000E48007900280AD10C48007806280AD04E
:10EC20000E48817D09488172090AC17203E0002102
:10EC300006488172C1720020C6E70520C4E70000C3
:10EC40004154434C4F53450070060020071B0020E1
:10EC50007106002000680140000D004007040020FC
:10EC600010B500221146E1204002FFF7C9FEFFF770
:10EC70003BFE00200949087000F034F800200849E4
:10EC8000887000BFC8798979000208430549488027
:10EC90000020087000BF042010BD0000BE0200204C
:10ECA000071B00209A02002010B5FFF703FE802109
:10ECB0000A48F4F7FAFD0A2000F0A4FD40210748B5
:10ECC000F4F7F3FD00200649C870002104480172E2
:10ECD0004172FEF7FBFB022010BD0000000D00405A
:10ECE000071B002010B5C0B01B21684601704170A1
:10ECF0000021817000230422C11C3C4800F005FB68
:10ED00000023022201A903313848001D00F0FDFA5A
:10ED1000002406E00021204609306A461154601C98
:10ED2000C4B2402CF6DB0023022212A902312F4884
:10ED3000353000F0EAFA022110A801730121417375
:10ED40002A48801E017A10A881730021C173002413
:10ED500006E00021204650306A461154601CC4B2BF
:10ED6000402CF6DB002406E00021204690306A4665
:10ED70001154601CC4B2202CF6DB002406E00021F4
:10ED80002046B0306A461154601CC4B2142CF6DB25
:10ED9000002406E000212046C4306A461154601C5D
:10EDA000C4B2072CF6DB002030A9C872002409E0A9
:10EDB00030A8C07A6946095D4018C1B230A8C17256
:10EDC000601CC4B2CB2CF3DB162030A9087300BF43
:10EDD000CD2269460648FFF78CF80A2000F012FDA4
:10EDE000FFF782FD00BF40B010BD0000E903002026
:10EDF0000068014010B5FFB0FFB084B01C4901A805
:10EE0000F1F713FA01A80330FEF7F0F90446672181
:10EE1000684601714471211281711548401E844277
:10EE20000BD910201349C870002112480172417299
:10EE300005207FB07FB004B010BD00BFE01C82B2DF
:10EE400001A90D48FFF755F80A2000F0DBFCFFF799
:10EE50004BFD00BF00BF0749C8798979000208430C
:10EE6000064948800020087000BF0420E1E7000048
:10EE700004040000071B0020006801409A020020E3
:10EE800010B5FFB0FFB084B0434901A8F1F7CDF948
:10EE90000020009041480078012805D100203F491A
:10EEA00008703F48FFF76AFD3E488078012857D137
:10EEB00000213C4881703C488078002811D13848B6
:10EEC000FBF738F93849887008468078012847D11F
:10EED00001023348F1F7A9F903207FB07FB004B0F5
:10EEE00010BD3148807801283AD16A46D11D2C489E
:10EEF000FCF780FA044668460088002829DD684649
:10EF000000882549491E884223D26721684601713D
:10EF10000088C1B26846417100880112684681715B
:10EF200000BF0088C01C82B201A92048FEF7E1FFA3
:10EF30000A2000F067FCFFF7D7FC00BF00BF1A49AA
:10EF4000C87989790002084319494880002008706F
:10EF500000BFFF2101311248F1F767F92046BCE7F5
:10EF600013480078012814D10F488078002803D175
:10EF700002200D49C87006E00B488078012802D1B4
:10EF800003200949C8700021074801724172052019
:10EF9000A3E70420A1E7000004040000BE02002053
:10EFA000151B0020151C0020071B002000680140D5
:10EFB0009A0200202021020C01D010211046020AE2
:10EFC00001D010460839020901D01046091F8208F5
:10EFD00001D01046891E420801D0881E7047081AC9
:10EFE000704730B47446641E2578641CAB4204D369
:10EFF000635D5B00E31830BC18471D46F8E702E08C
:10F0000008C8121F08C1002AFAD1704770470020B3
:10F0100001E001C1121F002AFBD1704780F3108864
:10F0200070470000F0B585B00446002004902248E7
:10F03000808AA0421ED22049898A601AF1F7B7FB64
:10F0400000901E4801680098F1F7D4F901901C481F
:10F0500001680198F1F738F90746F1F79FFC05467A
:10F060000022184BF1F7A9FA03910290F1F7D2FCB4
:10F0700004901DE01049898A081BF1F798FB009065
:10F080000E4801680098F1F7B5F901900C48016845
:10F090000198F1F76EF90746F1F780FC054600226A
:10F0A000084BF1F78AFA03910290F1F7B3FC049050
:10F0B000049805B0F0BD000040FBFF1FC402002013
:10F0C000C80200200000E03FF0B587B004460027EA
:10F0D00013490A20085EF1F771FB05460022114B27
:10F0E000F1F7E2FA039102900D490989614308465C
:10F0F000F1F778FB054600220B4BF1F7D5FA0191A9
:10F100000090039B029AF1F7B3F905910490F1F78F
:10F11000BBFB0746002F00DA0027384607B0F0BDDA
:10F1200080FAFF1F0000594000408F4010B50024B6
:10F1300000BFF1F7D3FE012801D1002010BD204609
:10F14000641C401C0028F4D10120F7E710B5012011
:10F150008007F2F727FC0120F2F712FC01231A4680
:10F1600040213348F4F758F801231A465902304831
:10F170004030F4F751F801231A4619462C48F4F7A9
:10F180004BF801231A46590329484038F4F744F84C
:10F190002848C07B8021084080282FD025488078CF
:10F1A000012803D023488078032827D121480179FA
:10F1B000C278080210432049884218D01D480179BE
:10F1C000C278080210431C49491C88420FD01948D4
:10F1D0000179C278080210431849884207D00123F8
:10F1E0001A46202112484038F4F716F806E00123A9
:10F1F000002220210E484038F4F70EF81E20002887
:10F2000005DBC206D20E012191400D4A116000BFFC
:10F2100000211E20FBF72AFD1E20002806DBC20667
:10F22000D20E01219140064A803A116000BF10BD04
:10F23000C00C004072030020010700000113000011
:10F2400080E100E010B5F3F745FAFDF7C7FAF5F7EE
:10F25000A1FFFAF77BFCFCF789F8FFF719FBFCF735
:10F26000E7FEFDF77DF9FFF725FB10BD10B5012482
:10F2700002F03AFB002800D10024F3F74BFC0028F1
:10F2800000D10024F2F7D8FD002800D10024FBF7BC
:10F290004FF9002800D1002410BD000010B5002453
:10F2A0000C48F0F7E1FF0C49884206D201F0B1F8B2
:10F2B00008490948F0F7F0FF0124002C08D02A2360
:10F2C0003D221202FF2101310248801F01F05EFB46
:10F2D00010BD0000080300200506062410B5012417
:10F2E00002F020FB002800D10024F3F721FC0028C5
:10F2F00000D10024F2F7ECFD002800D10024FBF738
:10F30000FFF9002800D1002410BDF0B50446002B01
:10F310000CD125460E46002005E02F783770761C6C
:10F320006D1C471CB8B29042F7DB0EE0012B0CD1EC
:10F33000A7187D1E0E46002005E02F783770761C3A
:10F340006D1E471CB8B29042F7DBF0BD0FB4F0B5AC
:10F3500085B004460D460DA80230F0F785FF0190F8
:10F36000F1F72CFA0646F04AF04BF1F735F9224650
:10F370002B4603910290F1F725FB47D800BFEC48DC
:10F38000C0780007C00F002809D0E948C0780821DC
:10F390008843E749C8709021E648F1F78FFE00BF27
:10F3A00000BFE348C078C006C00F002809D0E0487D
:10F3B000C07810218843DE49C8709121DD48F1F7FB
:10F3C0007DFE00BF00BFDA48C0788006C00F00286D
:10F3D00009D0D748C07820218843D549C8709221E8
:10F3E000D448F1F76BFE00BF00BFD148C07840069B
:10F3F000C00F002809D0CE48C07840218843CC49AE
:10F40000C8709321CB48F1F759FE88E10EA802306D
:10F41000F0F72AFF0190F1F7D1F90646C24AC34B33
:10F42000F1F7DAF822462B4603910290F1F7CAFA77
:10F430006ED800BFBE48C0780007C00F002830D18A
:10F44000BD48C0780007C00F00282AD0B848C0784F
:10F45000082188430830B649C870B848C0780821E8
:10F4600088430830B549C8709021002001F078FE2B
:10F47000B348C0780007C00F00280ED09020F1F7E5
:10F48000DBFD012809D1AF48C07808218843083046
:10F49000AC49C8700120AC4908709021A548F1F72B
:10F4A0000EFE00BF00BFA248C078C006C00F0028F3
:10F4B00009D09F48C078102188439D49C870912188
:10F4C0009C48F1F7FBFD00BF00BF9948C07880065B
:10F4D000C00F002809D09648C0782021884394495D
:10F4E000C87092219348F1F7E9FD00BF00BF904832
:10F4F000C0784006C00F002809D08D48C078402150
:10F5000088438B49C87093218A48F1F7D7FD06E1FB
:10F510000FA80230F0F7A8FE0190F1F74FF9064668
:10F52000814A824BF1F758F822462B46039102900C
:10F53000F1F748FA5CD800BF7D48C078C006C00F1C
:10F54000002830D17C48C078C006C00F00282AD0DF
:10F550007748C0781021884310307549C8707748C3
:10F56000C0781021884310307449C8709121002060
:10F5700001F0F6FD7248C078C006C00F00280ED01A
:10F580009120F1F759FD012809D16E48C07810216A
:10F59000884310306B49C87001206B490870912175
:10F5A0006448F1F78CFD00BF00BF6148C078800659
:10F5B000C00F002809D05E48C078202188435C49EC
:10F5C000C87092215B48F1F779FD00BF00BF584831
:10F5D000C0784006C00F002809D05548C0784021A7
:10F5E00088435349C87093215248F1F767FD96E06C
:10F5F00010A80230F0F738FE0190F1F7DFF8064668
:10F60000494A4A4BF0F7E8FF22462B460391029005
:10F61000F1F7D8F94AD800BF4548C0788006C00F36
:10F62000002830D14448C0788006C00F00282AD076
:10F630003F48C0782021884320303D49C8703F486A
:10F64000C0782021884320303C49C8709221002096
:10F6500001F086FD3A48C0788006C00F00280ED021
:10F660009220F1F7E9FC012809D13648C078202121
:10F67000884320303349C8700120334908709221F3
:10F680002C48F1F71CFD00BF00BF2948C078400698
:10F69000C00F002809D02648C0784021884324495B
:10F6A000C87093212348F1F709FD38E000BF2048D6
:10F6B000C0784006C00F002830D11F48C0784006EF
:10F6C000C00F00282AD01A48C07840218843403013
:10F6D0001749C8701948C0784021884340301749FD
:10F6E000C8709321002001F03BFD1548C07840060A
:10F6F000C00F00280ED09320F1F79EFC012809D1FD
:10F700001048C0784021884340300E49C87001201D
:10F710000D49087093210748F1F7D1FC00BF05B0EF
:10F72000F0BC08BC04B018477B14AE47E17A843FB4
:10F73000C0080020B402002014000020DA080020D5
:10F7400022000020CC0800200800002010B5012174
:10F750000448F2F77DF9002204210348FBF710FC6E
:10F7600010BD000007000001800D004010B50446E8
:10F770000C480068C02188430A49086008460068B0
:10F78000C02108430749086007492046F0F7B2FC4A
:10F7900006490870084600787D21C900484304499D
:10F7A000088010BD0024004040420F00BA02002033
:10F7B000BC0200200146114A12884A43104B5A618C
:10F7C00000229A611A46126901231A430C4B1A61EE
:10F7D00000BF0B4A1069C207D20F002A04D00122D1
:10F7E00012040240002AF4D0054A1269520852005D
:10F7F000034B1A6100229A6170470000BC0200208E
:10F8000000E000E00146114A12784A43104B5A6169
:10F8100000229A611A46126901231A430C4B1A619D
:10F8200000BF0B4A1069C207D20F002A04D0012280
:10F8300012040240002AF4D0054A1269520852000C
:10F84000034B1A6100229A6170470000BA0200203F
:10F8500000E000E0F0B585B006460D4600200190BE
:10F86000288805284ED1707800020390B07803995B
:10F87000084303900398401C80B20390F078040280
:10F8800030790443012C3ADB7D200001844236DAD2
:10F89000374600202880012038707F1C2888401CB3
:10F8A00028806007400F002808D02046E117490F44
:10F8B0000918C910491CC9B2029106E02046E11797
:10F8C000490F09184905090E0291029838707F1CEA
:10F8D0002888401C2880002322463846039900F0DF
:10F8E0004BFC00900098002804D0009801F06AF8C2
:10F8F000019009E0298802980818288004E0032074
:10F90000019001E003200190019805B0F0BDF0B531
:10F9100085B006460D4600200190288805284DD167
:10F92000707800020390B07803990843039003981D
:10F93000401C80B20390F078040230790443012C1B
:10F9400039DB7D200001844235DA374600202880EB
:10F95000022038707F1C2888401C28806007400FD8
:10F96000002808D02046E117490F0918C910491C82
:10F97000C9B2029106E02046E117490F091849056E
:10F98000090E0291029838707F1C2888401C28803C
:10F9900022463846039900F0F3FB009000980028B7
:10F9A00004D0009801F00EF8019009E0298802982F
:10F9B0000818288004E00320019001E00320019052
:10F9C000019805B0F0BDFEB505460C46002001903B
:10F9D0002088052838D1687800020290A87802991A
:10F9E000084302900298401C80B20290E878060218
:10F9F0002E79012E25DB7D2E23DC2F460020208052
:10FA0000032038707F1C2088401C20807006000E68
:10FA100038707F1C2088401C2080002332463846E6
:10FA2000029900F0B1FB00900098002804D00098E3
:10FA300000F0C8FF019009E0208871004018208084
:10FA400004E00320019001E0032001900198FEBD35
:10FA5000FEB505460C46002001902088052838D1C7
:10FA6000687800020290A8780299084302900298F0
:10FA7000401C80B20290E878060228790643012EE5
:10FA800024DB7D2E22DA2F460020208004203870CF
:10FA90007F1C2088401C20807006000E38707F1C60
:10FAA0002088401C208032463846029900F09EFB98
:10FAB00000900098002804D0009800F083FF019087
:10FAC00009E0208871004018208004E003200190A4
:10FAD00001E0032001900198FEBDF0B587B0044617
:10FAE0000D460020029028880A2863DB6078000217
:10FAF0000690A0780699084306900698401C80B2AC
:10FB00000690E078060220790643607900020590AD
:10FB1000A0790599084305900598401C80B205908E
:10FB2000E0790702207A0743607A0490012E3FDBD8
:10FB30007D2E3DDC012F3BDB792F39DC79000498E9
:10FB4000814235D101233A4620460A30059900F01A
:10FB50001BFB01900198002822D1039428801720D4
:10FB6000039C2070039C601C03902888401C288004
:10FB70007006010E039801700398401C03902888BA
:10FB8000401C2880002332460699039800F0FCFAB6
:10FB900001900198002803D128887100401828801E
:10FBA0000198002806D0019800F00CFF029001E0B7
:10FBB00003200290029807B0F0BD000070B5054622
:10FBC0000C46064802880649681CF0F715FB0348F6
:10FBD0000088401C2080002070BD000056070020D7
:10FBE000101E0020FEB504460F4600200090388805
:10FBF00005282BD160780502A0780543681C85B2E2
:10FC0000207900281FD1E078FF2802D0E078002872
:10FC100019D1002069464871E078FF2802D10120FF
:10FC2000087102E000206946087101231A4629463E
:10FC300001A800F0A1FA0646002E09D0304600F0D7
:10FC4000C1FE009004E00320009001E0032000903A
:10FC50000098FEBDF8B504460F4600200090388895
:10FC6000052813D160780502A0780543681C85B289
:10FC700001231A462946E01C00F086FA0646002EAB
:10FC800006D0304600F09EFE009001E00320009078
:10FC90000098F8BDF0B585B005460E4600200190ED
:10FCA000308805283EDD68780702A8780743781C6D
:10FCB00087B2E878040228790443687903906007E2
:10FCC000400F002808D02046E117490F0918C91035
:10FCD000491CC9B2029106E02046E117490F0918F4
:10FCE0004905090E0291012C19DB7B200001844299
:10FCF00015DC03990298884211D101232246394626
:10FD0000A81D00F039FA00900098002804D000984F
:10FD100000F058FE019007E00520308004E0032049
:10FD2000019001E003200190019805B0F0BDFEB5FF
:10FD300004460E46002001903088062829DB6078B2
:10FD40000702A0780743781C87B2E0780502207983
:10FD5000054360790290012D18DB782D16DC6806CA
:10FD6000010E0298814211D101232A463946A01D75
:10FD700000F00AFA00900098002804D0009800F0E3
:10FD800021FE019007E00520308004E0032001906F
:10FD900001E0032001900198FEBD0000F8B5054682
:10FDA0000C4616461F4600200090002C03D0012C64
:10FDB00001DBF72C02DD0220009037E01C480470C4
:10FDC000002D20D11B481C4908601C481C490860B4
:10FDD0001C481D4908601D481D49086000201D4938
:10FDE00008601D481D4908601D481E4908601E48DE
:10FDF0001E4908603A4631460D480078069B00F0DF
:10FE0000DBF8009002E00220009000BF00BF0098E5
:10FE100000280BD102F00EF8002802D10320009038
:10FE200004E0134805700120124908700098F8BDDD
:10FE3000A006002035010100A80600205D01010098
:10FE4000AC0600206D000100A40600201500010092
:10FE5000B0060020B4060020011F0100B8060020F3
:10FE6000D11F0100BC0600208D1F0100C00600202C
:10FE7000A1060020A206002038B5002543480078DE
:10FE8000002801D0062038BD684601F0C1FF0128D6
:10FE900079D168460078012815D13D4A3D493E4850
:10FEA0003E4B1B6898470546002D0CD13A48007818
:10FEB0003B490978884203D037480078002802D1AE
:10FEC000022001F0BFFF684601F0A2FF01285AD1CD
:10FED00068460078022856D12E48006800783149DB
:10FEE0000870012030490870002418E0E0002F4914
:10FEF000085C002800D114E0E0002C49085C294986
:10FF0000097888420AD1E00028494018204942680F
:10FF10002048006890472449087002E0641C102CB7
:10FF2000E4DB00BF1C48007800282CD01E48007875
:10FF3000002819D00020164908801A48007880212E
:10FF4000084313490A880988491C114B1980114933
:10FF50000968885414480178184602880088401CB3
:10FF600018800C480068815411480078012800D19D
:10FF700000BF0748028807480168094800780D4B10
:10FF80001B689847054600207DE70000A206002078
:10FF9000520700204C07002050070020B006002028
:10FFA000A00600205107002054070020CC060020A6
:10FFB000A1060020A4060020F8B50E4614461F46F0
:10FFC000002000900120FFF729F83B460822214637
:10FFD000304601F04DFF012802D00320009011E0CF
:10FFE0004B200002844201D9232504E06100084827
:10FFF000F0F780F80546A8B201F066FF012801D0AD
:020000040001F9
:10000000032000900020FFF709F80098F8BD0000D9
:10001000A07F1700F8B504460D4616460020009054
:1000200000270120FEF7FAFF0E480088042813DBA2
:100030000C4801880C4801F0CFFE00280CD10A487A
:100040000078207007480088C01E30800648401C99
:1000500028600120009000E005270020FEF7DEFF69
:100060003846F8BD6E0700204E1E0020F8B5054644
:100070000E461746002000900120FEF7CFFF2848CB
:100080000078012844D1701E2649086001202649C5
:10009000088024480068057008460088C019088058
:1000A000084601881F48006801F096FE04461E4A73
:1000B0001088421C1C4B1A801C4A145421121A46E8
:1000C0001088421C1A80194A1154012018490870DE
:1000D0000EE014490968087801F0E0FE1148006854
:1000E000401C1049086010480088401E0E490880D6
:1000F0000D4800880028ECD1FF2101310B48F0F7B2
:1001000094F8002001F09EFE00200949087001E0EB
:10011000052000900020FEF781FF0098F8BD000048
:1001200065070020680700206C0700204E1E002095
:100130006407002010B50120FEF770FF002006497B
:1001400008700021012001F053FE01F053FE002051
:10015000FEF764FF10BD00006507002010B5012008
:10016000FEF75CFF0021084601F042FE01F041FE6F
:100170000020FEF753FF10BD10B50446012010BD4E
:100180000346012070470000F0B504461D460020DC
:10019000152903DB8F18242F00D8134E152920DBD7
:1001A0008F18242F1DD80B46153B002D02D0012D92
:1001B00016D10FE00BE05F00F75B3F122770641C65
:1001C0005F00F75B2770641C5B1C571EBAB2002AE5
:1001D000F1DC05E002E05B1C571EBAB2002AFADC33
:1001E00000E00120F0BD0000301E002070B5034685
:1001F00000207D25ED00A94218DB8D18FB26B600F6
:10020000B54213DC0A4D2D884C1B0CE06500094EED
:10021000755B2D121D705B1C6500755D1D705B1C90
:10022000641C551EAAB2002AF0DC00E0012070BD5B
:100230005A0700205C070020FFB5FFB0FFB085B073
:1002400007461C460021FFA8C1600121890202A8BF
:10025000EFF7EBFF0221019100264802844204DD02
:1002600000207FB07FB009B0F0BD00BFFCF708FCF4
:10027000F2F730FA0121C9025048F3F714FB00BF2E
:1002800040214E48F3F70FFB012189034B48F3F758
:100290000CFB00BF00BF00261FE00121890202A85D
:1002A000EFF7C3FF2246FFA8416902A8F2F76EFAF2
:1002B000A21E02A90231424801F074FD05466846BB
:1002C000407A01026846007A0918A94203D1012048
:1002D000FFA9C86003E0701CC6B2022EDDDB00BFC0
:1002E00000BFFCF739FCF2F723FA00BFFFA8C06893
:1002F000012807D100232246394602A8FFF705F856
:100300000120AEE700BFFCF7BBFBF2F7E3F90121E8
:10031000C9022A48F3F7C7FA00BF40212748F3F77C
:10032000C2FA012189032548F3F7BFFA00BF00BFD5
:1003300000261FE00121890202A8EFF776FF22467E
:10034000FFA8816902A8F2F721FAA21E02A90231D0
:100350001B4801F027FD05466846407A01026846C1
:10036000007A0918A94203D10120FFA9C86003E05F
:10037000701CC6B2022EDDDB00BFFFA8C0680128DA
:1003800013D100232246394602A8FEF7BEFF2246BB
:10039000FFA8416902A8F2F731FA00BFFCF7DCFBC5
:1003A000F2F7C6F900BF01205BE700BFFCF7D4FB02
:1003B000F2F7BEF900BF002053E70000800C0040B8
:1003C000FFFF0000F8B506460F4614461D46012003
:1003D00000902A463946304600F01CF8002807D124
:1003E0002A463946304600F015F8002800D1009022
:1003F0002A462146304600F00DF8002807D12A464B
:100400002146304600F006F8002800D10090009800
:10041000F8BD704770B5FFB0FFB082B005460E461C
:10042000144601208002844204DD00207FB07FB0AA
:1004300002B070BD00BFFCF723FBF2F74BF90121BE
:10044000C9021248F3F72FFA00BF40210F48F3F713
:100450002AFA012189030D48F3F727FA00BF00BFEC
:10046000224631462846F2F7C9F922463146684607
:10047000F2F78CF900BFFCF76FFBF2F759F900BFF8
:1004800022466946284601F061FACFE7800C004019
:1004900010B5002823D0124B0022001F196803E07A
:1004A000814203D80A4649680029F9D1002A0AD0B6
:1004B0001368841A9C4204D1006818181060104612
:1004C00002E0506000E01860002907D002680B1AB3
:1004D000934203D10B68D21802604968416010BD95
:1004E0007807002001460148405C70475221010016
:1004F00001460148405C70475220010010B5FEF7EC
:10050000A1FEFCF7BDFA10BD10B50121490251480A
:10051000F3F7BFF9002803D14F480078401C00E0F2
:1005200000204D4908700121C9034A484030F3F7C3
:10053000B0F9002803D149480078401C00E00020B1
:10054000464908700121890342484030F3F7A1F978
:10055000002803D142480078401C00E000204049B8
:1005600008704048C088002802D108703B490870D4
:100570003A480078052815D10020384908703A48D3
:100580000078012803D10220374908700AE0364874
:100590000078022803D101203349087002E00120CD
:1005A000314908702C480078002816D12B48007873
:1005B000002812DD2A48007800280ED101202B499E
:1005C00008702848C088002807DD00BF1E21254884
:1005D000C18000202349087100BF1F48007800280F
:1005E00016D11E480078002812D11D480078002836
:1005F0000EDD01201D4908701A48C088002828DD3A
:1006000000BF1E211748C18000201649087120E054
:100610001148007800281CD110480078002818DD07
:100620000F480078002814DD0120104908700D489B
:10063000C088002807DD00BF1E210A48C1800020B5
:100640000849087100BF01200949087002200949C2
:10065000087010BD000D0040D2020020D30200201F
:10066000D40200209A0200207B0600207906002098
:10067000B0020020B102002010B50020154908701A
:100680001548C08800280BDC144800784007400F4C
:10069000012805D0114840788007C00F00280ED0EF
:1006A0000F480078012804D100200D490870F9F79F
:1006B000F7FAF9F769FA00200A49087008E00948D2
:1006C0000078002804D1012006490870F4F784FE60
:1006D00010BD0000790600209A020020C00800200A
:1006E0007A0600207E06002010B501210448F1F7AB
:1006F000AFF90022FF2101310248FAF741FC10BD99
:1007000007000001C00C004010B501210448F1F7BA
:100710009FF9002280210348F4F7C5F810BD0000BE
:1007200007000001800D00401CB5FDF7B5F8FFF78C
:10073000E5FE01F087F800F0FFFFFEF707FDF4F794
:1007400033F8FFF799FFA7E05448007801287DD1DE
:10075000002052490870F4F727F85148F3F79CFD40
:1007600000283ED14F4840794006C00F002838D0BD
:1007700000BF4D4840794006C00F002830D149489D
:1007800040794006C00F00282AD0474840794021D0
:100790008843403044494871444840794021884367
:1007A0004030424948711821002000F0D9FC4048EF
:1007B00040794006C00F00280ED01820F0F73CFC0E
:1007C000012809D13B4840794021884340303949CC
:1007D000487101203849087018213848F0F76FFC3B
:1007E00000BFFFF791FEFFF747FF01F0E3F9FAF7CB
:1007F00025FE2B48017868460170294841786846F3
:10080000417027488178684681702548C1786846DC
:10081000C1702348017968460171214841796846D1
:1008200041712748019A009900F094FE244800F095
:10083000D3FBFCF70DFB1A48017868460170184895
:100840004178684641701648817800E01EE06846AD
:1008500081701348C1786846C170114801796846B3
:1008600001710F484179684641710199009800F083
:100870007BFC1448F3F732F8114801F0BDFAFAF79F
:10088000A9FAFCF7F1FE0E48FEF712F90E480078BF
:10089000012801D1FFF7F0FE56E700009802002082
:1008A000CC02002014000020C0080020DA0800203C
:1008B00022000020CC08002008000020B402002004
:1008C000AA020020DE02002079060020F0B50B30DD
:1008D000C108C900144F0026144A0FE003688B4278
:1008E0000BD38B4205D95C1A4318456830C3083BCB
:1008F00000E04368136002C004E0021D1068002895
:10090000ECD13046002803D13868002801D00020FF
:10091000F0BD064A06481060064A121AD208D200F4
:1009200044C001203860D7E77C070020780700200A
:10093000541F0020502F0020F8B504460E461546DF
:100940002078B04202D16078032801D00020F8BDA1
:10095000A07828702878FA2801DD0020F7E72878A9
:10096000001D275C39022878C01C205C081887B25B
:100970002878C21C2146044801F014FAB84201D07C
:100980000020E4E70120E2E7FFFF0000FFB581B0AF
:1009900004460F461D46AA1EA11C094801F002FA92
:1009A00006462670301260702B4639462046039A60
:1009B000FFF708FD002801D105B0F0BD0120FBE7DD
:1009C000FFFF00000146002904D0012904D00729B7
:1009D00006D103E0002005E0022003E0062001E04C
:1009E000042000BF00BF70470FB470B5469E459D00
:1009F00040A8008A062804DA002070BC08BC04B0B5
:100A0000184700210CE004A8405C002802D004A88C
:100A1000441807E0402901DD0020EEE7481C81B2C0
:100A2000FF29F0DD00BFFF210531681A8D4218D083
:100A300008DCE81FFA3800280DD001280DD0022864
:100A400021D10CE0FC2813D0FD2813D0FF38FD384D
:100A5000002818D110E00020CFE70020CDE70020CB
:100A6000CBE731462046489B479AFBF7EFFEC4E7A9
:100A70000020C2E70020C0E731462046489B479A45
:100A8000F1F778FFB9E70020B7E7000070B500255F
:100A90000026FBF765FD04215948F2F7FAFE0546EA
:100AA0000CE0701CC6B20A20FEF784FE04215448F4
:100AB000F2F7EFFE05460A2E00DD01E0002DF0D131
:100AC00000BF002D01D0002070BD4E48407B0028A3
:100AD0001BD10121C9024A48C038F2F7E6FE0121C4
:100AE00009034748C038F2F7DEFE0120FEF762FE38
:100AF000012189034248C038F2F7D5FE0121C9031C
:100B00003F48C038F2F7CFFE5BE03E48407B01280B
:100B10001AD1C1023A48C038F2F7C7FE01210903D1
:100B20003748C038F2F7BFFE0120FEF743FE01212F
:100B300089033348C038F2F7B8FE0121C9033048B1
:100B4000C038F2F7B0FE3CE02E48407B02281AD1B4
:100B500081022B48C038F2F7A8FE0121090328487A
:100B6000C038F2F7A0FE0120FEF724FE0121890320
:100B70002348C038F2F797FE0121C9032048C03846
:100B8000F2F793FE1DE01F48407B102819D1C101E8
:100B90001B48C038F2F787FE012109031848C03806
:100BA000F2F783FE0120FEF705FE012189031448B8
:100BB000C038F2F778FE0121C9031148C038F2F7B6
:100BC00072FE0120FEF7F6FD012149030C48C038F2
:100BD000F2F76BFE0B490A79CB78110219430846EC
:100BE00000F0C0F9044600200749C87008710320CE
:100BF000487088700846047101204871022063E73C
:100C0000000D0040720300208906002070B53348B3
:100C10000079002804D031480079401E2F4908711E
:100C20002E480079002856D12D48C07A0300FEF7DF
:100C3000D8F90906090C0F121D15171A1D004B24AF
:100C4000240116E04B24640113E04B24A40110E0BE
:100C50004B24E4010DE04B2424020AE0214C08E07F
:100C6000E124240205E0E124640202E04B24E401D3
:100C700000BF00BF1A48007B002804D0012804D020
:100C8000022806D103E0002505E0022503E0012546
:100C900001E0002500BF00BF002229462046FBF7E7
:100CA00045FDFBF7BFFC00200F4948700121C90337
:100CB0000E48F2F7FAFD0A20FEF7A4FD084A917BE0
:100CC0001379D6781A023243104600F0C7F9032090
:100CD0000249887070BD0220FCE7000089060020F0
:100CE00072030020C0DA0000BE020020000C0040A9
:100CF00010B5FFB085B000248D484078012804D19C
:100D000000208B494870FBF7D5FC8A488078012881
:100D10003ED10021874881708748017880A8017200
:100D20008548417880A841728348817880A8817283
:100D30008148C17880A8C1727F48017980A8017379
:100D40007D48417980A841737B48817980A881736F
:100D5000072282A93FA8EFF74FFA0120FF210531B2
:100D6000F4223D913E907349F0396846EFF744FA1A
:100D7000FF220532714941A8EFF73EFA41A80FC89A
:100D8000FFF732FE0446FF2101316C48EFF74DFAC0
:100D9000012C47D1684840796749897988423ADB14
:100DA000E1036748F2F77FFDA1036548F2F77BFD99
:100DB000610363484030F2F776FDE102604840305D
:100DC000F2F771FD21035E484030F2F76CFDA1039C
:100DD0005B484030F2F767FDE10359484030F2F7D5
:100DE00062FDFBF7ABFB00BF564840798007C00FA0
:100DF000002809D05348407902218843514948715D
:100E000085215148F0F75AF900BF00204F4908707A
:100E10007FB005B010BD48484079401C4649487134
:100E20000220F5E744488078401EC0B242498870ED
:100E300000287BD108464078401EC0B24870002888
:100E400072D10121C9033E48F2F72DFD012189032A
:100E50003B48F2F728FD0121490339484030F2F7B9
:100E600022FD0121C90236484030F2F71CFD012164
:100E7000090333484030F2F716FD01218903304859
:100E80004030F2F710FD0121C9032D484030F2F740
:100E90000AFDFBF753FB2D480078FA2840DA2B486F
:100EA0000078401CC0B229490870012838DB00BF17
:100EB000244840798007C00F002830D12448407969
:100EC0008007C00F00282AD01E484079022188439D
:100ED000801C1C4948711F48407902218843801CAE
:100EE0001C4948718521002000F03AF91A484079E0
:100EF0008007C00F00280ED08520F0F79DF801284C
:100F000009D11648407902218843801C1349487151
:100F100001201349087085210B48F0F7D0F800BF75
:100F2000002075E702E0FFE7022071E703206FE78A
:100F3000BE020020AA1D002089060020AA1C002055
:100F4000000C0040C0080020B402002090060020E1
:100F500014000020DA08002022000020CC08002025
:100F6000080000200146FF220532881A91421ED057
:100F700008DCC81FFA3800280DD001280FD002283D
:100F800026D110E0FC2816D0FD2818D0FF38FD38F7
:100F900000281DD117E001200E4A907170470120F2
:100FA0000C4A9071FAE701200A4A9071F6E7012095
:100FB000084A9071F2E70120064A9071EEE701209D
:100FC000044A9071EAE70320024A90710120E5E7A4
:100FD0006420E3E78906002010B504462078012844
:100FE0000ED1607900280BD1E078002808D120705C
:100FF00018480078002803D1012016490870607055
:1010000014480078002806D0012805D0022808D00E
:10101000032810D10AE00FE0FFF738FD0D490870F2
:101020000AE0FFF7F3FD0B49087005E0FFF760FEEB
:101030000849087000E000BF00BF0648007800289B
:1010400007D16078012804D1002060700120024996
:10105000087010BD89060020FA02002070B5054610
:101060000C46FF210531681A8D4215D008DCE81FB7
:10107000FA3800280DD001280CD0022835D10AE01A
:10108000FC2810D0FD280FD0FF38FD3800282CD1C7
:101090000BE02BE02AE029E03122FF21F631204647
:1010A00000F028F822E021E020E0114840790128F2
:1010B00005D104226421204600F01CF814E00C48FD
:1010C0004079022806D10422FF213331204600F066
:1010D00011F809E006484079032805D10422FF21D0
:1010E0004731204600F006F800E000BF00BF70BDA9
:1010F00089060020FEB506460C4615466846067071
:101100000321417021128170C4702912017145714F
:10111000062269460F4800F045FE0746684687717B
:101120003912C17100BF012189030B48F2F7BDFBE1
:10113000082269460948FCF7DCFE0A20FEF762FB3C
:10114000012189030448F2F7AEFB00BFFBF79AFACE
:10115000FEBD0000FFFF0000000C004000680140E1
:10116000024600207047000013B582B000200190B5
:101170003E4840788007C00F002805D03C49C87C15
:10118000897C04020C4304E03949487C097C040250
:101190000C4301AB224603990298F3F701FC0128A6
:1011A00001D1344908706846007B002806D16846A2
:1011B000407B002802D101202F4908706846C07A80
:1011C00000280AD16846007B002806D16846407B8B
:1011D000002802D10120294908706846807A012838
:1011E0000ED16846C07A00280AD16846007B0028E4
:1011F00006D16846407B002802D1012020490870B2
:101200001C480078012807D11E484078002803D1E7
:101210001849087000F038F817480078012808D1FC
:1012200018484078002804D113490870012000F0C4
:1012300087F912480078012808D112484078002820
:1012400004D10E490870022000F07AF90C480078A9
:10125000012808D10B484078002804D108490870BB
:10126000032000F06DF9F3F747F91FBDC008002017
:10127000E703002001030020FE020020FF020020FF
:1012800000030020AA02002030B595B000230622FA
:1012900000A902319E48FEF738F89E4A0020014618
:1012A0001578284355782D02284395782D04284336
:1012B000D5782D0628431579294355792D022943E0
:1012C00095792D042943D27912061143034602AAC7
:1012D000EEF7EBFF8F4A08320020014615782843CD
:1012E00055782D02284395782D042843D5782D066E
:1012F00028431579294355792D02294395792D04E1
:101300002943D27912061143034604AAEEF7CDFF12
:101310008148806B06908048C06B07907E48006CC7
:1013200008907D48406C09907A4931310A7810461E
:101330004A78120210438A7812041043C9780906C9
:1013400008430A90734A3532002001461578284335
:1013500055782D02284395782D042843D5782D06FD
:1013600028431579294355792D02294395792D0470
:101370002943D2791206114303460BAAEEF795FFD3
:10138000644A4532002001461578284355782D02DD
:10139000284395782D042843D5782D0628431579C0
:1013A000294355792D02294395792D042943D27972
:1013B0001206114303460DAAEEF777FF554A3D3258
:1013C000002108461578294355782D022943957840
:1013D0002D042943D5782D062943157928435579BD
:1013E0002D02284395792D042843D2791206104303
:1013F0000B4601460FAA1846EEF757FF4748EEF78F
:1014000033FF05464649EEF7B8FF0446EFF727FAE3
:10141000C1B210A801714148401F417D10A841711F
:101420003E48401DEEF720FF05463D49EEF7A5FF7B
:101430000446EFF714FAC1B210A881713748401F73
:10144000817D10A8C17100230C2212A93548FDF737
:101450005CFF522200A90231334800F0A3FC694628
:10146000088000BF3148EEF7FFFE04467D23DB0015
:1014700054222F49F1F7ACFB002808D12B492C4806
:10148000EEF70AFF00212948801F0171417100BF5A
:101490002648EEF7E9FE0446542221466846F1F755
:1014A00029FC00BF2148EEF7DFFE2249884209D21D
:1014B0001E48EEF7D9FE044654341C492046EEF788
:1014C000EBFE03E019491A48EEF7E6FE1748801FC5
:1014D00041790279080210437D21C90088420CD26B
:1014E0001248801F4179027908021043401C81B2E2
:1014F0000E48801F0171090A417100BF5A230E4A2C
:101500000E490A484638FFF741FA15B030BD0000D1
:10151000CC02002052120020B01D0020E302002067
:1015200000002041C0080020FFFF0000210500202E
:1015300000581400CC9F1500984C00009810000033
:10154000704710B50446002010BD10B503460020BA
:1015500010BD000037B582B00446002001906846F7
:10156000007C002806D16846407C002802D1042077
:101570006B4908706846C07B00280AD16846007C29
:10158000002806D16846407C002802D10420644926
:1015900008706846807B01280ED16846C07B002811
:1015A0000AD16846007C002806D16846407C0028A5
:1015B00002D104205A4908705A4840788007C00F69
:1015C000002805D05849C87C897C05020D4304E0F9
:1015D0005549487C097C05020D4301AB2A46049914
:1015E0000398F3F7DDF9012802D104204C49087073
:1015F0004E480078002802D0032049490870484826
:101600000078002807D0002045490870607800283D
:1016100001D1012020704448007DC007C00F002880
:1016200023D000201CE00C2800DB1DE06946CA7BAB
:1016300043003D491C31C95C8A420FD169460A7C8E
:10164000430039491C31591849788A4206D1694604
:10165000497C002902D10121344A1170411C88B211
:101660003149C97E8142DEDC00BF2F48007D022166
:10167000084002281CD12B4840788007C00F002862
:1016800005D02948017EC27D0D02154304E026489D
:10169000817D427D0D021543234B19332A4604995F
:1016A0000398F3F77DF9012802D105201F4908703E
:1016B0001F49C87A897A00020843002818DD1C49AE
:1016C000487B097B00020843002811D117480078A5
:1016D00000280DD10620154908701549C87A897A65
:1016E00000020843401E81B211488172090AC1728A
:1016F0000E480078002811D00C4800780C4908707A
:1017000000200A490870A078002807D1E078002856
:1017100004D10320074948700120A07005B030BDF6
:10172000B0020020C0080020E7030020B102002022
:10173000071B0020DE0200200EB53C480078102177
:1017400088433B4989798906C90F0122514051409C
:101750000901102211400843344908703549C978FD
:10176000012900D100E00021C800082210402F49C3
:101770008978914301432D4A9170104680788021E9
:1017800088432B4989794907C90F012251405140AB
:10179000C901802211400843244988700846C07856
:1017A000800880002249C9790906890F08431F492A
:1017B000C87008460078C008C0001D49497849072C
:1017C000490F084319490870FBF730FB1A48F2F734
:1017D00063FD002821D11948C07918498979174A31
:1017E0005279164B0092019102901A79D978987823
:1017F0000123FBF7E7FA00280FD10F4840790E4983
:1018000009790D4AD2780C4B0092019102909A7896
:10181000597818780123FBF7D5FA09490879FDF7BB
:1018200023F8F9F7E7FBFAF7F1F80EBDC00800203E
:101830000A000020F9120020CC0200204A120020E9
:101840004C03002010B596B02C210BA8EEF7EDFC50
:101850002C216846EEF7E9FC012400BFFBF710F9E4
:10186000F0F738FFE1021E48F2F71DF800BF4021F3
:101870001B48F2F718F8A1031948F2F716F800BF51
:1018800000BF2A2221020BA8F0F780FF0BA802302C
:10189000EEF7EAFC1349884200D10FE02A223D21ED
:1018A00009026846F0F772FF00A80230EEF7DCFC90
:1018B0000C49884201D1012400E00024002C02D10F
:1018C000FDF7D4FC01E0FDF709FDFDF7E7FC00BFE3
:1018D000FBF742F9F0F72CFF00BF16B010BD000077
:1018E000800C00400506062410B50C490C48EEF7A4
:1018F000D3FC0A49091D0A48EEF7CEFC202107480F
:101900000830EEF792FC2A233D221202FF2101311A
:101910000248801EFFF73AF810BD000004030020C3
:101920000506062410B52A233D221202FF210131AB
:101930000548FEF781FC002803D1FFF7D5FF002002
:1019400010BD0120FCE700000203002070B5034633
:101950000C460021002000BF07E05D5C665CB542DC
:1019600001D0002003E04D1CA9B29142F5DB00BF7D
:10197000914200D1012070BD00B58DB00121144805
:10198000F0F766F80120F0F761FC0221684601716A
:1019900008030390801004900520000205900020A9
:1019A00006900C4802900C480990002007900021F6
:1019B00008A8417081700121C1701520F9F726F93E
:1019C0000220F0F775FC01A8F0F77AFC0DB000BD1D
:1019D00004000002FF030000E809002010B5022007
:1019E000F0F766FC00210220F0F7FAFB01218902E2
:1019F0000548EEF71AFC04490220F0F71FFC01210C
:101A00000220F0F7EDFB10BDE8090020F8B505460F
:101A100000270220F0F70AFC06461C48864216D032
:101A20000220FDF7C7FE0CE00220F0F7FFFB0646A0
:101A30000220FDF7BFFE3846791C8FB2642800DD16
:101A400004E00220F0F7F2FBB042EDD100E0F8BD77
:101A50000E48301A84B2002C15DD01208002844229
:101A600011DC844201DA844200DBF0E72C70200AAA
:101A7000687000232246A91C0448FDF746FC01209B
:101A800081026918887000BFE1E70000E8090020C2
:101A900070B58AB006460C46154601211F48EFF77F
:101AA000D7FF0022012149021D48EFF775FC0022F3
:101AB000FF2101311A48EFF76FFC00220121890252
:101AC0001748F9F75DFA012189021548F1F7EBFE95
:101AD000079608A84470002C03D1012008A90870BB
:101AE00002E0022008A9087008A885706846EFF790
:101AF0006BFE6A4607A90B48FCF720F80E20F9F7A1
:101B000085F801210748FCF73CF901210548FCF75D
:101B10006AF90448FCF7CBF90AB070BD0700000170
:101B2000000C00400078014038B52048C078030020
:101B3000FDF757FA0906090C0F121D15171A1D009B
:101B40004B24240116E04B24640113E04B24A40130
:101B500010E04B24E4010DE04B2424020AE0144C75
:101B600008E0E124240205E0E124640202E04B24C1
:101B7000E40100BF00BF0D480079002804D001280F
:101B800004D0022806D103E0002505E0012503E08A
:101B9000022501E0002500BF00BF044800958178C0
:101BA000234600221046FEF7F9F838BDE203002074
:101BB000C0DA000070B5734840788007C00F002875
:101BC00002D07148FFF722FF7048807801287DD14C
:101BD0006D4800880C2879DD6B4880786828F6D13C
:101BE00069480088801E84B26748801C005D00023E
:101BF0006549891C621C895C084305462246624986
